S01700004B32324642657A63616C6D61785631332E533139B7
S3450000000000000120C50100000D020000D1440000110200001302000015020000000000000000000000000000000000001702000019020000000000001B0200001D02000000
S345000000402D290000352900003D290000452900004D290000552900005D290000652900006D290000752900007D290000852900008D290000952900009D290000A52900005A
S34500000080AD290000B5290000BD290000C5290000CD290000D5290000DD290000E5290000ED290000F5290000FD290000052A00000D2A0000152A00001D2A0000252A000015
S345000000C02D2A0000352A00003D2A0000452A00004D2A0000552A00005D2A0000652A00006D2A0000752A00007D2A0000852A00008D2A0000952A00009D2A0000A52A0000CA
S345000001005D1D0000AD2A0000B52A0000BD2A0000C52A00009D1F0000CD2A0000D52A0000DD2A0000E52A0000ED2A0000F52A0000FD2A0000052B00000D2B0000152B0000E6
S345000001401D2B0000252B00002D2B0000352B00003D2B0000452B00004D2B0000552B00005D2B0000652B0000000000006D2B00007D2B0000852B00008D2B0000952B0000D9
S34500000180752B000000000000484B00000000002064010000484B00000000FF1F00000000484B0000000000140000000000020020280B00000000FF1F0000000000000014A2
S345000001C00000000038B572B602F0C4F90C4C0D4DAC4206D30C4DAC420AD362B604F09BF9FEE7D4E90001A2680C3400F019F8EFE754F8080B54F8041C00F01BF8EBE700BFD5
S3450000020088010000AC010000C4010000FEE7FEE7FEE7FEE7FEE7FEE7FEE7FEE7FEE7FEE710B50023934200D310BD1C585C500433F8E700231A468B4200D370471A500433BD
S34500000240F9E7FFFFFFFFFFFFFFFFFFFFFFFFFFFFFFFFFFFFFFFFFFFFFFFFFFFFFFFFFFFFFFFFFFFFFFFFFFFFFFFFFFFFFFFFFFFFFFFFFFFFFFFFFFFFFFFFFFFFFFFFFFFFD6
S34500000280FFFFFFFFFFFFFFFFFFFFFFFFFFFFFFFFFFFFFFFFFFFFFFFFFFFFFFFFFFFFFFFFFFFFFFFFFFFFFFFFFFFFFFFFFFFFFFFFFFFFFFFFFFFFFFFFFFFFFFFFFFFFFFFF78
S345000002C0FFFFFFFFFFFFFFFFFFFFFFFFFFFFFFFFFFFFFFFFFFFFFFFFFFFFFFFFFFFFFFFFFFFFFFFFFFFFFFFFFFFFFFFFFFFFFFFFFFFFFFFFFFFFFFFFFFFFFFFFFFFFFFFF38
S34500000300FFFFFFFFFFFFFFFFFFFFFFFFFFFFFFFFFFFFFFFFFFFFFFFFFFFFFFFFFFFFFFFFFFFFFFFFFFFFFFFFFFFFFFFFFFFFFFFFFFFFFFFFFFFFFFFFFFFFFFFFFFFFFFFFF7
S34500000340FFFFFFFFFFFFFFFFFFFFFFFFFFFFFFFFFFFFFFFFFFFFFFFFFFFFFFFFFFFFFFFFFFFFFFFFFFFFFFFFFFFFFFFFFFFFFFFFFFFFFFFFFFFFFFFFFFFFFFFFFFFFFFFFB7
S34500000380FFFFFFFFFFFFFFFFFFFFFFFFFFFFFFFFFFFFFFFFFFFFFFFFFFFFFFFFFFFFFFFFFFFFFFFFFFFFFFFFFFFFFFFFFFFFFFFFFFFFFFFFFFFFFFFFFFFFFFFFFFFFFFFF77
S345000003C0FFFFFFFFFFFFFFFFFFFFFFFFFFFFFFFFFFFFFFFFFFFFFFFFFFFFFFFFFFFFFFFFFFFFFFFFFFFFFFFFFFFFFFFFFFFFFFFFFFFFFFFFFFFFFFFFFFFFFFFFFFFFFFFF37
S34500000400FFFFFFFFFFFFFFFFFFFFFFFFFEF9FFFF2DE9F0414B688AB04FF000080133CDE9048805460E4617468DF80F8003D105200AB0BDE8F081002AF9D0946806210DF1EF
S345000004400F0202F0A7FE317A002977D07368082BEDD13368002BEAD05A88D88862809A88A280E0805A7862701B78237013F0600F16D10C2A60D8514B53F82260002E5BD04C
S3450000048005AB04AA21463846B04705AB019304AB0093002302462146284602F0B3FCC7E703F0200248B31F0627D4BAB10121089006AA2846CDF81C808DF82410069400F0D0
S345000004C0C3F8089B0593079B04930028DDD10146E388049A284602F0F1FDA9E75E062BD5002307930890012306AA132128468DF82430069400F0E2F8E3E77AB1002301211D
S34500000500089006AA284607938DF82410069400F09BF8089B0593079B0493B6E759060BD507920123089006AA132128468DF82430069400F0C3F8ECE70520A6E79DF80F3021
S34500000540032B09D162781D4B214653F82250384605AB04AAA8476BE77368002B3FF467AFE288002A3FF463AF94F9000022780028FFF65DAF12F0200010D0326807928DF8B8
S34500000580241006AA012128460694089300F05CF805AB019304AB009301237BE752060BD5326807928DF8240006AA132128460694089300F083F8EBE70520E9E7C049000066
S345000005C070B5124B86B0CDE903314023ADF804308026012303AA01A90546ADF80660ADF8083002F079FD044660B98DF8060003AA01A9284602F070FD044618B13146284651
S3450000060002F089FD204606B070BD00BF11040000054B1A6832B19A7B824202BF0022C3E900229A73704700BF00040020054A13682BB1927B824202D10B6000207047042089
S34500000640704700BF000400202DE9F0478A4614461AB1184F3B68984222D004231846BDE8F087002309EB031340689B6822465146984705280346F1D0002808BF00250136E9
S345000006807A68107AF3B2984211D9106808FB030083681B79032BE4D0002BF0D10123E1E7DFF81490002601254FF00C08E8E72B46D4E700BF00040020F44900002DE9F0412C
S345000006C00D4E3368984204460D46174611D1012907D13146FFF774FF324602212046FFF7B3FF73683A46294620465B68BDE8F04118470420BDE8F081000400202DE9F047EA
S3450000070006469046002A45D0002943D04B68002B40D0214D2B683BB1AC7B844214BF022401242046BDE8F0871C4BA873C5E901132A461B4900F036F8044630B1286802F0CB
S34500000740A6FC3046FFF764FFEBE782464FF00C096B681A7A5FFA8AF18A4217D909FB01F7196839448B681B79032B03D10A1D304600F040F96B68196839448B681B7913B9B0
S345000007800A1D304698470AF1010AE1E72B68C8F80030C6E70424C4E70004002010040020BD060000F8B51746002A34D01B4C23683BB194F86D30834214BF02250125284639
S345000007C0F8BD84F86D00A16084F86C3084F86F3022460826013EC2E90333137502F10C02F8D1012804D9266084F86D600625E6E70B4B63603C606368084A1B6811469847C1
S34500000800054620B1054802F042FC3E60D7E7022384F86E30D3E70325D1E700BF18040020144A000070B542EA410400EB041404F1280694F82D4044F040047471456825F4B3
S34500000840FF7424F0010444EA021242EA41147279C2F3001244EAC202536072790B4BC2F3001144EAC1040499C2F3C00203EA014343EA821343F088038268236092F8943052
S3450000088003F0DF0382F89430002070BD0000FF03F8B50E461746044618BB134D134B144AEA61FF2285F8A200AB60012183F880200246284602F046FE0E4BAA686B60C3F38E
S345000008C0072182F89C10C3F307411B0E82F8B010284682F8B43002F0C9FC3D602E602046F8BD0624FBE700BFC80400200020074088040020000200202DE9F04390F89430F9
S3450000090087B004461BB9012007B0BDE8F0834268926851799942F6D31268002AF3D003F10053013B02EBC30612F833500C2700239D42E8D9706807FB03F28118825C082ABF
S345000009402CD10D7A00239D421DD80027CB7884F89530002FD7D00026DFF89080DFF89090A760012035463B79B34219D80123E560C4F88450C4F8883084F88C5084F88F5014
S3450000098084F89650C0E748681A0100EB0317805C94F893209042D9D00133D4E70133C7E7B9688DF8085006237343CA18013610798DF80900CB5C8DF806305188ADF8041070
S345000009C052788DF80720DA09206814BF84F8913084F8923003AA01A914BFCDF80C90CDF80C80049402F078FBBDE700BFCD0B00008D0A0000F8B51E4C25680F461646002D95
S34500000A0034D11C4BA3611C4BE3611C4B23621C4BE3631C4B236421461B4B2365FFF706FE30B1C4E9005584F8945084F89350F8BD236833B9606084F8940084F893000320EF
S34500000A40F5E7FF2384F89330236A84F894007022606167601A700A22DA7198701873587384F88D0084F88E003460E0E70220DEE79005002050060020700600203C060020A5
S34500000A8028060020300600206C0500207FB54B6814465A1C0E462CD194F88530A3B163681D688DB1A269D37B03F07F03282B0BD100230968029101930093537B8DF80C30F6
S34500000AC06A4601212046A84794F89650012D03D00125284604B070BD002384F89630E26994F8911020680D2302F0E2FAA4F88E50EFE7E26894F88B5093429CBFD21AE2601F
S34500000B00012D0CD1002394F89110206884F88B3084F8865084F8853002F01CFBD9E794F88520BAB90D2BD3D10B681968264B9942CED1012584F88E2094F89210A2692068D9
S34500000B4084F888501F2302F0B9FA84F88D50C0E701252AE062681568002DB9D001933368029323690093A3695A7B8DF80C20DB7B03F07F03282B03D16A4601212046A84779
S34500000B80E368002BE4D0A3695A7B736804EB02122046926DB3FBF2F223691344236103F0C7F8E3680546002B93D1002384F88530012384F88E30E26994F8911020680D232F
S34500000BC002F076FA85E700BF555342537FB514464A68531C0E462CD194F88430A3B163681D688DB1A269D37B03F07F032A2B0BD100230968029101930093537B8DF80C3027
S34500000C006A4602212046A84794F88D50002D40F0B581B4F886304BB91F23A26994F89210206802F04BFA012384F88D30284604B070BDE3689A429CBF9B1AE360A369DB7B62
S34500000C4003F0BF03152B06D163681B681BB100220B212046984794F88C30012B0CD1002594F89210206884F8873084F88450A4F88C5002F06FFAD9E794F88450002D37D01F
S34500000C80736801933368029323690093A3695A7B8DF80C2062681568CDB1DB7B03F07F032A2B03D16A4602212046A847E5688DB1A3695A7B736804EB02122046926DB3FBA0
S34500000CC0F2F223691344236103F06FF80546E368002BABD1002384F884300D23E26994F89110206802F0E4F9012384F88E309DE794F88830002B00F0288173681F2B40F07B
S34500000D002481A3699E4A1968914240F01E815E7B16F0F00F40F01981997B11F0E00240F0148194F890000130864280F00E8101390F2900F20A81E16984F88D209148E260FC
S34500000D40086058688A60486084F8882093F90C009E68197B002802DB321E18BF0122002884F8842008DA3EB194F88620012084F8850022B1054659E7002284F88520DB7BAA
S34500000D80032B04D0226A0020907010735073CA092F2B666284F839204ED8112B09D8032B66D0042B70D0002B66D0204603F01BFB58E0123B1D2BF8D801A252F823F000BF2D
S34500000DC05F0E0000AB0D0000AB0D0000990E0000AB0D0000AB0D0000AB0D0000AB0D0000470E0000B90E0000AB0D0000A90E0000810E0000AB0D0000AB0D0000AB0D000047
S34500000E00AB0D0000A10E0000AB0D0000910E0000AB0D0000AB0D0000690E0000AB0D0000570E0000AB0D0000AB0D0000AB0D0000AB0D0000B10E00009E2B29D007D8552B2A
S34500000E402AD05A2BB1D1204603F0AFF90AE0A82B0AD0AA2BA9D1204603F056F902E0204603F009F9054636E0204603F028F9F9E7204603F0DFF8F5E7204603F06BF9F1E743
S34500000E80204603F049FAEDE7204603F026FAE9E7204603F0DAF9E5E7204603F0AAF9E1E7204600F075F8DDE7204603F056FAD9E7204603F070F9D5E7204603F06FFAA3697B
S34500000EC01B7D05463BB9304A137843F0010313702E4B19225A70236A9B7843B1E3691A7B2AB9A269D27B032A1CBF01221A73052D0ED194F88430012B1AD194F887200AB912
S34500000F0084F88C30002384F88430022384F88F3094F88430002B7FF489AE94F88530002B7FF484AE94F88B30002B7FF47FAED4E694F88530012BE8D194F886200AB984F837
S34500000F408B30002384F88530DFE794F89210206802F000F994F89110206802F0FBF8002384F88D30012384F88F3040F20113A4F886304FF48073A4F8883057E6002555E6E1
S34500000F805553424355534253DC0B0020E10B002070B5374B04461868A36988B05D7B8DF81C500023CDE90533636800901B681BB105AA11212046984794F89030AB423EBF19
S34500000FC0236A05229A70069B38BF00252BB1059A1AB104EB0515C5E91523A36994F84C50DA8A52BA91B2002D40D06269002A14BF022003205B7B053304EB0313002D5A6808
S345000010009B6812BA14BF02250125039201920C221EBA02EBC00243EA05631BBA8A4204964FEAC006029328BF0A468DF8036069460023206D11F8015BC5540133042BF8D152
S3450000104001A9206D11F8015BC55401330C2BF8D1012384F83A30236DE3620023A26284F83830204602F0F2FE08B070BD2846C1E7504A0000364BD9784A1E072A65D8DFE84B
S3450000108002F00415263444445361382292FAA2F23049120E0A70304A002111702F4A012111700222DA702E4B1A8070470C2292FAA2F22849120E0A70274A00211170274AAF
S345000010C0012111700322DA70254B0222ECE7062292FAA2F21F49120E0A701F4A002111701E4A012111700422EDE7012191FAA1F21848120E0270184A00201070174A117001
S345000011000522DA70164B1022CEE73C2292FAA2F21048120E0270104A0020107001200F4A01441070D970CFE7382292FAA2F20949120E0A70084A00211170084A0121117001
S345000011400822C0E76422DA7070470022FBE700BFB00B0020EC0B0020EB0B0020EA0B0020920B0020044A431E113013F8011F02F8011B8342F9D17047B50B0020044A431E6E
S34500001180113013F8011F02F8011B8342F9D17047C70B0020094A0A4808B50023D370094A1370094A1380FFF7DDFF0848FFF7E6FF074B4FF400721A8108BD00BFB00B0020ED
S345000011C0AE4A0000ED0B0020920B00209C4A0000940B002030B542F21074B0FBF4F4C4EBC403C3EB4313C4EB031300EB03139BB24FF47A70B3FBF0F0C0EB801200EB821243
S3450000120000EB420203EBC2039BB26421B3FBF1F1C9B2C1EB412201EB8202C1EBC20203EB82039BB20A22B3FBF2F2D2B2C2EB4235C2EB8505303403EB450304F0FF043030AC
S34500001240303130323033302C00F0FF00C9B2D2B203F0FF0309D1302806D1302911D1302A11D12022114610462024094D85F8244085F8250085F8261085F8272085F828302B
S3450000128030BD2020F0E7202108460C46EDE700BFB00B0020584A1188F8B531BB574C584DE378584E584F652B4CD023D8132B1DD88BB3FFF7DFFE3B782978544801EB032126
S345000012C089B2C0F8801003F09FF833786BB172B6337801EB03239BB2C0F8803003F094F80023C0F88010337062B6F8BD642B1BD0002317E0C92B3DD0FA2B52D0C82BF7D189
S345000013002171902393FAA3F31B0E2B70012333703970C92312E02B7033703B704FF4FA7313800123E370C6E72171802393FAA3F31B0E2B700123337039706523E370022351
S345000013401380B8E72379112B12D8E018417990F90500002816DB2970297891FAA1F1090E29700421397001210B4431702371E6E7C823D7E72379112B0DD8E018C17D90F9AD
S345000013801700E6E701F07F012970214909780029E2D0FF21DFE7FA23E3701E4B0A229A7089E71C4B9B78002B85D16423E37094F82A30042B1AD801A252F823F0B712000069
S345000013C0D1130000E1130000E1130000E91300001148FFF7D3FE114B1888FFF7FBFE6AE70F48FFF7CBFE66E70E48FAE70E48FFF7C5FE94F82A00F0E7920B0020B00B0020F5
S34500001400EC0B0020EA0B0020EB0B002000F00F40ED0B0020E10B0020544A0000A00B0020784A00008A4A0000664A0000174B18499A6B42F400729A639A6B42F480629A63CB
S345000014409A6B42F400629A639A6B42F480529A639A6B42F400529A630E4A40F2FF53C1F894304FF48073136053609360D360136153619361D3611362936200224A61064A86
S345000014805360936013615361704700BF0080044000F00F4000B0044000900440F52910B52BD00AD8C9B3022927D000F500730022834249D000F8012BFAE7B1F5F47FF4D16E
S345000014C0244A431E00F10A0112F8014B03F8014F8B42F9D1204A00F1390112F8014B03F8014F8B42F9D100F13A03002200F50070834229D003F8012BFAE7F82303707F226C
S34500001500FF2343708370C270031D002200F50070834219D003F8012BFAE7104A431E00F13D0112F8014B03F8014F9942F9D100F13E0300F5FF720021934207D1552380F8C8
S34500001540FE31AA2380F8FF31002010BD03F8011BF2E700BFFE4A0000094B0000C04A0000F0B5104C104E114F22688A4201D301200CE0855C0D2D02F1010201D12260F3E74A
S345000015800A2D338803D10020F8542260F0BDFD5401339BB2B3F5967F22603380E4D36620F4E700BFA0060020AC0B0020F90B00200C4A1378591C11700B4AD35CA3F1300049
S345000015C0C0B209280DD9A3F14102052A03D8A3F13700C0B27047054A137843F00203137000207047F80B0020F90B0020DC0B00202DE9F041154B164A1B781288DFF85880EA
S3450000160003449342C4BF134A13784FF00006C8BF43F002030546C8BF13703446AE4202D12046BDE8F081FFF7C3FF0746FFF7C0FF98F8003000EB071053FA80F3240288F829
S34500001640003054FA80F40136E8E700BFF80B0020AC0B0020DC0B0020F70B0020F8B53B4B1B88002B53D03A4D3A4C2A783A4F3B4E002363F3410223703B7033782A70532BE8
S3450000168001D067201FE0364B02221A707378303B092BF6D801A252F823F000BF43170000C9160000131700002B170000831600008316000083160000C5160000C516000061
S345000016C0C51600000220F8BD0120FFF791FF20700220FFF78DFF234B18602378033B2D78237015F00205CCD120780028EBD00120FFF77EFFEBB22278F0540135EBB29A427E
S34500001700F5D80120FFF774FF3B78FF2B1BD10120D9E70120FFF76CFF20700320FFF768FF104B18602378043BD9E70120FFF760FF20700420FFF75CFF0A4B18602378053B80
S34500001740CDE70020BFE76820BDE700BFAC0B0020DC0B0020F60B0020F70B0020F90B0020F80B00209C06002038B50B4B0B4C19682368B3EB113F4FEA11350CD24FF48052CE
S34500001780084600F05DFA256028B1054B6B2283F82A2083F82B0038BD9C06002098060020B00B002030B51B4B1B4C1D6894F82A301A49012B87B014D1B5F5004F11D1184A93
S345000017C001440823013B11F8010B02F8010B13F0FF03F7D1134A137843F00403137007B030BD0A18D3790493937903935379029313790193D37800939378095C5278284658
S3450000180000F08AF90028EAD06C2384F82A3084F82B00E4E79C060020B00B0020F90B0020EE0B0020DC0B0020F8B5184E3368B3F5004F01D20020F8BDB3F5801F22D813F004
S34500001840070321D1124C13482278FF27511C12F00705C9B212D103B122702378002BE9D0FFF782FF2846FFF79DFF33680833336023780835083B2370EDB2EEE7875401234E
S345000018800A46E3E76920D6E76A20D4E79C060020F60B0020F90B00202DE9F043404C94F82A7087B0064688461546002F43D1114602F0B7FD002844D0012384F82A30394BD5
S345000018C0C3F80080384B1F60384B1F80384BFF221A705A709A70DA701A715A719A71DA71344B1A7867F382021A70334BDFF8CC80DFF8B89000271F6029463046FFF730FEA3
S34500001900002849D1FFF7AAFE012806D1FFF78CFFB8F800300133A8F80030022808BF84F82A006328A9F8007012D984F82A00012007B0BDE8F083012F10D11A4B1B688B42E2
S34500001940D3D094F82A00632894BF00200120EFE70028D1D0134A13680133136094F82A30022BEED1134B1B785B0711D51049CB7904938B7903934B7902930B790193CB783E
S3450000198000938B784A7809784FF4004000F0C4F8032384F82A30D4E76328C6D8DAE700BFB00B00209406002098060020AC0B0020EE0B0020DC0B0020A0060020A00B0020DE
S345000019C008B50F4B0F4A5A640F4800F017FD0F4B0F4A1A6000221146022000F0B7FC0D4A1378002103F0C703137008460A4A00F05FFD0A4800F08AFB094B0A4A1A6008BD0E
S34500001A0000800440000007132C4A0000BC0A00200024F40000400640404B0000344A00005401002000389C1C2F4A936B43F4806370B593632D4B40F20312DA6002F0E4FCE3
S34500001A402B4B1B6D1B0709D54FF400400368013304D04368013301D002F035FD254B264A9A60BFF34F8FBFF36F8FFFF7A9FFFFF7DDFC224A224E1368224C23F001031360C2
S34500001A8000F03CF9FFF786FB00F0A8FA1E4B4FF400121A6000F016F9FFF7FCFB33781B4D13F0010F0ED06B781BB9194B186801F0EAFA94F82A3013B1033B012B0FD8042338
S34500001AC084F82A302A78134B22B91A78D2431A700A222A701B7823B102F0A1FCDAE76D23EEE702F09DFCD5E70080044000A0044000F00F4000ED00E00000000000D0004011
S34500001B00DC0B0020B00B002084060020E10B0020AC060020250D00202DE9F04F85B01E46B0F5004F9DF840309DF838909DF83CA09DF844709DF84880019315467AD3019AB1
S34500001B4007EA080313400AEA030309EA030333402B400B40FF2B6DD0034600F108041A78FF2A03F1010367D1A342F8D1334C3023237072B60723E371C0F30742C0F30723CA
S34500001B805FFA80FBA27103926371029384F804B084F80B90A6726572217284F80F80A773019B637384F80CA002F006FF94F800C01CF0310FDDE9023205D062B62078C0B232
S34500001BC005B0BDE8F08F4FF0020C84F807C0A271637184F804B04FF0010B84F80BB084F80F90A6736573217302F0E6FE237813F0310F02D062B62120E2E704304FF002031D
S34500001C00E371C0F30743A371C0F30723C0B26371207184F80BB084F80F80A773019B637384F80CA002F0C8FE207810F03100E1D162B6C5E70020C3E70420C1E700000240C0
S34500001C40B1F5004F2DE9F047154608D31C4C3023237072B601260027884202D962B6002018E0C0F3074AC0F307295FFA80F8E67184F806A084F8059084F80480E672A7729A
S34500001C80677202F099FE237813F0300F04D062B62078C0B2BDE8F0872378DB070DD50923E37184F806A084F8059084F8048002F083FE237813F0300FE9D12844CCE700BFD3
S34500001CC0000002400A4B1A785AB100221A70094A0423013B13F0FF0304D1074A1378013313707047117809B1013911700132F0E7AF0B0020E10B0020E40B002013B5144CFF
S34500001D00002301A920468DF8043000F00DFC022000F0B2FA64210F4A0023A0FB010102F033FDC4F80001D4F8083143F00203C4F80831094B102283F830234FF480325A6048
S34500001D40D4F8083143F00103C4F8083102B010BD0070034040420F0000E100E01D4B0122C3F80C211C4A13880BB1013B13801B4A13780133DBB2092B03D81370BFF34F8FD6
S34500001D80704700231370164A136801331360154A136801331360144A06231046013B13F0FF0311D10378002BE8D10A2303700F4B01221A700E4A13880BB1013B13800D4AE2
S34500001DC0138801331380D9E7117809B1013911700132E3E700700340920B0020AE0B00208006002090060020E50B0020AF0B00209E0B0020900B0020024B0B6012234B6015
S34500001E000020704734000020087A20B9034B0B6020234B6070470520704700BF14000020887A0E4B10B520B91A685B680A604B6010BD9B680C891A8994420CD102280AD8CF
S34500001E401A685B6800B252F8202053F820300A604B600020ECE70520EAE700BF48000020023908B513460F2913D8DFE801F00814171E12122A2E12121212121232325A6890
S34500001E803AB119689868FFF707FD10B1154B01225A72012008BD144A9A60FAE713489860D3E90012FFF7FAFAEFE71149096801221A60490A4FF40072C3E903229A605960B2
S34500001EC0E7E724225A600B4AE6E708225A600A4AE2E74FF400725A60054A1268520A1A60D7E700BFAC060020BC080020BC0600208406002010010020A406002001391529AB
S34500001F0016D8DFE801F00B15151515151515101E373C4115151515151515272E1E4B0020587398727047107820B91B4B587398720120704701282CD1174B587312789A721B
S34500001F407047154B597B0029F2D01288110AEFD1DA72EDE7002AEBD00F4B9B7A137000207047002AE4D01088000A12D10A4BDB7A13807047002ADBD01146FFF73DBF002AA3
S34500001F80D6D01146FFF740BF002AD1D01146FFF747BF0520704700BFAC06002008B5034B186801F0C8FBBFF34F8F08BDAC06002008B500F0E5FABDE8084002494FF4A02071
S34500001FC000F0C0B8006CDC02034B302283F835234FF400125A60704700E100E038B5FFF7E7FF0D4A0D4C13680D4D23F001031360002022462946C4E90000A081FEF77EFB24
S3450000200010B92B685B686360FFF7DEFF2068BDE8384001F034B800BF00D00040AC06002040010020034B1B7BDB0754BF024B034B1868704700400640BC0A0020C00A002060
S3450000204008B5114A9379D9061BD4FFF7EBFF88B113785178127BC3F3C20311F0300F20FA03F0D2B206D0D20704D4062B03D0072B05D0400908BD1423B0FBF3F0FAE70C23AD
S34500002080FAE7024B1868F5E70040064050010020064B9A79D20755BF054B064A1868187A42BFC0F342031068D840704700400640500100204C010020034B1B781B0646BFEB
S345000020C0024B18680020704700500640BC0A002008B50C4B1B68C3F38143022B09D0032B0AD063B9FFF7E8FFB0F5004F18BF002008BD054B1868FBE74FF47A70F8E7002014
S34500002100F6E700BF00700440C00A00200C4A436802F5805110B54B6403784C681B0403F4803324F4803423434B60437811689B0403F4402321F440210B43136010BD00BF5D
S34500002140007004401A4B5A6B22F4802210B55A63044650B95A6822F480225A600120144A536B43F48023536310BD124A914218D00AD8114A914218D002F1B77202F5585254
S34500002180914210D0002005E00C4A9142FAD109229A64012006494A6822F4A02222434A60DDE70222F4E70522F2E70022F0E700BF0080044000D8B805006CDC02000E2707E1
S345000021C010B50C4C63789A0701D5002010BDA3799B06FAD4FFF734FF0028F6D0E378E278C3F341135B0003EBD213034A32F813305843EBE700400640404A0000034B1878D9
S3450000220010F0020001D0FFF743BF70470040064008B5094A907910F040000CD0FFF702FF137903F01F030133B0FBF3F0537903F01F031833584308BD00400640034B5B68DE
S34500002240DB0301D4FFF7BCBFFFF7E2BF00800440084B9B79C3F38103022B09D0032B03D0012B03D1FFF714BFFFF7D2BFFFF7A8BFFFF7D8BE0040064008B513280BD8DFE8D0
S3450000228000F00C0C151C230A2A2E320A0A363A3E420A0A0A0A46002008BDFFF7D9FF1D4B5B6C1B0F0133B0FBF3F0F5E7FFF7D0FF184B5B6CC3F30363F4E7FFF7C9FF154B08
S345000022C05B6CC3F30353EDE7FFF7C2FF114B5B6CC3F30343E6E7BDE80840FFF7AFBFBDE80840FFF7F5BEBDE80840FFF7E5BEBDE8084002F002B9BDE80840FFF77FBFBDE8C1
S345000023000840FFF75DBFBDE80840FFF781BF4FF47A70C1E70080044010B50B490A7B0B7B00F0010403F0FE0323430B7302F00103834205D1002010BD00BF013BFCD1F9E76A
S3450000234040F2DD53F9E700BF0040064070B51D4B9C799D791E7AC6F342069642C4F38104EDB217D0EE070CD5012C02D01D78AD0707D55D7805F0FE055D70124DAB79DE07E9
S34500002380FCD4104D2B7A520002F00E0203F0D0031A432A720B4B5A7801F0010502F0FE022A435A701A7802F0FC020243012C1A7001D0820704D59A7902F001028A42FAD19A
S345000023C0002070BD0040064042780B4B02F01F021A715979827801F0E00102F01F020A435A711A7901780A4342F040021A719A795206FCD5704700BF00400640036849F653
S345000024009702934210B522D912498B4294BF01210221114A0479137803F0F003234313701378847903F05F0323430C4C13706378407903F0C303034343EA0113637028B1D8
S3450000244013781A0602D5A3799B07FCD510BD0021DFE700BF00127A00005006400040064010B5124B5A7802F0FD025A701A7802F03B0242F0800208461A709A7902F01C020B
S34500002480082AFAD15A79094C02F0BF025A71A3799A06FCD4FFF798FF637943F040036371A3799B06FCD5002010BD00BF0040064013B50C460192FFF72FFF01992046FFF7AD
S345000024C0CFFF064A137803F03F0313709379C3F38103032BFAD1002002B010BD0040064008B50368002BB4BF034B044B1B689847BFF34F8F08BD00BFD00A0020D40A002040
S34500002500024B03481968FFF7EBBF00BFC40A002000C00240024B03485968FFF7E1BF00BFC40A002000D00240094AD36B43F40003D363036823F0020303600B7823B10368D6
S3450000254023F0010303607047036843F00103F9E700800440084AD2F8883043F47003C2F88830064B4CF22052DA814DF62812DA814FF4E9721A80704700ED00E00020054099
S345000025804C4A137813F0C00F74D153795B0664D4137858073DD4137B474813F0010F537818BF4FF4004013F0300F27D0137BD90724D4117801F03801302924D0382925D033
S345000025C01378C3F3C202202393409BB2B0FBF3F3384AD27802F0E002802A35D021D8402A2FD019D832B3202A28D0344A526C120F0132B3FBF2F3324A136070471378C3F309
S34500002600C2020123E0E74FF4A063DFE74FF4C063DCE74FF40043DBE7602AE6D14FF420620AE0C02A13D0E02A14D0A02ADDD14FF4B76201E04FF420725343D6E74FF4A0629B
S34500002640FAE74FF4F062F7E74FF43772F4E740F69502F1E740F67132EEE71379164903F01F030133B1FBF3F1537903F01F0318334B43BAE7137803F0C003402B09D1537876
S34500002680DB0713D5137A0F4AC3F3420322FA03F3ABE7137803F0C003802BAED1137B13F0010F054B18BF4FF400439EE74FF400439BE700BF004006400024F400008004405E
S345000026C05401002000093D0010B5174A1749002001F04BFF4FF480734FF480620021124801F024FF124A1349012001F03EFF4FF480730F484FF48062002101F017FF0E4B14
S345000027001B68022B0EDD0D4A0A49022001F02DFFBDE8104009484FF480734FF48062002101F004BF10BD00BFDC0A0020434B0000180B0020454B00003C4A0000540B0020A1
S34500002740F8B5044638B90B4B0B4E1F680546A74205DC2846F8BDBDE8F84001F094BF304601F091FF002818BF4FF0FF3501343C36EDE700BF3C4A0000DC0A00202DE9F8435C
S34500002780C6683D4B334004460D4690461BB902273846BDE8F883D0F81490484602F0EEF807460028F3D1B8F1010F2CD0B8F1020F2ED0B8F1000FEAD1002DE8DBB00404D574
S345000027C02368E26A9A4238BFE362A169A9420EDC2368E26A934238BF134622695818801AA84204DB206B01EB000CAC4534DC0023C4E9013346F02006A56226F4032626F067
S345000028004006E660C4E7204600F038F80544D3E7484602F0ADF8B0F1000CE26804DA42F08002E2600127B3E723681846A3691946E36A98422CBF0918C9180B462169920645
S34500002840A3EB010303D5A26A9342B8BF13466345ACBFED186544AFE76D1AB10744BF281AA060F10744BF9B1AEB1A154448BF6360256026F02006C0E703001000C3689A073D
S3450000288005D10E4B21221A604FF0FF30704703F020021B0309D512B1806A013870470368826900691344181AF7E70AB1806A70470368826900691344181A7047D80A0020D0
S345000028C02DE9F041D5685769EB0280460E46144605D5384602F04CF845F01005A061124B2B408BB1A169384602F054F8002806DAE36843F08003E3604FF0FF3011E025F4C6
S34500002900003525F01005E56032464146384602F04DF820F00041761AA1690E44A6610028E6D1BDE8F08100BF1000020008B5FDF776FC08BD08B5FDF772FC08BD08B5FDF7B2
S345000029406EFC08BD08B5FDF76AFC08BD08B5FDF766FC08BD08B5FDF762FC08BD08B5FDF75EFC08BD08B5FDF75AFC08BD08B5FDF756FC08BD08B5FDF752FC08BD08B5FDF7C1
S345000029804EFC08BD08B5FDF74AFC08BD08B5FDF746FC08BD08B5FDF742FC08BD08B5FDF73EFC08BD08B5FDF73AFC08BD08B5FDF736FC08BD08B5FDF732FC08BD08B5FDF781
S345000029C02EFC08BD08B5FDF72AFC08BD08B5FDF726FC08BD08B5FDF722FC08BD08B5FDF71EFC08BD08B5FDF71AFC08BD08B5FDF716FC08BD08B5FDF712FC08BD08B5FFF73F
S34500002A007FFD08BD08B5FFF785FD08BD08B5FDF706FC08BD08B5FDF702FC08BD08B5FDF7FEFB08BD08B5FDF7FAFB08BD08B5FDF7F6FB08BD08B5FDF7F2FB08BD08B5FDF714
S34500002A40EEFB08BD08B5FDF7EAFB08BD08B5FDF7E6FB08BD08B5FDF7E2FB08BD08B5FDF7DEFB08BD08B5FDF7DAFB08BD08B5FDF7D6FB08BD08B5FDF7D2FB08BD08B5FDF7C8
S34500002A80CEFB08BD08B5FDF7CAFB08BD08B5FDF7C6FB08BD08B5FDF7C2FB08BD08B5FDF7BEFB08BD08B5FDF7BAFB08BD08B5FDF7B6FB08BD08B5FDF7B2FB08BD08B5FDF788
S34500002AC0AEFB08BD08B5FDF7AAFB08BD08B5FDF7A6FB08BD08B5FDF7A2FB08BD08B5FDF79EFB08BD08B5FDF79AFB08BD08B5FDF796FB08BD08B5FDF792FB08BD08B5FDF748
S34500002B008EFB08BD08B5FDF78AFB08BD08B5FDF786FB08BD08B5FDF782FB08BD08B5FDF77EFB08BD08B5FDF77AFB08BD08B5FDF776FB08BD08B5FDF772FB08BD08B5FDF707
S34500002B406EFB08BD08B5FDF76AFB08BD08B5FDF766FB08BD08B5FDF762FB08BD08B5FDF75EFB08BD08B5FDF75AFB08BD08B5FDF756FB08BD08B5FDF752FB08BD08B5FDF7C7
S34500002B804EFB08BD08B5FDF74AFB08BD08B5FDF746FB08BD08B5FDF742FB08BD2DE9F34705468A460068174600240DF1030206211E468DF8034000F0EDFA9DF80330012B67
S34500002BC036D89AF8009019F01F0905F10C080FD128684246042100F0DDFAAB8903F00303AB8102233360C7F8008002B0BDE8F087B9F1010F04D10223AC8120463360F2E7AF
S34500002C00B9F1020F12D1BAF8043028688DF8043001AA0521ADF8064000F0BCFABDF8063003F00303AB81C6F80090DCE70520DAE70520DAE72DE9F04385B0B1F8028004467F
S34500002C400D46006817461E460DF10302002306218DF8033000F09EFA9DF80330022B4FEA182928D8EB880293B9F1010F0BD101AA0B212068FDF722FD019B3B60029B33605F
S34500002C8005B0BDE8F083B9F1020F5FFA89F35FFA88F804D18DF80C8001AA0C21E9E7032B07D1AB888DF80E80ADF80C3001AA0D21DFE70520E0E70520E2E77FB504460D46D3
S34500002CC0006800260DF10F0206218DF80F6000F061FA9DF80F30012B1FD820688DF80F600DF10F02062100F076FA6B8843B9012320688DF80F300DF10F02062100F06BFAD8
S34500002D00AA1C032120680192FDF79EFC019A20680921FDF7D3FC04B070BD0520FBE773B504460D46006800260DF1070206218DF8076000F02FFA9DF80730032B0CD0022B79
S34500002D4018D86B888DF807300DF107020721206800F041FA02B070BD20683246072100F03AFA0028F6D101238DF807300DF107020621ECE70520EDE737B5002305460C462C
S34500002D8000688DF806300DF1060206218DF8073000F000FA9DF80630012B02D9052003B030BD6378032B04BF01238DF80730237813F01F0309D16388012BEFD128680DF1D5
S34500002DC007021421FDF77AFCE9E7022BE6D16388002BE3D1A1880B0706D19DF807302868C9B253B100F0B6F99DF807302868221D33B10521FDF728FCD1E700F0BBF9F3E728
S34500002E000621F7E770B5052A05460C46DDE9040113D1227812F0600F0DD012060BD4E288002A08BF0123DB01284603F08001BDE8704000F08FB90123F5E70A68E3889A4285
S34500002E4088BF0B600B6802680021284600F030F958B994F90030002B07DA0346024601462846BDE8704000F029B970BD73B50446154600681E460DF10702002306218DF832
S34500002E80073000F087F99DF80730012B0AD8012304F10C0233602A6020681521FDF70EFC02B070BD0520FBE7F7B504460F46006815461E460DF10702002306218DF8073026
S34500002EC000F068F99DF807306BB9B988012304F10C0233602A600B022068A3811621FDF7EDFB03B0F0BD0520FBE737B5002304460D4600688DF807300DF10702062100F0E5
S34500002F0049F99DF8073093B9AA88AB782068254643EA022325F80C3F04212A46FDF794FB20682A460A21FDF7C9FB03B030BD0520FBE7F7B504460D46006817461E460DF125
S34500002F400702002306218DF8073000F023F99DF807306BB9AB8820682546082125F80C3F2A4600F017F902233D60336003B0F0BD0520FBE7F8B50E460446F0B14768F7B11A
S34500002F80CD0945EA4105EDB20C2000FB054090F814C0BCF1000F14D14FF0010C80F814C036064CBFBE68FE682068B04720B10C2303FB054400232375F8BD0320FCE70620EB
S34500002FC0FAE70220F8E720B1436823B15B690068184703207047062070477FB50446002949D0002847D08368002B46D00A7A102A1FD1012380F86F3000220E21FFF7E3FF1A
S345000030000025022384F86E3084F86C50234604F160021D75C3E903550C339A42F9D1A368002201212046984784F86F50002004B070BD12F00C0020D1530003F01E0343EA50
S34500003040D2130C2202FB0342D568B5B10E6801964E68497A02968DF80C1051B1207584F820000C2202FB034301A91A692046A847DDE71175F5E70320D9E70120D7E7002263
S345000030801146FFF7A0BF00220121FFF79CBF10B5044658B1436823B15B6800689847002363600020206084F86D0010BD0320FCE701F00F0141F08001FFF75CBF01F00F0121
S345000030C0FFF758BF20B1436823B11B69006818470320704706207047F0B4B8B1C9B1C2B18D7815F00C0614D16C0004F01E0444EAD5140C2707FB0403156852681E75DD6094
S345000031001A61F0BC0A460221FFF75DBF0320F0BC70470420FBE737B504468DF80710A8B1CDB20DF107020321FFF74DFF15F00C020ED16B0003F01E0343EAD5130C2101FB8B
S345000031400343C3E903221A7503B030BD0320FBE70420F9E707B511F00C0F8DF8071007D10DF107020421FFF72EFF03B05DF804FB0420FAE707B511F00C0F8DF8071007D107
S345000031800DF107020521FFF71EFF03B05DF804FB0420FAE7DAB1023906291AD8DFE801F004071113090E15000F21FFF70CBF1021FBE790F86E3013700020704790F86C301B
S345000031C0F9E70621F1E70721EFE70921EDE7042070470120704703390B292BD8DFE801F0062A2A090F2A2A2628222A241121FFF7EABEFAB1137880F86E300020704790F811
S345000032006E30032B0AD0AAB1137880F86C30032380F86E3000F16C021421E8E700F16C020821E4E70A21E2E70B21E0E70C21DEE70D21DCE70120704737B590F82D4000F182
S345000032400C03C4F3001224F0280403EBC2030825002244F02004C0E90952036280F82D4011460095FDF7DEFA03B030BDF0B58368FF2283F8882093F8942042F0020283F86C
S345000032809420002283F89820456825F4FF7525F00105144600F12C0745EA421141F0080C0C60CCF8004041F0100C41F018015601CCF800400C6046F010010144BC51CC62D0
S345000032C002F130010132042A03F82140E4D180F8A04093F8942002F0FD0283F89420FF2283F88C20892283F8842080F8A14093F8942002F0DF0283F89420F0BD88B18368FE
S34500003300FF22002083F8802083F8840083F8980083F8940093F8002142F0C00283F800217047032070472DE9F3410446480000F01E0040F001000E4604EB00114FEA00187D
S3450000334091F82D707D06C7F3801C07D4C1E9082347F02002C1F828C081F82D2004EB08018A8DC2F309059D4228BF1D4694F8A130D3B904EB00108B6A026A0095134406F0B2
S345000033800F0101222046FDF74DFA0746A044D8F828302B4304D1330702D12046FFF74CFF384602B0BDE8F0810127EFE7F7B54D01064605F4F0746BB911F00F050AD10444A0
S345000033C094F82D3065F3861384F82D30FFF734FF012037E03019344490F82D50C5F380176D065CBFC0E90823876294F82D0040F0200084F82D00A08DC0F30900984228BFF7
S345000034001846A36A1344F26904F1280582B196F8A0406CB940280BD840EA0307BF0707D06B7964F345136B71012386F8A030134696F8A120002ACBD1009001F00F0130460F
S34500003440FDF7F0F903B0F0BD1FB54B0003F01E0343EAD11300EB031404F1280294F82D40640613D500EB03138DF80C101B6A019300214FF0FF348DF80D100294537961F3B3
S3450000348086135371006801A9FFF7A7FD002004B010BDF8B501F00F056A0042EAD11300EB0313476893F82D20CE0922F00C0283F82D2027F4FF77320127F0010742EA451283
S345000034C03A439F8DC7F309073F04283347F0080717609B88C3F3090342F008021B0443F008031360836803EB8503044693F8C02002F0FD0283F8C02055B1FFF7A5FFA268FB
S3450000350092F8943003F0DF0382F894300020F8BD002EF4D1FFF790FEF1E770B5044601F00F06CB0943EA4605FFF78EFF3036A368002003F8260004EB0514A38D60F3090373
S34500003540A38570BDF8B50C460546002800F0EF800F2900F2EE80DFE811F010002900390078007F00B000B700BB00CD00EC00EC00EC00EC00EC00D300E6008368002283F88A
S3450000358000211A7F510742BF1A7F42F080021A7793F8082142F0100283F8082193F8942042F0010283F894202046F8BD83681A7F520742BF1A7F02F07F021A7793F808218B
S345000035C002F0EF0283F808210024EDE7002A00F0B0809678D778138806F00F046000012F4FEAD61140EAD61027B2AE6821D140F2FF3C634528BF634605EB0010127943EAFD
S34500003600C233828D23F4405302F440521343838506EB8703012993F8C0200CBF0420082002430C4383F8C020CED12846FFF704FEBAE706EB870E402B9EF8C0C04CF0010CE4
S3450000364028BF40238EF8C0C0D6E7002A71D0BDE8F8401178FFF761BF002A6AD0117801F00F077B0043EAD116CC09FFF7EDFE05EB061303F1280293F82D3043F0040353710A
S345000036806B68240123F4FF7323F0010344EA47141C435379C3F3001344EAC3049388AA68C3F309031B0443F08C03236092F8943003F0DF0382F8943086E7002A39D0BDE801
S345000036C0F8401178FFF7E5BE9AB3002414806BE77AB3137813F00C042BD1580000F01E0040EAD31005EB001595F82D30C3F38003538059E7EAB18368127883F8982063E711
S34500003700002464F07F01E6B2C9B22846FFF705FF013431462846FFF700FF042CF1D12846FFF7A4FD50E722B1002414703CE703243AE7012438E72DE9F04F89B0002800F003
S345000037404B810468A36893F880A093F884200AEA020A1AF0080F76D0082293F8901083F8802063680D09C1F3C00B23F4FF73C1F3800123F00103CA0043EA451342EA0B1282
S345000037801A434BEA450617685268039204EB06124FEA061892F82D20500654D5C7F38309B9F10D0F08BF84F8A310C7F30947BBF1000F00F08880A04404EB061098F82D300F
S345000037C0D8F82820C3F3C00E8EF0010E3A446EF3C303C3F3001EC8F82820416A8EF0010E6EF3041388F82D308B1A05D0B8F82CC0CCF3090C67455FD2036A069204EB0616B5
S34500003800059396F82D3006F128006FF386134371002F5CD08388C3F30902B7FBF2F302FB1373002B53D1002D3FD194F8A33004EBC3035B8A99424AD200952B4601222946DC
S345000038402046FCF7EFFF1AF0010F0FD0A268012384F8A13082F880300023CDE905331023ADF81C30206805A9FFF7B7FB1AF0800F00F0B2808021A36893F88020100600F1B1
S34500003880A88094F83D305A0704D494F82D305B0740F1A28080212046FFF7FBFD0021204609B0BDE8F04FFFF7F4BD4279D2090ED0009301222946C3E7026A45F0800120467F
S345000038C0FFF731FDBFE7D5B9CFB9CDE90555A9F10D06D6F1000949EB060945EACB158DF81D908DF81C50206805A9FFF776FBA26892F8943003F0DF0382F89430A3E704EB5F
S34500003900080C9CF82D20910612D4C2F3001243EAC203596804EB0613186ADCF828301844814202D03A4600F0FDFD002384F8A03004EB080304EB06119A6A3A449A624B6AE2
S34500003940ADBBB9F10D0F32D194F82D0040F0080084F82D0094F83D0040F0080084F83D00300104EB061606F1280C96F82D60C6F3001E8EF0010E6EF304168CF805603BB186
S345000039809B1A05D0BCF80460C6F30906B7421AD2B9F10D0F0CBF039B0B6A06922044059390F82D306FF3861380F82D308FE7A04498F82D00C0F3C00C8CF0010C6CF3C30084
S345000039C088F82D00CCE70A6A20462946FFF7EEFC39E783F880104EE709B0BDE8F08F836870B5044693B1002501200626A3681A79954202D30023A36070BD9A68206806FBC3
S34500003A0005F30135D15CFFF786FBEFE70120F3E710B5044648B1FFF7E2FF0023C4E9003384F8943084F8933010BD0320FCE7F0B504468FB01646002A00F07281002800F0FA
S34500003A406F81C9B20139052900F26E81DFE811F038010600450069008E00C000002380F89430436801AA1B6805219847019B0546002B00F05781013B84F8903001AEA6465F
S34500003A804FF0010CB36833B3736823B3331D0FCB0EF1540787E80F0094F890205FFA8CF39A4208D30CF1010CBCF1040F06F110060EF1100EE6D1226A702313700A23D37177
S34500003AC0002393701373537384F88D3084F88E3028460FB0F0BD0125DEE74368002B00F0238190F8943012789A4200F01D810BB1FFF775FF337884F89430002384F89330F9
S34500003B002046FCF7F9FE05460028E1D11F23A26994F892102068FFF7D1FA012384F88D30D6E74368002B00F0FF80168890F89530B3EB162F40F0F88090F89330F6B2B34289
S34500003B4000F0F280FFF74BFF2046FCF7D5FE054648B91F23A26994F892102068FFF7AEFA012384F88D3084F89360B1E74368002B00F0DA808368002B00F0D68090F8863066
S34500003B8083B9117890F8912091424FF0010007D184F8860084F88E3031782068FFF7DAFA054600E0012594F88730002B90D1317894F8922091428BD1012284F8872084F8E7
S34500003BC08D30317820680FB0BDE8F040FFF7C2BA4368002B00F0A8808368002B00F0A48090F88950012D3FF473AF90F88650012D40D1127890F891309A4209D1002380F80E
S34500003C00863080F88E3031780068FFF7B3FA054694F88730012B0ED1327894F892309A4209D1002384F8873084F88D3031782068FFF7A0FA054694F88F30023B012B29D847
S34500003C4094F88A30012B17D1B4F88630002B7FF43FAF94F88D20206894F8921084F88A30012A25D184F88D30FFF72CFA002384F88F302DE70125CBE794F88E30206894F8B3
S34500003C809110012B0CD184F89630FFF71BFA002384F88F3094F88A30012B7FF419AFD3E70D23E269FFF704FA012384F88E30EEE71F23A269FFF702FA012384F88D30D5E748
S34500003CC013681A7802F01F05012D2DD15978FE2916D0FF297FF4FCAE988894F89510884224D1598811BBDB8803BB13061ED440F20113A4F88630A4F8885084F88A50E7E634
S34500003D00988894F89510884210D1598871B9DB88012B0BD1120609D59034C6E90145D7E60325D5E60425D3E60125D1E60525CFE630B585B00369009383695A7BC3688DF894
S34500003D400C2000EB0211B3F5803F28BF4FF48033C96D8B4294BF019301914368044600251B6802956A4604219847A36922695B7B94F8911004EB03135B6D9A4206D2DDE98A
S34500003D8001322068FFF794F905B030BD012384F886300223206884F88B5084F8855084F88F30FFF7D7F92846EEE730B585B00369009383695A7BC3688DF80C2000EB02117A
S34500003DC0B3F5803F28BF4FF48033096E8B4294BF019301914368044600251B6802956A4603219847A36922695B7B94F8921004EB03135B6D9A4206D2DDE901322068FFF742
S34500003E005DF905B030BD012384F887300223206884F88C5084F8845084F88F30FFF79AF92846EEE730B484695568647B126800EB04140129A46D026105FB04F4C46002D15A
S34500003E4030BCFFF775BF30BCFFF7AFBFD0E9093270B504464BB9C1698B6012B90A73104670BD02220A731846FAE790F8391000296ED0C56942B9AB60134694F89110E26A71
S34500003E802068FFF715F90FE090F83A10002954D0934290F8381013D99B1A0129AB60EBD100F13002FFF7BEFFE36908B918735CE001221A73236A03229A7011221A7354E021
S34500003EC04FF00002AA6010D1012907D100F13002FFF7A8FFE36940BB1873C1E7C26A90F891100068FFF7E4F8F4E7012916D18269527B00EB0212966DB3FBF6F206FB123343
S34500003F004263AB6000F13002FFF78CFFE36960B994F83820012ADFD102220CE0C26A90F891100068FFF7C4F8F0E701221A73236A03229A7011221A7392E7AB60C26A0B4680
S34500003F4090F891100068FFF7B3F8E3690222B5E76AB990F892100068FFF7FCF8E269636A93600123137384F88730052078E790F83A1059B190F892100068FFF7EBF8E3695F
S34500003F80626A9A6002221A730123ECE79342C56990F8386019D99B1A012EAB600DD100F13002FFF73FFFE36900283FF47FAF01221A73236A03229A7080E790F89210134629
S34500003FC0C26A0068FFF77AF8EDE7A96016D1012E0DD100F13002FFF725FFE36900283FF47BAF01221A73236A03229A70A3E7C26A90F892100068FFF761F8EEE7012E12D1F6
S345000040008269527B00EB0212966DB3FBF6F206FB12334263AB6000F13002FFF703FF0028E1D1E36974E7C26A90F892100068FFF745F8F4E710B586B0036A0493836903F1ED
S345000040400F025B7B8DF81430436801921B68044613B101AA0F2198471223A362012384F83A30236AE362002384F838302046FFF7EDFE06B010BD10B586B0036A049383692F
S3450000408003F10F025B7B8DF81430436801921B680022CDE90222044613B101AA08219847029BA362012384F83A30039BE362002384F838302046FFF7C9FE06B010BD10B4D8
S345000040C08269D37BD2F81110282B09BA15D1D38A5BBA9BB2012480F83A40527B00EB0212926D80F838405A4382620022C0E90C135DF8044BC262FFF7A9BEA82B0ABFD2F813
S34500004100153000231BBAE5E710B48269D37BD2F811102A2B09BA4FF0000414D1D38A5BBA9BB280F83A40527B00EB0212926D5A43C0E90A24012280F83820C0E90C135DF848
S34500004140044BFFF783BEAA2B0ABFD2F8153023461BBAE6E730B587B0036A0493836903F10F025B7B019204468DF81430012200238362C36280F8383080F83A20FFF766FE12
S3450000418063681B6805461BB101AA072120469847284607B030BD00220121826280F83A10C26280F83820FFF751BE10B586B0036A0493836903F10F025B7B8DF8143043684D
S345000041C001921B680022CDE90222044613B101AA09219847029BA362012384F83A30039BE362002384F838302046FFF72FFE06B010BD10B586B0036A0493836903F10F0253
S345000042005B7B8DF81430436801921B680022CDE90222044613B101AA0A219847029B039AA362002384F83A3084F83830E2622046FFF70CFEA3691B7CDB0704D5236A052271
S345000042409A7024221A7306B010BD30B5836985B05D7B8DF80C500023CDE9013343681B68044613B101AA1021984794F89030AB423EBF236A05229A70029938BF002531B188
S34500004280019B13B304EB0515C5E915310821A069437BC07B053304EB031325285A68A16202F1FF3212BA12D1E16B0A609B681BBA4B60012384F83A300023E16284F83830BF
S345000042C02046FFF7C3FD05B030BD1946DFE7216C4A609B681BBA8B60EBE770B5002504460126856280F83A60C56280F83850FFF7ADFDE3691A7B022A0DD0A269127C02F019
S345000043001F02172A1BBF1E73236A1D7305221EBF9A7024221A7370BD30B587B0036A0493836903F10F025B7B019204468DF81430012200238362C36280F8383080F83A20F0
S34500004340FFF784FD63681B6805461BB101AA0C2120469847284607B030BD30B587B0036A0493836903F10F025B7B019204468DF81430012200238362C36280F8383080F8F7
S345000043803A20FFF763FD63681B6805461BB101AA0D2120469847284607B030BD30B587B0036A0493836903F10F025B7B019204468DF81430012200238362C36280F83830F5
S345000043C080F83A20FFF742FDE3691B7B022B054606D063681B681BB101AA0E2120469847284607B030BDC16910B401240C73036A00228A60052182629970202119735A737D
S345000044005DF8044BFFF722BD82B006230193019B5A1E01920BB902B0704700BFF7E77047704710B50378532B0ED14378302B0BD10379302B08D14379302B05D18379302BAC
S3450000444002D1C379302B37D000202CE0845C0D2C2AD1841864780A2C08BF1346013292B28A422DD2002BF1D00A3B9BB2C25C322AEAD118444378452BE6D1837803F0FD0396
S34500004480352BE1D1C378332BDED10379332BDBD14379312BD8D18379332BD5D1C079A0F139035842584110BD0A2CD7D1841864780D2C08BF1346D1E7002308220139CFE7AB
S345000044C0002BC1D0D0E7D0F800D0D0F804F0704704207146084202D0EFF3098001E0EFF3088081690A884BF6AB639A4200D0FEE70231816120210160704710B5FDF7A0FD6B
S34500004500044610B90024204610BDFDF7A1FEB4EBD00FF7D8F7E708B5FEF7D6F8BDE80840FDF782BA00F0EBB900F003BA70B5C468A50708D0B2F5007F11D0B2F5806F04D029
S34500004540B2F5807F0BD0012008E000F124010123224301610160C361C260002070BD5E1E6FF07F45AE42F3D3EDE770B50D4606461046144600F02DF82B78722B17D0772B3B
S3450000458018D0612B23D1082348F2020215F8011F2B2912D0622915D01B07E260666104D5022200212046FEF7E9F8204670BD00230122EBE704230222E8E742F0030243F09D
S345000045C00203E3E742F0040243F00103DEE70024EBE7F0B5C468A10789B0054622D0220718D4D0E90467FEF7ABF8384600F0BAF9230502D5304600F08FF8A40DA40514F190
S34500004600A54F07D1296A2022684600F0C9F9684600F00BF83C2200212846FFF785FF002009B0F0BD4FF0FF30FAE710B5044600F006F801462046BDE8104000F0A5B910B5E4
S34500004640431C8207044614D1204654F8042BA2F1013121EA020111F0803FF5D0D1B281B112F47F4F0BD012F47F0F14BF2046033003E010F8012B002AE3D1C01A10BD0230B2
S34500004680FBE70130F9E7C36870B513F00306044611D09B0611D5856A00F056F8E36823F44053E360204600F00EF80022064629462046FEF763F8304670BD816905680D4454
S345000046C001696D1AEAE738B501680569C36A0446C06820F40022E26000F08202022A02D04FF0FF3038BD10F48030FBD0994238BF19468D4208D1E368E562002023F480336E
S345000047002560A060E360EDE72246491B2846FEF7D7F80028EFD0E3E7A8B14FF0805340F80C3C50F8042C72B11368B3F1805F0AD150F8083C516803330B4440F8083C936888
S3450000474040F8043CEDE77047C368826923F0200310B5C360836A9A4204460ED0FFF7B3FFE36823F4405323F0100343F01003E360A36AA3612369E3622360E36823F4804335
S3450000478023F04003E36010BD5FF0000C30B51C0022D112006FD0914206D305460846002100F06FF80446284600F06BF80A462146BDE830401CF0404F08BF704703D54942DD
S345000047C0404261F100015FEA8C0C38BF70475B42524263F10003704742D41C0C04BF1B040CF1100C13F07F4F04BF1B020CF1080C13F0704F04BF1B010CF1040C13F0404FD5
S3450000480004BF0CF1020C5FEA83035CBF0CF1010C5B00CCF1200E22FA0EF4234302FA0CF200FA0CF520FA0EF001FA0CF4204321FA0EF114461A4600F024F8A4FB0023AA1A15
S3450000484071EB03033CBF1B190138CCF1200E22FA0CF203FA0EF4224323FA0CF30021A7E7821A71EB03033CBF02460B464FF0000141F100009CE700200021BDE8304000F067
S345000048803DB80423B1EB122F09D2090241EA10610002013B08BF7047B1EB122FF5D30018494134BF9142891A4041494134BF9142891A4041494134BF9142891A4041494118
S345000048C034BF9142891A4041494134BF9142891A4041494134BF9142891A4041494134BF9142891A4041494134BF9142891A4041A3F1010313F00F0FD2D17047704740EA04
S345000049000103DB0703460CD40346043A22BF51F804CB43F804CBB2F10402F7D2043208BF7047013A24BF11F801CB03F801CBF8D87047034613F0030F0ED101F0FF0141EA18
S34500004940012141EA0141043A24BF43F8041BB2F10402F9D202F10402013A24BF03F8011BFAE7704703B469460220ABBE02B0704703B469460C20ABBE02B0704703B46946C9
S345000049800920ABBE02B0704703B469460E20ABBE02B0704703B469460A20ABBE02B070470FB469460D20ABBE04B070470FB469460520ABBE04B070475FF800F001000020E8
S345000049C09D2B0000792D000000000000792D0000000000001F2D0000352C0000000000006D2E0000BB2C0000A92E0000EB2E0000332F0000F5090000113A00002F3A00006A
S34500004A00030000000000000000000000000000000000000091080000FD32000027330000AD33000049340000453500000024F40000048000010200000000110003000000C1
S34500004A408002DC020005B80580079508000A710B000000004C4F4144494E472046494C452078787878784641494C45442020434F444520787878787846494E4953484544EC
S34500004A8021202020202020202020454A45435445442120202020202020202020524541445920464F52205331392046494C45455A63616C204D61782055504441544576341F
S34500004AC0EB3C904D53444F53352E300002200200020002FFFFF8F3003F00FF00F900000000000000000029BDA5DD024E4F204E414D4520202020464154313220202050479B
S34500004B0054524541445920202020004B9C429238923800009D429238000000000000504754455A55504441544508000000000000000000009D4292380702000000000000B9
S34500004B4000070072007700FF034B80221A701A781206FCD5704700BF0000024009022000010100803209040000020806500007058102400000070502024000001201000213
S34500004B8000000040C91FB082010101020301FFFF8400002004000000E400002001000000700000200301000000000000020000005801002000000000010000007800002039
S34500004BC00806500060000020010000000403090420035000470020005400520049004F004E0049004300200049004E0043002E002203500047005400200045005A00430090
S34500004C0061006C005500700064006100740065002000FFFF180342004F004F0054004C004F004100440045005200200000010020F000002009040000040000002000000098
S34500004C4022000000180000008400002088000020A8000020CC0000200080040220000000504754284E585029455A43616C204D61782055504441544530303034611E000001
S34500004C80000000005800002034010020FD1E00000100000000093D000080000000004001810240000000020240000000FFFFFFFFFFFFFFFFFFFFFFFFFFFFFFFFFFFFFFFF0B
S34500004CC0FFFFFFFFFFFFFFFFFFFFFFFFFFFFFFFFFFFFFFFFFFFFFFFFFFFFFFFFFFFFFFFFFFFFFFFFFFFFFFFFFFFFFFFFFFFFFFFFFFFFFFFFFFFFFFFFFFFFFFFFFFFFFFFFEE
S34500004D00FFFFFFFFFFFFFFFFFFFFFFFFFFFFFFFFFFFFFFFFFFFFFFFFFFFFFFFFFFFFFFFFFFFFFFFFFFFFFFFFFFFFFFFFFFFFFFFFFFFFFFFFFFFFFFFFFFFFFFFFFFFFFFFFAD
S34500004D40FFFFFFFFFFFFFFFFFFFFFFFFFFFFFFFFFFFFFFFFFFFFFFFFFFFFFFFFFFFFFFFFFFFFFFFFFFFFFFFFFFFFFFFFFFFFFFFFFFFFFFFFFFFFFFFFFFFFFFFFFFFFFFFF6D
S34500004D80FFFFFFFFFFFFFFFFFFFFFFFFFFFFFFFFFFFFFFFFFFFFFFFFFFFFFFFFFFFFFFFFFFFFFFFFFFFFFFFFFFFFFFFFFFFFFFFFFFFFFFFFFFFFFFFFFFFFFFFFFFFFFFFF2D
S3450000800000000120C58100000D82000093C90000118200001382000015820000000000000000000000000000000000001782000019820000000000001B8200001D820000B9
S34500008040B5B00000BDB00000C5B00000CDB00000D5B00000DDB00000E5B00000EDB00000F5B00000FDB0000005B100000DB1000015B100001DB1000025B100002DB10000E4
S3450000808035B100003DB1000045B100004DB1000055B100005DB1000065B100006DB1000075B100007DB1000085B100008DB1000095B100009DB10000A5B10000ADB100009A
S345000080C0B5B10000BDB10000C5B10000CDB10000D5B10000DDB10000E5B10000EDB10000F5B10000FDB1000005B200000DB2000015B200001DB2000025B200002DB2000054
S345000081000DA8000035B200003DB2000045B200004DB2000055B200005DB2000065B200006DB2000075B200007DB2000085B200008DB2000095B200009DB20000A5B20000B3
S34500008140ADB20000B5B20000BDB20000C5B20000CDB20000D5B20000DDB20000E5B20000EDB20000F5B2000000000000FDB200000DB3000015B300001DB3000025B30000FC
S3450000818005B3000000000000C8D20000000000200C000000C8D200000000FF1F00000000C8D200000000001400000000100000201C0E00000000FF1F000000000000001449
S345000081C00000000038B572B602F05EFF0C4C0D4DAC4206D30C4DAC420AD362B604F04BFCFEE7D4E90001A2680C3400F019F8EFE754F8080B54F8041C00F01BF8EBE700BF02
S3450000820088810000AC810000C4810000FEE7FEE7FEE7FEE7FEE7FEE7FEE7FEE7FEE7FEE710B50023934200D310BD1C585C500433F8E700231A468B4200D370471A500433BD
S34500008240F9E7FFFF38B5094B094C19682368B3EB113F4FEA113506D24FF48052084602F057F8256038BD0020FCE700BF8C030020840300207FB5154B02461868144BB0F59D
S34500008280803F995C1A4412D1124900230133DBB212F8010B01F8010B082BF7D10E4AD37843F00103D370002007B05DF804FBD3790493937903935379029313790193D378D5
S345000082C000939378527801F08FFFEDE78C030020390800206B0900202C0800200B4A1378591C11700A4AD35CA3F13000C0B209280AD9A3F14102052A02D8373BD8B270478F
S34500008300044B04221A700020704700BFD0080020D4080020D30800202DE9F041134B144A1B781278DFF8508003449342C4BF114B03224FF000060546C8BF1A703446AE42C1
S3450000834002D12046BDE8F081FFF7C8FF0746FFF7C5FF98F8003000EB071053FA80F3240288F8003054FA80F40136E8E7D0080020D2080020D3080020CF0800202DE9F74390
S345000083804B4C4C4DDFF84C814B4F4C4E002323702B7001AB01220DF10301404604F08AF8D8B101232B702178434B454C454F00225A5422703A701A78532A4FF0020259D175
S345000083C05B784149303B0A70092B4ED8DFE803F01B1B35414D2727272727019A2378002AE1D09DF803200D2A05D1328801323280002BCED0D7E70A2AFAD0952BC9D8591C95
S34500008400FA542170C5E70120FFF786FF20700220FFF782FF2D4B18602378033B23702378002B3DD123782A480021FF255A1C5E07D2B239D1D9B1237019E00120FFF76CFF63
S3450000844020700320FFF768FF204B18602378043BE4E70120FFF760FF20700420FFF75CFF1A4B18602378053BD8E702232B7003B0BDE8F0832A70D2E7FFF74EFF09F8080042
S34500008480013623785FFA86F843454FF00100F3D8FFF742FF3B78FF2B1CBF05232B70C1E7DFF82C900026ECE7C55401211346BDE7D2080020D3080020D4080020060600203F
S345000084C0D1080020CF080020D00800208C0300203908002010000020F0B5824C87B000F07DFD237C122B29D8122B2BD8DFE813F042006A008C00960038002A002A002A00CF
S345000085002A002A00B800C300DB002A002A002A015601610163010E2B14D8DFE813F05E01670169016B016D016F0113001300130071017B01350184018F019101653BDAB255
S345000085400E2AE8D9684A6949694800F0C5FC694B187000F0D5F907B0BDE8F04000F03EBD654B66491D68664E00220B78002B6CD1032342E0634A6448002100F0ADFC634B17
S345000085801870634B00251D705A4B1D70614B1D7000F088F900F0B4F95F4B1D805F4B1D605F4BFF22DA701A705A709A701A715A719A71DA715B4BDA7865F30002DA70237C8C
S345000085C001331AE0FFF7DAFE574B1B78052B13D9564B1A78532A0FD15B78302B0CD1544B1B784BB9464A53490E2312F8015B11F8010B854203D010B16523237411E1013BD7
S3450000860013F0FF03F1D1DAE74B4A3948002100F063FC384B187000F073F9D0E7FFF7AEFE434B1B780BB16623E7E7344B1B78002B00F0F780304B1B68B3F5004FC0F0F18078
S34500008640B3F5803FBBD30A23D7E7D0B20132375C285C874201D06723CFE7013B0B7084E7364A2348002100F037FC224B187000F047F90C23C1E7FFF781FE2B4B1B780BB9DF
S345000086800F23BAE72A4B1B78002BCCD11B4B1B78002B00F0C680184B1A68294B1B689A428DD26823A9E7144F254B3A68134E1A600025337813B9237C013B9EE7FFF7C2FD84
S345000086C008B1692399E72846FFF7D4FD08B16A2393E73B6808333B6033780835083B3370EDB2E6E71A08002097D10000C40A0020830A0020420A00208C030020D1080020AE
S34500008700390800209ED00000850B0020440B0020C30A0020C109002006060020840300206B0900202C080020D2080020D4080020D3080020A1D10000B0D00000BDD0000043
S3450000874088030020414804F029F80021404A414800F0C2FB404B187000F0D2F83F4BDB78D90711D53E49CB7904938B7903934B7902930B790193CB7800938B784A780978D0
S345000087804FF4803001F030FD364804F0A6F800287FF415AF237C0133237410E7324A3348002100F099FB324B187000F0A9F8122323E7304AF3E700F019FC237ADA0730D585
S345000087C0BFF34F8F2C492D4BCA6802F4E0621343CB60BFF34F8F00BFFDE7294A2948002100F07AFB284B18706E2306E7274AF5E7274AF3E7274AF1E7274AEFE7274AEDE788
S34500008800274A1A48002100F067FB194B187000F049F800E70D4803F0C1FF237ADB073FF5CEAE07B0F0BD104A1048002100F054FB0F4B187000F064F87323DEE60D4AF3E782
S3450000884007B0BDE8F04000F0D1BB00BF10000020CDD00000040B0020C30A00202C0800206B0900207A020020D7D00000830A0020420A0020E6D0000000ED00E00400FA0578
S34500008880F3D00000850B0020440B002004D100001AD1000043D1000059D100006DD1000081D100000F4B002030B598710E4B0F4D18700F4B02221A700E4BFF221A702B78EE
S345000088C0122B09D90C492024CC549A1C0133D2B2DBB22A70CC548854084B9A786FF3C3029A7030BD0F080020C0090020440B0020BF090020BC090020850B00202C08002026
S34500008900154B1648002230B5DA71154B154D1A70154B007802211970144BFF21197014492B7809781944014412290DDD591C1148C9B22024C4544454D91C0233C9B2DBB292
S345000089402970C454425401220B498B7823F0120343EA42038B7030BD0F080020C1090020BE090020420A0020BD090020BB090020C30A0020830A00202C080020364B59792F
S345000089804A1E072A65D8DFE802F00415263444445361382292FAA2F23049120E0A70304A002111702F4A0121117002225A712E4B1A8070470C2292FAA2F22849120E0A709C
S345000089C0274A00211170274A0121117003225A71254B0222ECE7062292FAA2F21F49120E0A701F4A002111701E4A012111700422EDE7012191FAA1F21848120E0270184A05
S34500008A0000201070174A117005225A71164B1022CEE73C2292FAA2F21048120E0270104A0020107001200F4A014410705971CFE7382292FAA2F20949120E0A70084A00217A
S34500008A401170084A012111700822C0E764225A7170470022FBE700BF1A080020C70B0020C50B0020C60B0020F60500209A48018889B22DE9F84F51BB984B5A79652A55D035
S34500008A802BD8132A964E974C974D22D8002A38D0FFF774FF924A944B11781B78934C914801EB032189B2C4F8801002F03FFC03786BB172B6037801EB03239BB2C4F88030D8
S34500008AC002F034FC0023C4F88010037062B6BDE8F88F642A1ED000221AE0C92A4DD0FA2A5FD0C82AF7D19971902292FAA2F27C4C120E22707C4A11707A4A01211170C92284
S34500008B0012E0327022702A704FF4FA72028001225A71BFE79971802292FAA2F2120E327001222270297065225A711CE09A79112A1CD86F496A4C895C21706E49895C29B1E4
S34500008B406D490978C90744BF20212170217891FAA1F1090E2170644904240C700124614922440C709A710223038093E763498A7842F008028A70C822CAE79A79112A09D8D8
S34500008B805F49574C895C21705E49895C0029DDD05D49D6E759498A7842F010028A70FA22B6E75A4DAA79002A32D159485949DFF844E191F800C001784D4EDFF87881DFF854
S34500008BC078A1614588BF02700478122122464FF0200918F80270002F70D037701AF802700132D2B2013911F0FF010EF8017B06F10106EED1484E3278002A66D0013A3270AE
S34500008C003D490A7801320A70DA79AA7164225A71E879002840F0FE80404A414C1678414A94F800C092F800803F4ADFF8D890127806EB0801122940F38780944507D92F490B
S34500008C40207091F802C060F3410C81F802C0DFF8ECA0DFF8ACE0DFF8E8C02A4800215FFA81FBB345C0F0B180254FDFF8D8C0C8F1120157FA81FE2D4FC8B259FA81F111283F
S34500008C8040F2AD802A480178002900F0B380013901701D490A7801320A70DA79EA7164225A712A7A12B95A71FF232B720C4A002313700C4A13700C4A1370EBE6BCF1130F92
S34500008CC086F8009028BF00228CE7BCF1120F86BF01340470017093E7F60500201A080020C70B0020C60B0020C50B002000F00F40A909002085090020BC0900202C08002015
S34500008D009709002073090020BB0900200F080020C0090020440B0020BF090020C30A0020BE090020C1090020420A0020C2090020BD090020850B0020450B0020040B00202C
S34500008D40C40A0020020A0020C1F112019445C9B208D9DFF814C120709CF802E060F3410E8CF802E000293FF472AF3C4F207806EB090B06EB070E4FF0000C394F17F800A0F2
S34500008D805FFA8CF7BA4214D9BAF1000F11D0354F8EF800A017F800A00130C0B20CF1010C0BF801AB5FFA8CFA51450EF1010EE4D84DE791424FF0200738BF00208EF80070DF
S34500008DC02CBF4FF0000A8246E8E71AF801BB0EF801BB1CF801BB00F801BB01313FE71CF8019B0EF8019B013017F8019B01F8019BC0B244E732444244122AD8BF1A4A20780B
S34500008E00DBBF90782170421C61F34100CCBF227090703EE75A79642A3FF443AFFA2A7FF445AF124A0D481278114E124C124DC2F11202D1B250FA82F056FA82F2112902D97D
S34500008E40C8225A7132E714F8016B00F8016B013115F8016B02F8016BC9B2EFE797090020830A0020430A00202C080020C109002073090020020A0020C20900200E4A0F4866
S34500008E800023F0B553710E4A0E4F13800E4E0F4D0F4C104A1946013317F801CB06F801CBDBB214F801CB05F8011B122B00F801CB02F8011BEFD1F0BD1A080020970900202F
S34500008EC0F6050020C1D10000A909002085090020AFD100007309002030B50D4D0446002012F8013B33B90A4A2370917863F34511917030BD04F8013B21B1AB78C3F3401388
S34500008F0001F8013B3F289CBF431CD8B2E8E700BF2C0800202C4B2D489A6B42F4007210B59A639A6B42F480629A639A6B42F400629A639A6B42F480529A639A6B42F40052C3
S34500008F409A63234A4FF4407100249161D161016041601C6100F532204FF40073136053609360D360F023C0F8D4304FF48073136153619361D361A2F5005240F20311446550
S34500008F80116051609160D160116451649164D16440F2FF52C0F894200E4A136053609360D360136153619361D361136293624FF481735162D362084B44614FF4A0725A60A0
S34500008FC09A605A6110BD00BF0080044000D0044000C0044000B0044000900440024B00221A6026225A61704700F00F40014B00225A61704700F00F4008B50F4B0F4A5A6457
S345000090000F4801F0F9FD0F4B0F4A1A6000221146022001F097FD0D4A1378002103F0C703137008460A4A01F041FE0A4801F0A6FC094B0A4A1A6008BD0080044000000713E0
S3450000904024CC0000DC0500200024F40000400640DBD100002CCC00000800002000389C1C03685A1C02601878A0F16103192B01D8203870477F2882BF024B1B1813F8800CAC
S34500009080704700BF03D2000038B50023C3704FF0FF338363044602F0BCFA00284ED1B4F83A524AF655239D4227D094F83C30EB2B03D01833DBB2012B44D8B4F847305A1E2A
S345000090C01A423FD1B3F5007F3CD194F8490068B1431E18400AD194F84C30013B012B05D8B4F84D3013B1B4F852302BB94AF65520854214BF0320022038BD13490B2204F1F5
S345000091003C0002F05AF9D8B194F83C30EB2B03D01833DBB2012B0FD80C49082204F18E0002F04BF90028E7D0B4F847305A1E1A4202D1B3F5007FC8D00220DDE70420DBE7E7
S345000091400120D9E70320D7E7DED10000EAD100002DE9FF4100230B600F46164602F0B1F9051EC0F2C081B04B53F82540002C00F0BC813C60237806F0FE066BB1607802F05B
S34500009180E0F8C70708D40EB1410703D4002004B0BDE8F0810A20FAE70023E8B22370607002F0D4F8C20700F1A2810EB14307F1D400212046FFF768FF022840F095806E46C4
S345000091C004F2022304F242213246184602F0D2F810338B4242F8040BF7D1002556F8041B002978D02046FFF74FFF012874D80128A26B40F0B68004F146010B2311F8015FB1
S34500009200002D76D10133402BF8D1B4F8A430B3F5807F6ED194F8A830092B6AD104F1840002F0AAF84FF0FF33161841F10001B34275EB01035DD304F1900002F09BF894F815
S34500009240AA302062012BA37053D194F8A900834098B2608100284CD004F1980002F08AF880467248804544D808F10200E061626204F1940002F07EF88718276304F18C00C5
S3450000928002F078F89BB2024408FB03F0C01945EB0503864271EB0303A2622AD304F19C0002F068F82E46E06265B96389B34220D9E16A204602F08FF88119204602F0A9F932
S345000092C080B90136631993F83C30812B13D02035C5F30805E8E703200135042D7FF47EAF042806D1012052E70428FBD001287FF67EAF0D204BE705F1140004F13C063044B0
S3450000930002F038F801280546F3D9E3698342F0D96189236B821E02FB01336363A16A204601EBD51102F075F90028DBD105F07F0006EB800002F01EF8471C03D00135A84222
S34500009340ECD0D6E7C4E905000425394A2570138801339BB21380E380364BE360364B236114E7B4F84730B3F5007FC2D1B4F8526026B904F1600001F0FDFF064694F84C30F5
S345000093802662591E0129A370B3D894F8491061810029AED0481E0842ABD1B4F84D7027813807A6D1B4F84F0018B904F15C0001F0E1FFB4F84AE0BEF1000F9AD006FB03FC93
S345000093C00EEB17156544A84293D3431B8B42B3FBF1F08ED3194B98428BD80EEB02014FF6F57E704500F10203154429D840F6F57E7045C4E90921E36125630CD8002F3FF48D
S3450000940078AF0CEB010003EB430103F0010303EB5103012523E0002F3FF46BAF0CEB01005B0002251BE000BF90030020FDFFFF7F0808002008060020C80B0020F5FFFF0F43
S34500009440C4E90921B4F86610E361394325637FF450AF04F1680001F08DFF9B00032503F2FF13B6EB532FE062FFF443AF4FF0FF33C4E90533032D4FF0800323717FF465AFE2
S34500009480B4F86C30012B7FF460AF511C204602F0C0F800287FF459AFB4F83A2220714AF655239A427FF451AF04F13C0001F062FF104B98427FF449AF04F5087001F05AFF12
S345000094C003F1FF5303F50053203398427FF43DAF04F5097001F04EFFA06104F50A7001F049FF606131E70B2051E60C204FE603204DE600BF525261412DE9F047FF25066816
S3450000950004460F46A8460420A16B11B980B1042075E0304602F07DF8002870D1E06B0378002BF4D03278042A14D127B1832B60D10020BDE8F087852B5BD1236BE364204632
S3450000954002F073FD00285AD133691B7903F03F03A371EDE7C27AE52B02F03F02A27153D02E2B51D022F02001A1F1080CDCF1000141EB0C01B94247D10F2A4BD15A0641D5F6
S34500009580226B457BE26403F0BF03427BAA423BD1418B002938D10278D6F80CE0DFF88C9022F040024FF00D0C013A0CFB02F24FF6FF7A4FF0010C19F8018B30F80880BCF19D
S345000095C0000F24D0FF2A1FD82EF81280C446013201310D29EFD10178490607D5BCF1000F04D0FF2A10D800212EF81210013B5FFA83F80021204602F0BAFC002884D0002399
S34500009600A36396E79845C0D04FF0FF08F1E7D045DED0F9E7B8F1000F03D101F0E7FEA84286D04FF0FF33E36482E700BF83D200002DE9F04F002187B0D0F80090044602F05B
S34500009640D3F8804608BB99F80030042B3ED1D9F80C0001F0B0FF074600212046FFF74CFF054608B1804610E0D9F810309A8CBA42F2D193F823604FF0400AB54209D1D9F816
S345000096800C3033F81530002BE6D1404607B0BDE8F08F1AF01F0F08BF0AF1020AD9F8103033F80A0000F03AFCD9F80C30834633F8150000F033FC834503D10AF1020A013535
S345000096C0DBE7761BF6B2002EC6D1D8E74FF0FF33E3644FF0FF0A04F1400355460293A16B484601F096FF00285DD1E66B3778002F77D0F27AE52F02F03F03A37103D01207DD
S3450000970005D50F2B05D04FF0FF33E3644FE00F2B54D194F84B305B063FD4780645D5236B96F80DA0E36407F0BF07737B53453ED1738B002B3BD13578D9F80C30019305F007
S345000097403F05013D0D23DFF8A4B05D4301221BF8013BF35A6AB3FF2D29D81846059300F0DDFB019B0490691C33F81500039100F0D5FB049A82421AD1059B03991A460D461A
S34500009780194B9B45E3D13378590604D51AB1019B33F815305BB9013FFDB20021204602F0E6FB00289BD080466FE7BD42BDD0FF25F3E74FF6FF718B42E2D0F8E72DB93046EC
S345000097C001F014FE50453FF460AF94F84B30DB0799D402990B22304601F0EFFD002892D153E74FF0040850E790D2000083D200002DE9F04F90F84B5015F0A0059BB0044663
S3450000980040F0B9810668F26832F81530002B60D13378042B40F09C800F230E352046B5FBF3F5A91C02F068FC8046002840F08A80236B0135A3EB4513E364E3795F074AD577
S3450000984023F00403E371204602F0ACF800283ED1616B4FF0FF32204602F08CF8002836D1A368002B37D023680493236A0693636AA16A8DF8173004A823F0FF03CDE908381A
S34500009880CDF82C80179101F0AFFF00BB04A802F0CCFBE0B9D4E9042370894FF40071E0FB01233069C4E90423383001F071FD3069D4E90423283001F06BFDE379326943F015
S345000098C0010382F8213004A802F03EFC18B1804638E0013598E7D6E90354002140222046852301F064FD23700120C02384F820300A4640234FF0C10C8E4604EB00095E1CFE
S3450000990004F803C004F806E0023320B135F8110008B10131C9B2060AE05409F803600233DE06F2D135F81160571C7EB9023284F823106270284601F03EFE84F82400000A10
S3450000994084F8250040461BB0BDE8F08F3A46D6E704F140070C22394604A801F045FE9DF81BB01BF0010F72D04023DFF810A284F84B304FF001090B2204A93846D6F80C802A
S3450000998001F032FEB9F1050F56D9A8F102014B4631F8022F002A40D104A8072203F00F0C0CF13001392988BF0CF137010F2B00F8011D02F1FF324FEA13113FD802F168039C
S345000099C06B447E2103F8601C04F13F01084600239A4206D010F801CFBCF1200F03F1010E2ED1072A9CBF02F16800684403F1010396BF10F8600C20200132072BC854F0D9B0
S34500009A002046FFF715FE8046E0B909F10109B9F1640FB0D14FF0070894E7102002F0010C0CEB430313F4803F18BF83EA0A0301384FEA5202F2D1ABE74B46ADE70B46ADE73F
S34500009A407346C5E704287FF47DAF84F84BB01BF0020F1BBF0C350D230125B5FBF3F518BF01352946204602F047FB804600287FF469AF013D1AD1A16B304601F0CAFD80465C
S34500009A8000287FF45FAF01462022E06B01F08FFC0B22E06B394601F0A7FD94F84B30E26B03F0180313730123F3704BE7216B2046A1EB451101F098FE804600287FF442AFCD
S34500009AC0384601F093FC0190A16B304601F0A1FD804600287FF436AFF3680093E36B019A5A73E9B24FF00F024FF00D0CDA72DFF8908018734A1E0CFB02F29876D87684464C
S34500009B004FF0FF0918F801EB4FF6FF7A504503EB0E0B20D103F80E908BF801900CF1010CBCF10D0FEED14FF6FF7C604503D0009830F812200AB941F0400119700123F370E3
S34500009B400021204602F013FA804600287FF4FAAE013DB9D18FE7009830F8120003F80E0002F1010A020A8BF8012052460028D5D14FF6FF70D2E74FF00608E3E6211001006E
S34500009B8083D200002DE9F04FD0F800B087B00546019111F8013B2F2BFAD05C2BF8D00021019BA960E9611B781F2B00F212818023284685F84B3007B0BDE8F04F01F014BED8
S34500009BC0FE2E00F22D8129F81630013607E10123104612F8011B2F29F9D05C29F7D003B105900024059B0193A9F10202C6BB002229F81620002E00F0138139F81210202979
S34500009C00134602F10102F8D00BB92E2902D144F00304E4B2A9F1020131F816202E2A01D0013EF9D10B22202105F1400001F0BFFB4FF000084FF0080A474639F813005A1CEC
S34500009C40002800F0A180202803D02E2810D1B24212D044F00304E4B21346EEE70424C1E732F81630202B01D02E2BC0D1013EBDE7D04505D2B24246D1BAF10B0F3BD102E0AB
S34500009C80BAF10B0F31D195F84030E52B02D1052385F8403044F00304E4B207F00C030C2B03D007F00303032B02D144F00204E4B2A60709D4F80744BF44F01004E4B2790749
S34500009CC044BF44F00804E4B285F84B402846FFF7AFFC95F84B30002863D0042840F0A18013F0040F08BF05209BE0B24203D044F00304E4B248D8BF00FFB232464FF00B0A1D
S34500009D004FF00808A8E77F2839D944F00203DBB240F2B5110392029300F0CEF810F0800FDDE9023211D04F4900F07F00085C38B14D4C14F8011B002900F082808142F8D1C2
S34500009D4043F00303DBB25F2011E0FF28EFD90AF1FF31884504D344F00304E4B2D0467BE705EB0801040A81F8404008F1010805EB08011C4681F8400008F101086CE72346CC
S34500009D80D6E747F00207F2E795F84030E52B04BF052385F84030BAF1080F04BFBF00FFB27BE75A073DD4AB79DB0647D59BF80000042839D1AB682B622B69EA79DBF81000B5
S34500009DC023F0FF0313436B62EB6CAB62294602F017FA019B05932B68D3F80C90002605A801F0D9FB471C1BD0B0F5803F24BF030C29F8163083B228BF01361F2B7FF62EAF8F
S34500009E002F2B2CD05C2B2AD07F2B3FF6D9AE1749184611F8012B002A3FF4D2AE9042F8D1062007B0BDE8F08F2B6B0BF13C01C3F30803194402F0F9F9A860CAE70520F0E7ED
S34500009E40A0F1410189B219299BD9A0F1610189B219299EBF203847F0010780B287E7059A0023B5E603D20000FCD10000F3D100001FB5CDE9001003A81446039101F021FB11
S34500009E80002815DB0B4A52F820300BB100211970019B0BB10021197042F820302CB1002201A96846FFF754F90446204604B010BD0B24FAE7900300207F2801D880B27047AC
S34500009EC0B0F5803F11D240F2B51399420DD1084A002332F8021B814201D19BB202E00133802BF6D18033D8B270470020704700BF8ECF00007F280DD940F2B513994208D11A
S34500009F00FF2806D800F10040034B803833F8100070470020704700BF8ECF0000B0F5803FF0B522D21F4A204983B2B0F5805F28BF0A46141D34F8042C2146AAB1934213D331
S34500009F4034F8025C2E0AEFB252FA85F5A84223DA082E09D8DFE806F0050A10131517191B1D00801A34F810301846F0BD9A1A02F001029A1A93B2F7E7103B9BB2F4E7203BE9
S34500009F80FBE7303BF9E71A3BF7E70833F5E7503BF3E7A3F5E353F0E70434002ECAD101EB4702C6E79CCD0000E0CC00001A4B1B4800221A72D0F8902082F47F4282F0FF028A
S34500009FC0C2F34021120548BF41F002015972026D82F00F12C2F380414901900348BF41F010011972D10342BF197A41F004011972100742BF197A41F008011972510742BF0D
S3450000A000197A41F002011972920742BF1A7A42F001021A72704700BF1A08002000F00F4038B50B4CA3782A286FF3C713A3700DD0084D094901222846FFF71AFF30B9A378BA
S3450000A0402A7843F08003A370044B5A7438BD00BF2C0800209C030020C4D200001A08002000B5474B474A9A6097B0BFF34F8FBFF36F8F454B454C11221A70FEF7BDFFFEF7D6
S3450000A08049FF434A136823F00103136000F08EFB3223E371FEF7F2FEFEF704FCFEF730FC6379F92B3BD93B4DAB7800266FF3C7133046AB70667400F033FA374B1B681BB129
S3450000A0C031463046FFF7ACFF95F90230002B29DA002332492374684602F06DFB10BB304C304B2E4A2146684602F0E8FBD0B9628B44F250739A4215D1237F542B12D12A48D6
S3450000A100012204F11A0102F098F858B9FEF7E4F900F018FBFFF74AFFFEF7A8FCF6E7FEF7A5FCBDE74FF48033204A1968116059681F4B19601168013106D01968013103D092
S3450000A14012681B6895469F461A4A1B480021FEF7C3FE1A4B1A4A187000241A4B1A481C702146FEF7B9FE194B1870194B1C70FEF799FBFEF7C5FB00F0E5FAFEF777FCFAE771
S3450000A18000ED00E00080000000D007401A08002000D000402C08002080030020F2D100006002002090D200001000002098030020940300209ED00000850B0020440B002016
S3450000A1C0A4D20000C30A0020830A0020420A0020C1090020034B80221A701A781206FCD5704700BF000002402DE9F04F85B01E46B0F5004F9DF840309DF838909DF83CA091
S3450000A2009DF844709DF848800193154679D3019A07EA080313400AEA030309EA030333402B400B40FF2B6CD0034600F108041A78FF2A03F1010366D1A342F8D1334C30231B
S3450000A240237072B60723E371C0F30742C0F307235FFA80FBA27103926371029384F804B084F80B90A6726572217284F80F80A773019B637384F80CA0FFF7ACFF94F800C06C
S3450000A2801CF0310FDDE9023205D062B62078C0B205B0BDE8F08F4FF0020C84F807C0A271637184F804B04FF0010B84F80BB084F80F90A67365732173FFF78CFF237813F09A
S3450000A2C0310F02D062B62120E2E704304FF00203E371C0F30743A371C0F30723C0B26371207184F80BB084F80F80A773019B637384F80CA0FFF76EFF237813F0310FE1D1AA
S3450000A30062B60020C4E70420C2E700BF00000240B1F5004F2DE9F047154608D31C4C3023237072B601260027884202D962B6002018E0C0F3074AC0F307295FFA80F8E67146
S3450000A34084F806A084F8059084F80480E672A7726772FFF73FFF237813F0300F04D062B62078C0B2BDE8F0872378DB070DD50923E37184F806A084F8059084F80480FFF72F
S3450000A38029FF237813F0300FE9D12844CCE700BF00000240084A09494FF47A73138013889BB223B9064A13880133138002E0CB6A9B03F4D5704700BFF405002000C00240CC
S3450000A3C0F8050020032911D8DFE801F00702090D62B1074B1B685B0A1360002070472AB14FF40073F8E70AB10123F5E70420704780030020024B1868B0FA80F04009704727
S3450000A400800300201848036843F4806370B50360164BC362164B4363FFF7BCFF836BC36A144E43F40033C362134D4663FFF7B2FF846BAC73C36A43F40033C3624663FFF7A3
S3450000A440A9FF836BEB73C36A43F40033C3622306EAD50A4B4363FFF79DFF836BC36A43F40033C36270BD00BF00C0024000000A1AD7000180FF0001801A080020FF000108D3
S3450000A48070B5FFF7BFFF1F481F4C03681F4E43F4806303601E4BC3621E4B4363FFF77AFF836BC36A43F40033C3624463FFF772FF856BEDB2B570C36A43F40033C3624463BB
S3450000A4C0FFF768FF846BE4B2F470C36A43F40033C362114B4363FFF75DFF836BDBB23371C26A42F40032C2620C4A00211F2D116006D1272C04D1012B04BF4FF480031360CE
S3450000A50070BD00BF00C00240FF0001801A08002000000A1A9F000180FF0001088003002010B58AB02422002101A802F0A2FA184A937813F0010422D143F0010301A893708E
S3450000A54000F0F8FB134A8DF804400823CDE902232923CDE905330793022040F201130893ADF810408DF81240ADF8244000F07EFA01A90246084800F0D5FCFFF781FF074BE7
S3450000A5801868B0FA80F0400940000AB010BD00BF2C08002000366E0100C0024080030020012AF8B506460D465AD1FFF72BFF2D4B2D4C5A882D4F954288BF5D80236843F4C0
S3450000A5C0806323602A4BE3622A4B6363FFF7E2FEA36BE36AAD0243F40033E362C5F307433B436363FFF7D6FEA36BE36A43F40033E3622B0ADBB23B436363FFF7CBFEA36B7E
S3450000A600E36A43F40033E3626763FFF7C3FEA36BE36A43F40033E362002040F2FF15A84212D196F8FF3143F0006343F480336363FFF7B0FEA36BE36A43F40033E3620E4B4F
S3450000A64064229A700020F8BD335C3B436363FFF7A1FEA36BE36A43F40033E3620130DEE70320F0E7F805002000C002400000018000000A1A820001800F080020012A2DE9CE
S3450000A680F04106460D4650D1294CDFF8B480FFF7B9FE2368274843F480632360264BE362264B6363FFF776FEA36BE36AAD0243F40033E362C5F3074303436363FFF76AFE63
S3450000A6C02D0AA36BE36AEDB243F400330543E3626563FFF75FFEA36BE36A43F40033E3626063FFF757FEA36BE36A43F40033E362771E002540F2FF139D4215BF7B7896F8BD
S3450000A700FF31034343EA08036363FFF743FEA36B07F8013FE36A013543F40033B5F5007FE362E7D10020BDE8F0810320FBE700BF00C002400000018000000A1A03000180E3
S3450000A74000000108144A10B593786FF382039370124B1978F9B100211970114909230C4611F8010B10B1013801F8010C013B13F0FF03F5D10B490B7801330B70637853B90F
S3450000A78064236370937843F004039370064A13780BB1013B137010BD2C0800200B0800200F0800200C0800200E08002013B5144C002301A920468DF8043000F04FFC022035
S3450000A7C000F054F964210F4A0023A0FB010102F054F9C4F80001D4F8083143F00203C4F80831094B102283F830234FF480325A60D4F8083143F00103C4F8083102B010BD97
S3450000A8000070034040420F0000E100E01A4B0122C3F80C21194A13889BB21BB11388013B9BB21380164A13889BB21BB11388013B9BB21380134A13780133DBB2092B1370A4
S3450000A84016D900231370104B1A780AB1013A1A705A780AB1013A5A701A784AB90A221A700A4B01221A700A4A13780BB1013B1370BFF34F8F704700BF00700340F6050020C3
S3450000A880F40500200D080020180800200B0800200A080020034B1B7BDB0754BF024B034B1868704700400640DC050020D805002008B5114A9379D9061BD4FFF7EBFF88B165
S3450000A8C013785178127BC3F3C20311F0300F20FA03F0D2B206D0D20704D4062B03D0072B05D0400908BD1423B0FBF3F0FAE70C23FAE7024B1868F5E700400640040000207C
S3450000A900064B9A79D20753BF054B064A1B7A186842BF1068C3F34203D8407047004006400400002000000020034B1B781B0646BF024B18680020704700500640DC050020BE
S3450000A94008B50C4B1B68C3F38143022B0AD0032B0BD06BB9FFF7E8FFA0F5004358425841C00308BD044B1868FBE74FF47A70F8E70020F6E700700440D80500200C4A4368B0
S3450000A98002F5805110B54B6403784C681B0403F4803324F4803423434B60437811689B0403F4402321F440210B43136010BD00BF0070044010B50C4C63789A0701D500204D
S3450000A9C010BDA3799B06FAD4FFF772FF0028F6D0E378E278C3F341135B0003EBD213034A32F813305843EBE7004006408ED00000034B187810F0020001D0FFF781BF70470E
S3450000AA000040064008B5094A907910F040000CD0FFF740FF137903F01F030133B0FBF3F3507900F01F001830584308BD00400640034B5B68DB0301D4FFF7BCBFFFF7E2BFE8
S3450000AA4000800440084B9B79C3F38103022B09D0032B03D0012B03D1FFF752BFFFF7D2BFFFF7A8BFFFF716BF0040064008B5132848D8DFE800F00D0D161D24472B2F3347CD
S3450000AA8047373B3F43474747470A4FF47A7008BDFFF7D8FF1C4B5B6C1B0F0133B0FBF3F0F5E7FFF7CFFF184B5B6CC3F30363F4E7FFF7C8FF144B5B6CC3F30353EDE7FFF7DC
S3450000AAC0C1FF114B5B6CC3F30343E6E7BDE80840FFF7AEBFBDE80840FFF732BFBDE80840FFF722BFBDE8084001F07CBFBDE80840FFF77EBFBDE80840FFF75CBFBDE8084098
S3450000AB00FFF780BF0020C2E7008004400C4A137B03F0010383420CD0137B00F0010003F0FE030343137340F2DC5300BF013BFCD104E0117B01F0FE010B431373002070475E
S3450000AB400040064070B51E4B9C799D791E7AC6F342069642C4F38104EDB217D0ED070CD5012C02D01B789E0707D5154B5D7805F0FE055D709D79ED07FCD4114D2B7A52004C
S3450000AB8002F00E0203F0D0031A432A720C4A537801F0010503F0FE032B435370137803F0FC030343012C137001D0830705D5044A937903F001038B42FAD1002070BD00BFF4
S3450000ABC00040064042780B4B02F01F021A715979827801F0E00102F01F020A435A711A7901780A4342F040021A719A795206FCD5704700BF00400640016849F697039942A5
S3450000AC0010B522D9124B99428CBF02210121114A0479137803F0F003234313701378847903F05F0323430C4C13706378407903F0C303034343EA0113637028B113781A060B
S3450000AC4002D5A3799B07FCD510BD0021DFE700BF00127A00005006400040064010B5124B5A7802F0FD025A701A7802F03B0242F0800208461A709A7902F01C02082AFAD131
S3450000AC805A79094C02F0BF025A71A3799A06FCD4FFF798FF637943F040036371A3799B06FCD5002010BD00BF0040064038B515460C46FFF72BFF29462046FFF7CFFF064A46
S3450000ACC0137803F03F0313709379C3F38103032BFAD1002038BD00BF0040064008B50368002BB4BF034B044B1B689847BFF34F8F08BD00BFE4050020E0050020084B98425E
S3450000AD000AD003F58053984208D003F5FE23984214BF032002207047002070470120704700C0024008B5FFF7E9FF014B195408BD280E002008490822C0E901124FF47A726E
S3450000AD400023C0E90422826140F20112037083818373C2610384704720A107002DE9F04F87B00746049101680293002964DA00205B00039301250646844601464FF0FF3444
S3450000AD802E4B01932E4B53F821300593B2468046A64600260AE0B9F1100F47D0002C45D0B2468C46022580464E46A646019B53F8040B0193059B03FB00F9029BB3FBF9F06C
S3450000ADC082420BD3A2EB000B5C4507D9BBF1000F2FD0DE468046B2468C460125039BB3FBF9F0824206F1010902D3141A7445D2D3B9F1100F17D140465646744601310429B7
S3450000AE0001D0002CBCD1049B07EB83070D4BFA681340334343EA0C43013D43EAC573FB6007B0BDE8F08F74464046BCE78C460225E4E78C460125E6E70020F1E790CC0000CF
S3450000AE40D0CC0000F0FFFC7F2DE9F04F1746026887B0002A039005915ADA109D2D4AB2FBF3FC4FF4E0222C4CB4FBF3F302FB0CF2B5EB430F4FEA92024FEA430430D9DFF8C0
S3450000AE809CA014460F2300254FF0FF3103225AF8040BDFF88CB000FB0CF004909846A14608460023049C5BF8041B109E6143B6EB910F4FEA910403F1010E02D8A11B814207
S3450000AEC017D3BEF1100F1FD14C46434601460135042D01D00029DAD105990398009702E0002300971A4601F08BFD204607B0BDE8F08FBEF1100F2A46E9D00029E7D09846FB
S3450000AF00A14608467346CDE701464C464346F6E70024EAE700286BEE00CA9A3B80CC000040CC0000F7B50446FFF7E8FE404B0D4653F820100B0C03F1804303F58E231646BF
S3450000AF40186889B201228A4002431A602368AA7F23F480432360236843F001032360236843F000432360236823F08A4323F44C5343EA827395F8202043EA8263EA7F43EAD2
S3450000AF80026395F82120120202F44072134323602B7F697F22681B04012903F47C130CBF134322EA030323602F786A68334639462046FFF7D3FEA86804EB87020138D36888
S3450000AFC0C00623F0FE4300F0F04018432B7B9B0603F0806318436B7B5B0603F000731843AB7B1B0603F0807318432B69D06039460093012233462046FFF726FF6B69009354
S3450000B0003946334602222046FFF71EFFAB6900933946334603222046FFF716FF00212046FFF780FE236823F00103236003B0F0BD34CC0000024B03481968FFF74FBE00BFE5
S3450000B040E805002000C00240024B03485968FFF745BE00BFE805002000D00240094AD36B43F40003D363036823F0020303600B7823B1036823F0010303607047036843F013
S3450000B0800103F9E700800440084AD2F8883043F47003C2F88830064B4CF22052DA814DF62812DA814FF4E9721A80704700ED00E00020054008B5FDF7B2F808BD08B5FDF7CC
S3450000B0C0AEF808BD08B5FDF7AAF808BD08B5FDF7A6F808BD08B5FDF7A2F808BD08B5FDF79EF808BD08B5FDF79AF808BD08B5FDF796F808BD08B5FDF792F808BD08B5FDF7DA
S3450000B1008EF808BD08B5FDF78AF808BD08B5FDF786F808BD08B5FDF782F808BD08B5FDF77EF808BD08B5FDF77AF808BD08B5FDF776F808BD08B5FDF772F808BD08B5FDF799
S3450000B1406EF808BD08B5FDF76AF808BD08B5FDF766F808BD08B5FDF762F808BD08B5FDF75EF808BD08B5FDF75AF808BD08B5FDF756F808BD08B5FDF752F808BD08B5FDF759
S3450000B1804EF808BD08B5FFF755FF08BD08B5FFF75BFF08BD08B5FDF742F808BD08B5FDF73EF808BD08B5FDF73AF808BD08B5FDF736F808BD08B5FDF732F808BD08B5FDF7E7
S3450000B1C02EF808BD08B5FDF72AF808BD08B5FDF726F808BD08B5FDF722F808BD08B5FDF71EF808BD08B5FDF71AF808BD08B5FDF716F808BD08B5FDF712F808BD08B5FDF7D9
S3450000B2000EF808BD08B5FDF70AF808BD08B5FDF706F808BD08B5FDF702F808BD08B5FCF7FEFF08BD08B5FCF7FAFF08BD08B5FCF7F6FF08BD08B5FCF7F2FF08BD08B5FCF781
S3450000B240EEFF08BD08B5FCF7EAFF08BD08B5FCF7E6FF08BD08B5FCF7E2FF08BD08B5FCF7DEFF08BD08B5FCF7DAFF08BD08B5FCF7D6FF08BD08B5FCF7D2FF08BD08B5FCF728
S3450000B280CEFF08BD08B5FCF7CAFF08BD08B5FCF7C6FF08BD08B5FCF7C2FF08BD08B5FCF7BEFF08BD08B5FCF7BAFF08BD08B5FCF7B6FF08BD08B5FCF7B2FF08BD08B5FCF7E8
S3450000B2C0AEFF08BD08B5FCF7AAFF08BD08B5FCF7A6FF08BD08B5FCF7A2FF08BD08B5FCF79EFF08BD08B5FCF79AFF08BD08B5FCF796FF08BD08B5FCF792FF08BD08B5FCF7A8
S3450000B3008EFF08BD08B5FCF78AFF08BD08B5FCF786FF08BD08B5FCF782FF08BD08B5FCF77EFF08BD08B5FCF77AFF08BD82B006230193019B5A1E01920BB902B0704700BF65
S3450000B340F7E708B9FFF756B80120704708B9FFF7E7B80120704708B901F03ABB0420704708B901F02BBB0420704708B9FFF72AB8042070470068704703460068596870476D
S3450000B3800B0A017043700B0C090E8370C1707047110A02704170110C120EC2701A0A037142711A0C1B0E81708271C3717047024400F8011B9042FBD1704710B5034602442C
S3450000B3C013F8010B11F8014B9342A0EB040001D00028F5D010BDC3690239023B8B4283BF4389006B01FB030000207047034600F10B010020C20142EA500213F8010B50FA24
S3450000B40082F28B42D0B2F5D1704710B5417804460131002049010246022A08BF0422A35C03EBC0339BB2013203EB5003914298B2F2D810BD7FB5044601911D46114621B908
S3450000B44023785BB955B1012006E001A8FDF708FE01390028F3D1002004B070BD019B02940393029803783F2B01D02A2B1CD100231A4610F8011B3F2901780CBF013201233C
S3450000B4803F29F6D02A29F4D0039E02903146FFF7D1FF0028D7D1317801A8FDF7E1FD002DD9D00029DAD1D6E702A8FDF7D9FD064603A8FDF7D5FD86420146EDD1002ED0D1A9
S3450000B4C0C1E703684BB11A4612F8011B1F290BD93A29F9D11978302902D04FF0FF30704702339A42F9D102600020704738B50D46044618B9092000232B6038BD0368002BA6
S3450000B500F8D01A78002AF5D08188DA889142F1D15878FFF716FF10F00100EBD12368EBE738B5C3780446C3B100F13C05826B407801232946FFF714FF88B9A16BA36A226A88
S3450000B540E070CB1A934208D2A378022B05D10A44607801232946FFF703FF002038BD0120FCE738B50D4640F2B5111446FEF7A4FCFF2806D9012C0AD9030A68702B7002201A
S3450000B58038BD0028FCD024B128700120F8E70020F6E72046F4E738B50568044615F8010B20B140F2B511FEF7A5FC08B1256038BD4FF0FF30FBE738B50546002435F8020BBC
S3450000B5C008B9204638BDFEF7A9FC620802EBC432C3B213FA82F292B2C0F3072303EB520303EBC2339CB2E9E701380A4411F8013B00F8013F9142F9D17047C2F307238A76B0
S3450000B600CB760378032B01BF120C0A75120A4A75704738B5836B8B4205460C4610D0FFF77FFF60B922466878012305F13C01FFF792FE00281CBF4FF0FF340120AC6338BDBA
S3450000B6400020FCE702392DE9F047466B01F007044FF0010A0AFA04F405461746984606EB1136C1F3C809E4B2314628460136FFF7D0FF18B10120BDE8F087994605EB0902AC
S3450000B68092F83C30234214BF01210021414514D06340013F82F83C3085F803A0EBD0640014F0FF04EAD109F10103B3F5007F4FF001044FF00009E0D1D6E70220DBE70129B2
S3450000B6C0F8B50C4640F28B800668F3698B4240F286803378013B032B00F28180DFE803F00229374A01EB5105B16A304601EB5521FFF78FFF10B14FF0FF30F8BD6F1CB16A88
S3450000B700C5F30805354401EB5721304695F83C50FFF77FFF0028EED1C7F30807374497F83C3045EA0320E3074CBF0009C0F30B00E3E7B16A304601EB1421FFF76AFF002827
S3450000B740D9D1640004F4FF743444A08FD5E7B16A304601EBD411FFF75CFF0028CBD1A40006F13C0004F4FE742044FFF703FE20F07040C2E7D0E9043153EA0102C57901D02E
S3450000B780826802B95DBB82687789022DA4EB02020CD1013B41F1FF315B0A43EAC153B3FBF7F39A421BD81CD0601CA6E7032D02D183699342F8D8C3699BB9B16A304601EB0C
S3450000B7C0D411FFF726FF002895D1A0003C3600F4FE703044FFF7CEFD20F000408DE701208BE76FF0004088E7F8B505682B78042B0CBF4FF080524FF400128A4206460C4620
S3450000B80001D80220F8BDCA06FBD18268016312BB022B12D82B89B3EB541FF2D9E86AC6E90D200028EDD000EB54203C35C4F308042544B063F5630020E4E7EB6AC271002BDC
S3450000B840E8D06F891A467F02BC42114605D22846FFF7C1FDE3E71346F3E73046FFF72FFF431C024606D00128CBD9EB698342C8D9E41BE9E70120C5E701292DE9F8430646E5
S3450000B8800C46154608D9C3698B4205D90378022B5ED003D8012B21D002204FE0033B012BFAD8816A01EBD411FFF7B3FE002845D13278A40006F13C0304F4FE74042A23449E
S3450000B8C007D01846FFF756FD25F0704500F07040054329461846FFF753FD2CE001EB5107816A01EB5721FFF794FE38BB06F13C0807F10109C7F3080714F001041FBF18F8E8
S3450000B90007202B0103F0F00302F00F0214BF1343EBB208F80730B16A0123F37001EB59213046FFF776FE48B9C9F3080944B1C5F3071508F809500123F3700020BDE8F88329
S3450000B94018F80930C5F3032523F00F031D43F0E7816A01EB1421FFF75CFE0028EED1640006F13C0304F4FF741A191D55C5F307255570E0E7F8B504460E461746E3690BB927
S3450000B9801846F8BD012BA6EB030514BFAA1C3A462068691CFFF770FF0028F2D1E369013BE361EBE770B5C379032B044601D0002070BD81688369CD18A94202D10023E371AF
S3450000B9C0F5E74E1C20683246FFF756FF0028EFD13146F1E701292DE9F843056806460C46174602D80220BDE8F883EB698B42F9D97AB9A14621463046FFF761FEA04604460B
S3450000BA00B0B92B78042B02D1002F44D1F7710020E9E72B78042B02D1C379022BE9D04FF0FF3239462846FFF727FF0028E1D0DAE70128D7D0421C01D10120D4E72B78042BCE
S3450000BA4010D1D5E90632023A934213D308F10102A24203D02B78042B13D0A146EB69A342C8D8CEE7002241462846FFF705FF0028E7D0B8E70133AB612B7943F001032B71CF
S3450000BA80E4E70023A2EB090249462846FFF7DAFD0028E2D0A7E7F3798BB9B468BC4202D10223F371B3E721463046FFF708FE012898D9431CC0D001348442EFD0A7E7032B30
S3450000BAC0A5D1B368BB42A2D8B2691344BB42E7D29DE7F8B504460E46FFF722FD0546F8B931462046FFF777FC04F13C070646A0634FF4007229463846FFF759FC63899D42AB
S3450000BB0004D36089401B18BF0120F8BD6078012372193946FFF724FC0028F2D10135EDE70120F2E7F8B50446FFF7FAFC0546002842D12378032B37D12779012F34D104F128
S3450000BB403C0601464FF4007230465523FFF72FFC84F83A32AA2384F83B3252234122722184F83C3084F83D30612384F83E3084F8233284F83F2084F8201284F8211284F8A5
S3450000BB802222A16904F50970FFF7FAFB616904F50A70FFF7F5FB626A60780132A2633B463146FFF7DDFB2571002260781146FFF7DCFB003818BF0120F8BD2DE9F843002500
S3450000BBC0D0F800808D76836B07460C4633B398F80030042B47D1D8F8108040272E462B4698F8232095421BD303B916B93F23A376012626440023B376637398F80430237323
S3450000BC00DB062DD408F13800FFF7B6FBC4E90001B8F80C306381B8F80E302381BDE8F883B7F5187FE2D2FA0608BF0237013538F8070002372BB900F5205292B2B2F5006FD2
S3450000BC400CD306F11A01C6F1FF02214440EA0340FFF787FC0028C9D0064400200346BFE700200146D2E7C36C013343D1F96B00234F1E1D464FF02E0C17F8012F202A05F1CA
S3450000BC8001053ED0052A08BFE522092D03F1010004EB030633D10B2B9FBF001986F80DC00233427384BF72730346E5E7B9F1000F05D100F520539BB2B3F5006F0BD305F1F8
S3450000BCC01A01C5F1FF02214440EA0940FFF749FC98B10544002002368146D8F80C30985B0028E3D1B9F1000F18BF002525440023AB76BBE72E46A946EFE70546F2E7727387
S3450000BD0003460B2DB8D1E21800205073A27E92B943B104F10C0308255A78581CC2B91B1B0C3B02E03F23A3760123234400229A760B7B03B96373CB7A237301F11C00FFF737
S3450000BD4019FB002320606360CB8A63810B8B64E72E2A0AD01346413A192A03D80A7B154200D0203343730346D6E710251346F9E72DE9F047056807468846002939D1D5E916
S3450000BD800563002E4AD0EA69B24247D91BB900242046BDE8F0872B78042B45D1EB69B41E023B9C4228BF0024A1464FF0010A696B284601EB1931FFF72CFC00287FD1EA6926
S3450000BDC009F007030AFA03F3C9F3C801DBB2A2F1020C6A1892F83C0009F10102624500EA03003AD3002839D0002C39D000229146DDE7FFF764FC0128044601D80124C7E70F
S3450000BE00421C00F0B180EB698342C1D8AA69002ABDD02A78042A79D14646BFE7002BB6D02B78042B16D001263446EB690134A34202D8012EABD0022421463846FFF73FFC7D
S3450000BE4000287DD00128D9D0013000F08D80B442EBD19CE700240126A6E718BB09F10204631E033394D801231A4621462846FFF7E9FB0228C2D0012876D0B8F1000F23D13A
S3450000BE800223FB710028B9D1D5E90632023A93429CBF03F1FF33AB612B796C6143F001032B7175E7A2420DD05B0013F0FF0304D10131B1F5007F9AD00123914689E74FF0A4
S3450000BEC0FF34CDE70024CBE7FB79022B07D1731CA342D7D0BB68F31ABB610323FB7108F10102A242FB690BD00BB90123FB61224641463846FFF73EFD98BB0123FB61C3E78F
S3450000BF0013B10133FB61BDE70223FBE708F10104A34298BF022421463846FFF7D0FB01283FF46CAF431C1FD038B16E69012E05D9EB699E4228BF464676E70CB9464673E7B5
S3450000BF404FF0FF3221462846FFF796FC48B9B8F1000F99D0224641462846FFF78DFC002892D001287FF44AAF4FF0FF3410E72DE9F8430668076B3378042B14BF4FF4001334
S3450000BF804FF080532037BB429CBF00238363836B0446894673B1C7F30808B8F1000F3CD1416B0133836341B93389B3EB571F34D80023A3630420BDE8F8837389013B13EAB9
S3450000BFC057232AD1FFF77BFB0128054601D80220F1E7421C01D10120EDE7F369834216D8B9F1000FE4D0616B2046FFF7C1FE0546C8B10128EBD0431CEDD001463046FFF714
S3450000C00068FD0028E7D1E37943F00403E371656329463046FFF7DFF9A0633C3646442763E6630020C7E70720C5E72DE9F04105460068A96B0669FFF7ECFA044620B9E96B0D
S3450000C0400B78852B03D002242046BDE8F08120223046FFF7C9FA777801377F01A7F16003B3F5007FEFD821462846FFF780FF04280446E8D00028E7D1A96B2868FFF7C9FA5C
S3450000C08004460028E0D1E96B0B78C02BDBD12022B018FFF7A9FA96F823300F222C33B3FBF2F3B7EB431FCED34FF0400800212846FFF75DFF04280446C5D00028C4D1A96B59
S3450000C0C02868FFF7A6FA04460028BDD1E96B0B78C12BB8D106EB0800202208F12008FFF783FA4745E2D83046FFF78FF97488241A18BF01246400A7E7F8B50E460021076806
S3450000C1000446FFF771FB98B90546A16B3846FFF780FA68B93A78E36B042A1B780CD11B060ED5054601212046FFF721FF0028ECD0042808BF072006E0E52B01D0002BF0D15A
S3450000C1400135B542EED1F8BD03682DE9F0411E6905463046FFF759F9B070000AF070E96C77782846FFF740FB4FF0010804462CB1022C28BF0224E0B2BDE8F081A96B286873
S3450000C180FFF747FA04460028F2D1E86B20223146FFF72AFA2B6883F80380002FE8D021462846FFF7E4FE20360446013FDFE7C16CF8B54B1C0568066B04461CD10127A16B92
S3450000C1C02846FFF726FA90B92B78E26B042B0ABF1378E52303F07F031370EF70236BB3420DD200212046FFF7C2FE0028E7D0042808BF022003E0FFF7F7FA0028DED0F8BDB2
S3450000C20010B504463430FFF7B5F8886004F138000A46FFF7B1F8C2E9040194F8213003F00203D3710023D36110BD03284B8B04BF8A8A43EA0243184670472DE9F04F9BB0F2
S3450000C240164601910446002800F0328102F03F094A4603A901A8FCF77BFF074648B9039D0199049504A8FDF78DFC48B116F01C0F1AD100232360074638461BB0BDE8F08F6A
S3450000C2809DF95B30002BC0F20D8116F01C0F9DF8163040F0A680D80600F10681B10742D5DA0740D50720E4E70428E2D104A8FDF79FFA0028DDD149F0080919F0080F287885
S3450000C2C036D0042840F096802E69256021463046FFF796FF00211E22B01CFFF768F828691A222630FFF763F82B6920221A712B6960225A7221229A725822DA7219722B69CE
S3450000C300012283F8212004A8FFF71EFF0028B0D1A16841B102462046FFF75CFBA668013E6E610028A5D119F0080F18BF49F04009AB6B1399A364E1642878042840F08A8073
S3450000C340069B2362089B9DF81720286923F0FF0313436362179BA3622146FFF751FFEB88A3804FF0000A0022002304F15008C4E90E23256084F8309084F831A0C4F844A000
S3450000C3804FF4007251464046FFF711F819F0200F3FF472AFD4E9046956EA09033FF46CAFB5F80AB0A1684FEA4B2BB3457AEB0903C4E90E6959D22046FFF781F9B6EB0B06F7
S3450000C3C069F100090128014668D9431C68D0B3457AEB0903EFD30020216400287FF449AF44E013F0110F7FF45DAF76077FF565AF08203EE71399FFF718FF6023CB73212353
S3450000C4000B7458234FF000084B742023CB72064681F80E8042462846FFF7EFF8012381F81C8081F81D8081F81E8081F81F80EB70002E3FF478AF4246314604A8D5F838A09F
S3450000C440FFF7C8FA00287FF414AF51462846FFF7E0F864E7FFF7E9FEA06001F11C00FEF789FF00232061636179E72164C6F30803002B3FF401AF2846FEF7ADFFB0B1760A0B
S3450000C48046EAC95682196264687801234146FEF762FF00283FF4F0AE0120EAE602209BE7012099E70620E4E60420E2E60220E0E60927E1E62DE9F04F9A4687B0002388469E
S3450000C4C0CAF8003005A904461646FFF70FF8054690BB94F831507DBB94F8303013F00103019300F0AB80D4E90432D4E90E011B1A62EB0102B34272F1000238BF1E4604F188
S3450000C50050030293C6B1D4E90E01C0F30803002B40F08580DDF81490B9F80A20430A013A43EAC1531A401AD1014309D1A06801280DD8022584F83150284607B0BDE8F08FA9
S3450000C540216C03922046FFF7BAF8039AEFE7431C04D10123019D84F83130EDE72064216C4846FEF738FF0028E3D0B6F5007F02EB000733D3B9F80A1002EB562088424FEA70
S3450000C580562B88BFA1EB020B99F801005B463A464146FEF7E0FE0028DBD194F93020002A0BDA606CC01B584507D24FF4007204F1500108EB4020FFF717F84FEA4B27DAF85A
S3450000C5C000303B44CAF80030D4E90E32DB1942F10002C4E90E32F61BB84493E7626CBA421CD094F9303099F80100002B04F150010CDA01230391FEF7B3FE0028A9D194F8E2
S3450000C6003030039903F07F0384F8303099F8010001233A46FEF79FFE00289AD16764A16B029BC1F30801C1F50077B74228BF37463A4619444046FEF7D7FFC0E707257BE72E
S3450000C640F0B599B001A90546FEF750FF044600287DD195F8303013F0400478D01B06019E0FD56A6C7078012305F15001FEF778FE002840F0918095F8303003F07F0385F8D1
S3450000C68030303378042B65D12846FFF78BF9044600285CD1296C4FF0FF322846FFF76AF90446002853D12B6802932B6A04936B6A8DF80F3023F0FF03CDE90630A96A099081
S3450000C6C002A81591FFF790F8044600283FD102A8FFF7ABFC0446002839D13269137943F020031371EB79326943F0010382F821303069A9683430FEF743FE3069D5E904235D
S3450000C7003830FEF745FE3069D5E904232830FEF73FFE336960225A7321229A7358221C73DA7333695C75336902A81C745C749C74DC74FFF709FD044648B93046FFF7F2F9A9
S3450000C74095F8303023F04003044685F83030204619B0F0BDA96C3046FEF75BFF04460028F5D1EF6CFB7A43F02003FB722868AA683946FEF742FF296907F11C00FEF700FED8
S3450000C7806023FB7521233B7658237B760123BC75BC74FC74F370D0E70124D8E713B50446FFF74EFF28B901A92046FEF79FFE00B9206002B010BD30B585B00446019100287E
S3450000C7C03BD0002203A901A8FCF7C2FC48B9039D019925602046FDF7D5F928B1042800D105200023236021E094F94B30002B13DBA379DB06F4D52878042819D1A368236249
S3450000C8002369E279286923F0FF0313436362E36CA3622146FFF7F4FCEB88A38000212046FEF7E2FF0428DBD00028DAD105B030BDE16BFFF7FAFCA060EEE70920F6E773B52F
S3450000C8400D4601A90446FEF751FEC8B935B92946204602B0BDE87040FEF7C6BF01462046FCF74AFE10F0FB060AD129462046FFF7A4F931462046FFF77AFB042808BF0020DB
S3450000C88002B070BDF8B506460C46FFF7D8FF054690B98CB104F11A07A37E6BB10023306D1A463946FEF7C6FD30B921463046FFF7C6FF0028F0D005462846F8BD38B50D46E9
S3450000C8C0036511460446FFF776FF28B929462046BDE83840FFF7D6BF38BD70B5BCB00222019003A901A8FCF733FC78B9039C0199109410A8FDF746F940B99DF98B30002B40
S3450000C90045DB9DF84660F30702D507203CB070BD20780494042806F0100627D1206904A9FFF76EFC069DBEB1DDE90823CDE92A239DF81730269428958DF89F30002126A8F3
S3450000C940FEF752FF0028E1D1014626A8FCF7D4FD0028DAD00428D9D110A8FFF728FC0028D4D165B92046FFF7DDF8CFE71F99FFF75CFC0546002EEFD026942890DEE70246AF
S3450000C980294604A8FFF726F80028BFD1EAE70620BCE704207146084202D0EFF3098001E0EFF3088081690A884BF6AB639A4200D0FEE70231816120210160704708B508466E
S3450000C9C011461A46FDF7ECFD003818BF012008BD08B5084611461A46FDF750FE003818BF012008BD10B5FDF763FF044610B90024204610BDFEF726F8B4EBD00FF7D8F7E7EC
S3450000CA0030B505689DF80C40002D14DA022C13D0032C20D0012C0ED100EB81009205C1681B039BB202F440021A4321F4400323F470431A43C26030BD00EB81001205C16800
S3450000CA401B0203F4706302F440121A4321F4401323F47063EDE700EB81009204C1681B01DBB202F440221A4321F4402323F0F003DFE700F0BDB8FDF7F3BA5FF0000C30B5EB
S3450000CA801C0022D112006FD0914206D305460846002100F06FF80446284600F06BF80A462146BDE830401CF0404F08BF704703D54942404261F100015FEA8C0C38BF70479C
S3450000CAC05B42524263F10003704742D41C0C04BF1B040CF1100C13F07F4F04BF1B020CF1080C13F0704F04BF1B010CF1040C13F0404F04BF0CF1020C5FEA83035CBF0CF101
S3450000CB00010C5B00CCF1200E22FA0EF4234302FA0CF200FA0CF520FA0EF001FA0CF4204321FA0EF114461A4600F024F8A4FB0023AA1A71EB03033CBF1B190138CCF1200E92
S3450000CB4022FA0CF203FA0EF4224323FA0CF30021A7E7821A71EB03033CBF02460B464FF0000141F100009CE700200021BDE8304000F03DB80423B1EB122F09D2090241EA8F
S3450000CB8010610002013B08BF7047B1EB122FF5D30018494134BF9142891A4041494134BF9142891A4041494134BF9142891A4041494134BF9142891A4041494134BF914265
S3450000CBC0891A4041494134BF9142891A4041494134BF9142891A4041494134BF9142891A4041A3F1010313F00F0FD2D170477047034613F0030F0ED101F0FF0141EA01216A
S3450000CC0041EA0141043A24BF43F8041BB2F10402F9D202F10402013A24BF03F8011BFAE77047FFFF0024F4000004800001020000000011000C003C100D003C100C00301021
S3450000CC4002000000040000000800000010000000200000004000000080000000000100000002000000040000000800000010000000200000004000000080000000000100B0
S3450000CC80010000000300000005000000070000000200000004000000060000000800000010000000200000004000000080000000000100000002000000040000000800004B
S3450000CCC000100000002000000040000000800000020000000300000005000000070000007D1D0100632C001E9601A01E5A01001F0806101F0606201F0806301F0806401FC4
S3450000CD000606511F0700591F521F5B1F541F5D1F561F5F1F601F0806701F0E00BA1FBB1FC81FC91FCA1FCB1FDA1FDB1FF81FF91FEA1FEB1FFA1FFB1F801F0806901F0806D4
S3450000CD40A01F0806B01F0400B81FB91FB21FBC1FCC1F0100C31FD01F0206E01F0206E51F0100EC1FF31F0100FC1F4E210100322170211002842101008321D0241A05302C89
S3450000CD802F04602C0201672C0601752C0201802C6401002D260841FF1A03000061001A03E0001703F8000703FF00010078010001300132010601390110014A012E01790106
S3450000CDC0060180014D0043028101820182018401840186018701870189018A018B018B018D018E018F0190019101910193019401F60196019701980198013D029B019C0162
S3450000CE009D0120029F01A001A001A201A201A401A401A601A701A701A901AA01AB01AC01AC01AE01AF01AF01B101B201B301B301B501B501B701B801B801BA01BB01BC01C2
S3450000CE40BC01BE01F701C001C101C201C301C401C501C401C701C801C701CA01CB01CA01CD011001DD0101008E01DE011201F3010300F101F401F401F801280122021201B8
S3450000CE803A020900652C3B023B023D02662C3F0240024102410246020A015302400081018601550289018A0158028F015A0290015C025D025E025F029301610262029401A0
S3450000CEC06402650266026702970196016A02622C6C026D026E029C01700271029D01730274029F0176027702780279027A027B027C02642C7E027F02A60181028202A90127
S3450000CF008402850286028702AE014402B101B20145028D028E028F0290029102B7017B030300FD03FE03FF03AC0304008603880389038A03B1031103C2030200A303A30360
S3450000CF40C4030803CC0303008C038E038F03D8031801F2030A00F903F303F403F503F603F703F703F903FA03FA033004200350041007600422018A043601C1040E01CF04E9
S3450000CF800100C004D0044401610526040000C700FC00E900E200E400E000E500E700EA00EB00E800EF00EE00EC00C400C500C900E600C600F400F600F200FB00F900FF008C
S3450000CFC0D600DC00A200A300A500A7209201E100ED00F300FA00F100D100AA00BA00BF001023AC00BD00BC00A100AB00BB009125922593250225242561256225562555259F
S3450000D0006325512557255D255C255B251025142534252C251C2500253C255E255F255A25542569256625602550256C25672568256425652559255825522553256B256A2536
S3450000D04018250C25882584258C2590258025B103DF009303C003A303C303B500C403A6039803A903B4031E22C603B50329226122B1006522642220232123F7004822B0007B
S3450000D0801922B7001A227F20B200A025A0008002DC020005B80580079508000A710B455A63616C4D617820555044415445763500434845434B494E47202E2E2E0050524F60
S3450000D0C04752414D4D494E47202E2E2E0046494E49534845443A0044454C455445204641494C4544210046494C452044454C4554454400494E56414C494420533139204690
S3450000D100494C45005331392046494C452052454144204641494C55524500464154424F4F54204D49534D4154434821205553452055502D4152524F57205550444154452E6D
S3450000D1402E2E004F55542D4F462D4F52444552205331392046494C4500464C415348204552415345204641494C55524500464C415348205752495445204641494C55524566
S3450000D18000505245535320454E54455220544F2044454C4554450050524F424C454D213F004B32324642657A63616C6D6178005354415254494E47202E2E2E2020202020F5
S3450000D1C02050475420455A63616C4D61784642202020200702000000000000000700EB7690455846415420202000464154333220202000222A3A3C3E3F7C7F002B2C3B3D7F
S3450000D2005B5D00809A45418E418F804545454949498E8F9092924F994F555559999A9B9C9D9E9F41494F55A5A5A6A7A8A9AAABACADAEAFB0B1B2B3B4B5B6B7B8B9BABBBC5A
S3450000D240BDBEBFC0C1C2C3C4C5C6C7C8C9CACBCCCDCECFD0D1D2D3D4D5D6D7D8D9DADBDCDDDEDFE0E1E2E3E4E5E6E7E8E9EAEBECEDEEEFF0F1F2F3F4F5F6F7F8F9FAFBFC88
S3450000D280FDFEFF01030507090E10121416181C1E504754455A43414C4D41582E5331392E545854004E4F20434F444521205553452055502D4152524F5720555044415445EA
S3450000D2C02E2E2E002F00FFFF00093D000080000000004001FFFFFFFFFFFFFFFFFFFFFFFFFFFFFFFFFFFFFFFFFFFFFFFFFFFFFFFFFFFFFFFFFFFFFFFFFFFFFFFFFFFFFFFF96
S3450000D300FFFFFFFFFFFFFFFFFFFFFFFFFFFFFFFFFFFFFFFFFFFFFFFFFFFFFFFFFFFFFFFFFFFFFFFFFFFFFFFFFFFFFFFFFFFFFFFFFFFFFFFFFFFFFFFFFFFFFFFFFFFFFFFF27
S3450000D340FFFFFFFFFFFFFFFFFFFFFFFFFFFFFFFFFFFFFFFFFFFFFFFFFFFFFFFFFFFFFFFFFFFFFFFFFFFFFFFFFFFFFFFFFFFFFFFFFFFFFFFFFFFFFFFFFFFFFFFFFFFFFFFFE7
S3450000D380FFFFFFFFFFFFFFFFFFFFFFFFFFFFFFFFFFFFFFFFFFFFFFFFFFFFFFFFFFFFFFFFFFFFFFFFFFFFFFFFFFFFFFFFFFFFFFFFFFFFFFFFFFFFFFFFFFFFFFFFFFFFFFFFA7
S3450000D3C0FFFFFFFFFFFFFFFFFFFFFFFFFFFFFFFFFFFFFFFFFFFFFFFFFFFFFFFFFFFFFFFFFFFFFFFFFFFFFFFFFFFFFFFFFFFFFFFFFFFFFFFFFFFFFFFFFFFFFFFFFFFFFFFF67
S3450001000000000120C50101000D0201007F1B0300110201001302010015020100000000000000000000000000000000001702010019020100000000001B0201001D0201006E
S3450001004011DE020019DE020021DE020029DE020031DE020039DE020041DE020049DE020051DE020059DE020061DE020069DE020071DE020079DE020081DE020089DE0200A9
S3450001008091DE020099DE0200A1DE0200A9DE0200B1DE0200B9DE0200C1DE0200C9DE0200D1DE0200D9DE0200E1DE0200E9DE0200F1DE0200F9DE020001DF020009DF020067
S345000100C011DF020019DF020021DF020029DF020031DF020039DF020041DF020049DF020051DF020059DF020061DF020069DF020071DF020079DF020081DF020089DF020019
S34500010100FDCC020091DF020099DF0200A1DF0200A9DF020019CF0200B1DF0200B9DF0200C1DF0200C9DF0200D1DF0200D9DF0200E1DF0200E9DF0200F1DF0200F9DF0200EF
S3450001014001E0020009E0020011E0020019E0020021E0020029E0020031E0020039E0020041E0020049E0020000000000012E010059E0020061E0020069E0020071E00200E6
S3450001018051E0020000000000643E030000000020D4010000643E03000000FF1F00000000643E0300000000140000000000020020507700000000FF1F0000000000000014D4
S345000101C00000000038B572B61DF06AFD0C4C0D4DAC4206D30C4DAC420AD362B621F014FEFEE7D4E90001A2680C3400F019F8EFE754F8080B54F8041C00F01BF8EBE700BF74
S3450001020088010100AC010100C4010100FEE7FEE7FEE7FEE7FEE7FEE7FEE7FEE7FEE7FEE710B50023934200D310BD1C585C500433F8E700231A468B4200D370471A500433B9
S34500010240F9E7FFFF2DE9F0414B688AB04FF000080133CDE9048805460E4617468DF80F8003D105200AB0BDE8F081002AF9D0946806210DF10F021EF01AFA317A002977D06D
S345000102807368082BEDD13368002BEAD05A88D88862809A88A280E0805A7862701B78237013F0600F16D10C2A60D8524B53F82260002E5BD005AB04AA21463846B04705ABE5
S345000102C0019304AB009302460023214628461EF023F8C7E703F0200248B31F0627D4BAB10121089006AA2846CDF81C808DF82410069400F0C3F8089B0593079B049300289C
S34500010300DDD10146E388049A28461EF062F9A9E75E062BD5002307930890012306AA132128468DF82430069400F0E8F8E3E77AB100230121089006AA284607938DF824109C
S34500010340069400F09BF8089B0593079B0493B6E759060BD507920123089006AA132128468DF82430069400F0C9F8ECE70520A6E79DF80F30032B09D162781E4B214653F8E8
S345000103802250384605AB04AAA8476BE77368002B3FF467AFE288002A3FF463AF94F9000022780028FFF65DAF12F0200011D0326807928DF8241006AA0121284606940893CB
S345000103C000F05CF8024605AB019304AB009301237BE752060BD5326807928DF8240006AA132128460694089300F088F8EAE70522E9E700BFE81F030030B5104B87B0CDE995
S3450001040003310F4B019303AA012301A90546ADF808301EF0ECF8044660B98DF8060003AA01A928461EF0E3F8044618B1802128461EF0FCF8204607B030BD00BF450201002D
S3450001044040008000054B19689A7B29B1824202BF0022C3E900229A73704700BFF8060020054A1368927B23B1824202D10B60002070470420704700BFF80600202DE9F04756
S345000104800F4615462AB1DFF86C80D8F80030984226D004241DE01B6809FB003083681B79012B19D0032B19D053B902230AEB031340689B682A4639469847052817D000B116
S345000104C0204601360446D8F804301A7AF0B28242E1D82046BDE8F0870023E7E70123E5E7DFF814A0002601244FF00C09EBE70446EFE700BFF80600201C2003002DE9F04175
S345000105000D4E3368984204460D46174611D1012907D13146FFF770FF324602212046FFF7ADFF73683A46294620465B68BDE8F04118470420BDE8F081F80600202DE9F84FAA
S3450001054006461746002A49D0002947D04B68002B44D0234D2B68AC7B9BB9224BA873C5E901132A46204900F043F8044680B982466B681B7A5FFA8AF8434510D82B683B605E
S3450001058003E0A0420CBF012402242046BDE8F88F28681EF007F83046FFF754FFF5E70C23DFF8489003FB08F84FF0000B6B68196841448B681A7999F80C309A4204D1D9F8BB
S345000105C000300A1D304698470BF1040BBBF10C0F09F11009EAD10AF1010AC9E70424D4E7F8060020F0060020FD0401001C200300F8B51746002A35D01B4D2B6895F8852034
S34500010600BBB9A96085F8850085F8843085F887302A461E4601330A2BC2E90366167502F10C02F7D101280AD92E6085F88560062403E090420CBF012402242046F8BD0B4BC8
S345000106406B603D606B68084A1B6811469847044620B105481DF0A6FF3E60EEE7022385F88630EAE70324E8E7080700204C2003002DE9F043037B87B004461BB9012007B0EF
S34500010680BDE8F0834268926851799942F6D31268002AF3D003F10053013B02EBC30612F833500C2700239D42E8DD706807FB03F28118825C032A39D10D7A00239D422BDCD5
S345000106C00026CB786373002ED8D00025DFF86080DFF86090A66001202F463379AB42CEDD0623B1688DF808706B43CA18CB5C8DF806305188ADF8041052788DF80720DB09BE
S345000107000CBF43464B46206803AA01A9CDE9033401351DF06CFFE0E748681A0100EB0316805CA27B9042CCD00133C7E70133BAE771E7020053E7020070B50A4C23680E46AF
S3450001074015465BB92146FFF78BFE30B923683BB1FF2366602073A3732C6070BD0220FCE70320FAE790070020F8B50E461746044618BB134D134B144AEA61FF2285F8C20071
S34500010780AB60012183F88020024628461EF0CBFA0E4BAA686B60C3F3072182F89C10C3F307411B0E82F8B010284682F8B4301EF04FF93D602E602046F8BD0624FBE700BF93
S345000107C0E407002000200740A4070020000200202DE9F04390F8943087B004461BB9012007B0BDE8F0834268926851799942F6D31268002AF3D003F10053013B02EBC30607
S3450001080012F833500C2700239D42E8D9706807FB03F28118825C082A2CD10D7A00239D421DD80027CB7884F89530002FD7D00026DFF88C80DFF88C90A760012035463B7967
S34500010840B34219D80123E560C4F88450C4F8883084F88C5084F88F5084F89650C0E748681A0100EB0317805C94F893209042D9D00133D4E70133C7E7B9688DF80850062304
S345000108807343CA18013610798DF80900CB5C8DF806305188ADF8041052788DF80720DA0915BF84F8913084F892304B464346206803AA01A9CDE903341DF099FEBFE700BF40
S345000108C09D0A010061090100F8B51E4C25680F461646002D34D11C4BA3611C4BE3611C4B23621C4BE3631C4B236421461B4B2365FFF7B6FD30B1C4E9005584F8945084F8FD
S345000109009350F8BD236833B9606084F8940084F893000320F5E7FF2384F89330236A84F894007022606167601A700A22DA7198701873587384F88D0084F88E003460E0E7DE
S345000109400220DEE7A80800209C0900208C090020780900207009002064090020400900207FB54B6814465A1C0D462BD194F88530A3B163681E688EB1A269D37B03F07F0316
S34500010980282B0BD100230968029101930093537B8DF80C306A4601212046B04794F89650012D0BD1002384F89630E26994F8911020680D231DF007FEA4F88E5001252846C4
S345000109C004B070BDE26893429CBFD21AE26094F88B20012A0CD1002394F89110206884F88B3084F8862084F885301DF03EFEE5E794F88520AAB90D2BE0D10B681968264BCF
S34500010A009942DBD1012584F88E2094F89210A269206884F888501F231DF0DBFD84F88D50CCE762681668002EC8D001930B68029323690093A3695A7B8DF80C20DB7B03F0EC
S34500010A407F03282B03D16A4601212046B047E368FBB1A3696A685B7B04EB031320469B6DB2FBF3F22369134423611EF05DFDE3680546002BA3D1002384F88530012384F8EF
S34500010A808E30E26994F8911020680D231DF09BFD95E70125EFE700BF555342537FB514464A68531C0E462BD194F88430A3B163681D688DB1A269D37B03F07F032A2B0BD108
S34500010AC000230968029101930093537B8DF80C306A4602212046A84794F88D3063B9B4F886304BB91F23A26994F8921020681DF070FD012384F88D300025284604B070BDD1
S34500010B00E3689A429CBF9B1AE360A369DB7B03F0BF03152B06D163681B681BB100220B212046984794F88C30012B0CD184F88730002394F89210206884F88430A4F88C3074
S34500010B401DF093FDD8E794F88420002A37D0736801933368029323690093A3695A7B8DF80C2062681568CDB1DB7B03F07F032A2B03D16A4602212046A847E5688DB1A369E9
S34500010B8072685B7B04EB031320469B6DB2FBF3F22369134423611EF004FD0546E368002BABD1002384F884300D23E26994F8911020681DF008FD012384F88E309DE794F8C3
S34500010BC08830002B00F02C8173681F2B40F02881A369A0491868884240F022815D7B0F2D00F21E81997B1F2900F21A8194F890000130854280F0148101390F2900F21081C2
S34500010C00E16984F88D209448E260086058688A60486084F8882093F90C009A68197B002816DB92B1012084F88400002084F88500DB7B032B4FEAD11117D1626284F8391062
S34500010C4020461EF0F3FD0546B0E084F88420ECE7002084F88400002AE7D094F88600012584F885500028E3D047E7206A00252F2B857005734573626284F839104CD8112B91
S34500010C8007D8002B63D0042B69D020461EF0A7FFD9E7123B1D2BF8D801A252F823F000BF3F0D01008B0C01008B0C01006F0D01008B0C01008B0C01008B0C01008B0C010030
S34500010CC0270D01008F0D01008B0C01007F0D0100570D01008B0C01008B0C01008B0C01008B0C0100770D01008B0C0100670D01008B0C01008B0C0100470D01008B0C010082
S34500010D00370D01008B0C01008B0C01008B0C01008B0C0100870D01009E2B24D007D8552B25D05A2BB1D120461EF03BFE8BE7A82B09D0AA2BA9D120461EF0E2FD83E720461D
S34500010D401EF095FD7FE720461EF0B5FD7BE720461EF0FCFD77E720461EF0DAFE73E720461EF0B7FE6FE720461EF06BFE6BE720461EF03BFE67E7204600F074F863E7204652
S34500010D801EF0E7FE5FE720461EF001FE5BE720461EF000FFA3691B7D05463BB92F4A937843F0010393702E4B19229A70236A9B7843B1E3691A7B2AB9A269D27B032A1CBFB4
S34500010DC001221A73052D0ED194F88430012B1AD194F887200AB984F88C30002384F88430022384F88F3094F88430002B7FF485AE94F88530002B7FF480AE94F88B30002B63
S34500010E007FF47BAED0E694F88530012BE8D194F886200AB984F88B30002384F88530DFE794F8921020681DF020FC94F8911020681DF01BFC002384F88D30012384F88F307A
S34500010E4040F20113A4F886304FF48073A4F8883052E600BF55534243555342537A730020E85D002070B5364B04461868A36986B05D7B8DF814500023CDE903336368009099
S34500010E801B681BB103AA11212046984794F89030AB423EBF236A05229A70049B38BF00252BB1039A1AB104EB0515C5E91523A36994F84C50D98A49BA89B2002D3DD06269FC
S34500010EC0002A0CBF032002205B7B053304EB0313002D5A689B6812BA0CBF0125022501920C2202EBC00243EA05631BBA8A424FEAC006029328BF0A468DF80360694600239D
S34500010F00206D11F8015BC5540133042BF8D101A9206D11F8015BC55401330C2BF8D1012384F83A30236DE3620023A26284F8383020461EF087FB06B070BD2846C4E700BFEF
S34500010F40542503002DE9F04F834D844CAB7843F0800387B0AB70237803900F46062B55D8DFE803F04B50504B667B04007C4EDFF85082727BB37B9A4240F08680AB78794E8E
S34500010F8013F0200F0CD0784B78491A68784813F0F1F8AB786FF34513AB70338801333380744B1A6B12060AD580221A636E4B72491A686F4813F0DEF83388013333806F4D92
S34500010FC06F4B704800242C7000941B882246214606F006F9338828700246BBB16A4B6948214606F0E3F828700094024633886548214606F0F5F8287008E0644A002313701E
S345000110005E4A1370039800210DF08EFF039B202B0BD15F4C237823B1554820F0D0F9002323705C4A13780133137007B0BDE8F08F594D4F482A8A01290CBF5849584913F03F
S3450001104099F82A8A57494A4813F094F82378013323704B4B00221A80D8E7AB78980644BF6FF34513AB70434B1A6B110644BF80221A633B4A062323700023537393733A4A57
S345000110801360384A1380C1E7707BDFF838E10130C0B2FA2828BF0020142404FB00FC08EB0C010CEB0E0A0EF1080E91F809B0DAF804A058F80C205EF80CC04B6891F80890D1
S345000110C070734FF0000E1BF0800F9AFA8AFA9CFA8CFC81F809E03FF44CAF012F09D0324951F8040F984204D0013C14F0FF04F7D13FE7B9F1080FCDE904ACCA4628BF4FF03C
S34500011100080A1BF0020F14BF284929491848CDF800A013F02FF8B9F1000F08D12549144813F028F8164A13880133138021E722490F48DFF83CB013F01DF820490DF110096F
S345000111400024013419F8012B5846E4B213F012F8A2451A49F5D8E1E77A730020927300205B730020544A0020D8090020C72503007018FF1F00400240D6250300E573002046
S34500011180265B002026740020122D0300E7740020EA71002089730020065B0020582503006D25030087250300B83F00209E250300AE250300CD2D0300BE250300C1250300B5
S345000111C0002100200821002073B5984C2378072B054639D90D2B23D9632B2FD1944C237823B1944820F0EBF800232370924C637A5A060AD5914E6FF386136372337823B16A
S345000112008F4820F0DCF800233370202D01BF8D4A137801331370E37843F02003E37048E0012202FA03F111F4A85F40F0D48011F4206F40F0DB800D2B00F02081652002B012
S34500011240BDE8704002F0FEBD013B062B05D8DFE803F00C4759898BA7BF00774B1A786FF382021A700123237023E0774A724D00231370764A137095F90430002B22DA2878CB
S3450001128010F004005AD1032105F0EAF998B1142013F00AFF6E4902466E4805F03DFF6E4B187005F079FB63232370EB7843F02003EB7002B070BD2B7843F004032B702378C4
S345000112C00133D0E7152013F0EFFE61490246614805F022FF604B187005F05EFB6323C2E7594B5E4A5A495B4800251D7005F032FF594B1870504B1A7865F341021A7005F099
S34500011300F5FFDCE74C4BDA7842F01002DA70544A127842B104232370202DCAD1494A137801331370C5E7022804D0012808D11B78980715D40121084605F092F9022392E791
S34500011340082801D00428E7D11A78C2F34001C94361F341021A7002B0BDE8704005F0C6BF042380E705237EE7374A3B4D00231370364A2B70137005F00FFB38492D480122CB
S345000113801FF054FC30B1374A3149324805F0C4FE2870A1E7264B01221A7005F0F3F98EE7244B1A69304B1A60274A00231370274A6220137013F078FE25490246254805F021
S345000113C0ABFE254B187005F0E7FA23780133237002F06CF873E70022002316481FF0FCFF224A00231380224A137068E7092B0CBF1046022004F06AFA024608B1207058E7B1
S345000114001C492378097800293FF45AAF03F0FD03092B7FF44EAF154B00901B880146164805F0DEFE0C4B187043E700BF92730020EA7100207018FF1F7A730020E87100208B
S34500011440D013FF1F89730020E7740020E573002067740020A774002066740020A5710020A4700020E4250300883F0020EC5A0020EC710020EB710020267400203A4E737A3A
S3450001148043F00103737202F067FA032004F01EFAB8B12070737A3548D906027829D5F178012D41F01001F17015D16FF30413632A73723FF6FEAEFF2303702D4B00221A7028
S345000114C0F7E62C4B2C4A1B7812781343E2D16A2002F0B8FCDEE7632A2DD8082D11D0042D29D1264951F82230002B3FF4E2AE013B10E0632A1FD8F378082D43F01003F3703C
S3450001150015D11E4951F8223040F2E63083423FF6D0AE0133164C41F82230002222701849184800929BB205F05BFE2070C1E6042DD7D0012DBFD0202D7FF4BBAE124B0025C2
S3450001154063201D7013F0B0FD10490246104805F0E3FD104B1870064B1D706323237002B0BDE8704002F0BEB97A730020826A0020E5730020EB710020887300200C0B00202D
S34500011580E673002026740020E774002067740020A7740020667400202DE9F74F874C2378102B054614D8013B0F2B1AD8DFE813F021005D006F0094009600B200C600C90080
S345000115C0D400E0002801E10120022F026E023A02632B00F0A182652003B0BDE8F04F02F031BC774B1A786FF382021A700123237023E0744A724D00231370734A137095F91B
S345000116000430002B23DA287810F004004FD1052105F026F8A0B1142013F046FD6B4902466B4805F079FD6B4B187005F0B5F963232370EB7843F02003EB7003B0BDE8F08F80
S345000116402B7843F004032B7023780133CFE7152013F02AFD5D4902465D4805F05DFD5D4B187005F099F96323C1E7564B5A4A5749574800251D7005F06DFD564B1870504BE7
S345000116801A7865F341021A7005F030FEDCE74C4BDA78022842F01002DA7004D0012808D11B789D0716D40121084604F0D9FF02239DE7082802D0042840F0B4811A78C2F32F
S345000116C04001C94361F341021A7003B0BDE8F04F05F00CBE04238AE7052388E7394A3D4D00231370384A2B70137005F055F93A493A4801221FF09AFA30B1394A3349344833
S3450001170005F00AFD2870ACE7364B01221A7005F039F899E72B4A002313702B4A6220137013F0C2FC29490246294805F0F5FC294B187005F031F923780133237004F0E4F9F2
S3450001174082E70022002325481FF046FE264A00231380264A137077E7012004F00FFB08B120706AE7224B1B78002B7FF466AF6BE72048214D002303701A46194655F8046BD8
S345000117800131013618BF0132C9B21CBFD2B201236429F3D103B10270037853B90A2013F083FC0A4902460A4805F0B6FC094B187059E7124A13700B2319E700BF9273002066
S345000117C07A730020E7740020E573002067740020A774002066740020A57100207018FF1FE4250300EA710020EC5A0020EC710020EB710020D05D00200C0B0020D15D00201E
S34500011800DFF8D492DFF80CA3DFF8C88299F80070002388F80030504619461A46D346DEB2B74257D809B188F800209C4A9C499D489D4F05F071FC002638700096024698F82F
S3450001184000309749974805F0CBFC984B944938700246944805F0AAFC38700096024699F800308F498F4805F0BBFC914B8C49387002468C4805F09AFC8E4B99F800101E70E5
S345000118808D4B38701E708D4E33788B42024636D28B49844851F823308149B3F5006F21D205F0B8FD337838701BF8033002462BB1844B7B497B4805F079FC3870082D14D078
S345000118C0042D12D0102D3FD13378002B39D0013B3370B2E610F8016B16B10132D2B2012101339CE705F008FEDCE733781BF803201AB100220BF803209FE60122FAE798F895
S345000119000030994218D1704B6549664805F04EFC082D387001D0042DD4D198F8003099F80000B3FA83F35B090022D1B28842C9D90AF8013B0132F8E70BB9644BE4E7644BAC
S34500011940E2E799F80030C3E7022D0AD1337899F800200133DBB29A423370BFF46EAE0023B6E7012D5ED198F80030002B3FF465AE6AE64A4A4A494B484B4F05F0CDFB0026E2
S34500011980544B3870009602461B784549454805F027FC464B424938700246424805F006FC4D4B3870009602461B783D493D484B4E05F016FCB37A3870024618074CBF484B72
S345000119C0484B3749374805F0F1FB082D387001D0042D08D1B37AC3F3C002C2F1010262F3C303B37229E6012D1CD1344B1B78BCE7002200233C481FF0EFFC3C4A002313803C
S34500011A003B4A13703B4AD3880133D3801CE6334FBB7A022043F00403BB7204F0AFF9064640B12070202D7FF408AE334A13780133137002E6314B1B7843B9BA7A2378110776
S34500011A404CBF03F1FF3301332370EBE72C4A14491448154C274F05F05FFB207000960246BB880F490F4805F0BBFB264B0C49207002460C4805F09AFB207000960246FB88C8
S34500011A800749084805F0ACFB2070CBE71E4A1F491F4805F041FB074B1870D5E5EA25030067740020A774002066740020762C03008C3C0300E7740020E5730020D15D0020B2
S34500011AC00C0B0020F0250300F3250300F8250300FE250300CF5D0020D05D00207A730020042603000D2603007018FF1FEC5A0020EC710020065B002089730020EB71002084
S34500011B0014260300173503001C260300E874002028750020836A0020104C237823B110481FF04DFC002323700E4C637A5A060AD50D4E6FF386136372337823B10B481FF0D4
S34500011B403EFC00233370202D01BF094A137801331370E37843F02003E3706EE5EA7100207018FF1F7A730020E8710020D013FF1F897300202DE9F04F994D2B788DB05BB972
S34500011B80984B4FF40062C3F88820BFF34F8FBFF36F8F0DB0BDE8F08F934CA078632800F2CB8092490B8AFA2B10D0B3F5FA7F0FD08F4A904E7D2B18BF32460023062824D8E3
S34500011BC0DFE800F00852606A858DA8008A4AF4E78A4AF2E78A4A53631363824B4FF40062C3F88820BFF34F8FBFF36F8F854AD36B43F01003D363844B1922DA72A37E012BAC
S34500011C0005D932230B82A3780133A37028E02B78092B11D17D4B9B78DF06F4D40B8A322B01D1FA23EEE7FA2B01D17D23EAE77D2BE7D14FF4FA73E5E7013B052B0ED801A243
S34500011C4052F823F02B1C0100231C01005D1C01005D1C0100031C0100331C010000230B8200236373A37394E7694B1A6842F000421A601B68DE02F3D50223A3706379013343
S34500011C806371EDE7624B5A604FF0A0421A601B68DD01E5D50323B8E75D4B5A601A6822F000521A600022114602F108000001195002F508700132102A43F82010F4D14FF4A4
S34500011CC080225A63202299649A6204239DE7504B504A1A604C4B1922DA72052395E74C4B494A1B6813F0006F03D0D37A002BB7D18BE73C4B302183F84B134FF40061996075
S34500011D003F4B4FF400715963A3780133A3703223D372A5E700224049134640F2E240053282424B724B6001F11401F8D13B4A13703B4A1370642368E7354B344D196A1962AA
S34500011D406A7AAB7802F0010203F0100313432E4AD27A13432A7B02F00102134302D10023A37016E74807FAD4A37E012B34D91F4A128A322A02BF224A4FF400711163052B97
S34500011D8021D1234BD3F8002112F0706F0DD0D3F8002102F07062B2F1006F06D0D3F8003103F07063B3F1106F0DD11E4B9A7952B9174A4FF00171C2F804114FF04061C2F8B5
S34500011DC0001164229A7195F90230002B60DAAB786FF3C713AB70DCE601F09EFEF3E700BF8A73002000E100E05B730020065B00200200890F0200921F0200890702008903F9
S34500011E000090044000800440E85D00207A730020004002400F000220780D0020D25D0020D35D0020035E0020AB785349667B43F01003AB700B88013342F20F729BB2013618
S34500011E40F6B2934288BF01230B80FA2E4B4B28BF0026142707FB0637BE46BEE80F000DF1080CACE80F00DEF80030CCF8003000238A46797A7B726B7A667313F001033A7AEF
S34500011E8002AE0AD0069B009396E80F0001F0DAFC627BA37B9A42C7D17BE6C907F8D5082AF6D8374A964692F809C01CF0010F18D05168514510D1142202FB03EE0FCE7746FA
S34500011EC00FC733683B609EF809300CF0400C4CEA030C8EF809C0DBE70133FA2B02F11402E1D10FCE07AF0FC7DFF89CB033683B609BF80070F92F20D007EB87080EEB880867
S34500011F003B46FBB9142207AE02FB03EC0FCEACE80F0033681B4ACCF80030002352F8041F8A4525D1142202FB03E35A7A42F040025A7201378BF80070AAE7AB7843F0400343
S34500011F40AB70A5E703F1FF3914225FFA89F902FB09E6A8F1140872689245D3D20FCE08F1140CACE80F003368CCF800304B46C8E70133142BD2D1DCE7265B0020002100205C
S34500011F80780D0020B83F0020D25D002030B5B0B10D4A142311464FF0FF3551F8044F84420DD004B90D60013B13F0FF03F5D152F8041F013104D1054A02EB8303586230BD24
S34500011FC00133142BF3D1FAE7B83F0020983F002010B5074A00234FF0FF3152F8044F01338442DBB208BF1160142BF6D110BD00BFB83F00202DE9F04FB74EB84C737AB84FB5
S345000120006FF300037372B37A87B06FF38203B37212F00CFFB34B1B780546002B40D0327A2378520638D5632B3AD897232370B378DB0644D5AC4A1378002B40D10123137099
S34500012040AA4A13704FF00008552087F8008013F02BF841460246A648DFF8D49205F05CF8A44B89F800001B7882462BB1DFF8C4B2BBF81030002B7CD15C2013F015F852463B
S34500012080034600219A4805F091F8FA2389F80000237004F053FC15E0632B01D86F23C5E72378002BC3D1914901220A7092493A700B70924922700B8091490B70B7E73B78D2
S345000120C0002BBFD12378012B72D1DFF8209299F80030002B40F03281B378DA0640F1A181884A8948DFF85092002105F015F84FF00008824B89F80000CDF8008002461B881A
S345000121008148414605F06CF8804B89F80000024641467D4805F04AF87D4B89F800001B79CDF8008003EB830303EB830302469B094146754805F054F8764B89F800000246D3
S345000121404146714805F032F8012DB37889F8000040F0638165222270674A82F800806E4A4FF0FF3168F345131160B37007B0BDE8F08FB378D8068CD5684B5D48524641461D
S3450001218005F014F889F80000CDF800800246BBF810305748414605F023F8614B89F8000002464146524805F001F889F8000070E75C4A00217D2B117055D8642B10D89A1E38
S345000121C0042A45D9202D40F0C785574B1B780F2BCCD1564B02221A7033786FF3000332E3653B182BEED801A252F823F001260100C5210100C5210100C5210100C5210100D6
S34500012200C5210100C5210100C5210100C5210100C5210100292901008329010091290100512A01009F290100C5210100C5210100C5210100C5210100C5210100BB290100AC
S34500012240492A01004D2A0100512A0100752A0100033B264A032B00F21F81DFE813F03E015B017801950103F16902D2B2162AA9D8973B162BA6D801A252F823F07D2A010090
S34500012280C72A0100D32A0100C5210100C5210100C5210100C5210100C5210100C5210100C5210100D72A0100272B0100312C0100C5210100E52C0100FF2C0100C521010017
S345000122C0C5210100C5210100C5210100092D0100492D0100552D01007A73002089730020CE5D0020A4700020CC5D0020CD5D0020A97500208A730020D35D0020265B00206A
S34500012300D15D00202426030026740020AD3D03005B73002041260300BC0900202226030027260300CB5D0020937300209473002068750020065B0020E5730020B378A14ADB
S34500012340DFF8B082DFF8B0A2002113F0100389F800101BD05D20117012F0A6FE9A4902469A4804F0D9FEB37888F800005906024606D5974B9449954804F018FF88F80000A1
S3450001238000238AF8003004F007FBA5E65E201370039312F089FE8C4902468C4804F0BCFE039B8AF80030DFF844A288F800009AF80030092B834604D15F2012F075FE0346A3
S345000123C008E0013B052B26D8DFE803F0211F25250323804B7C497D485A4604F0E7FE9AF8003088F8000023F00403013B012BCAD8794B1B78002BC6D00246784B724973484D
S3450001240004F0D4FE88F80000BDE7754BE2E7754BE0E7754BDEE75C20CFE768F34513B370D0E6082D01D0042D0CD1704B1A78F2B909221A70684A1378C3F1010313700123FB
S3450001244089F80030012D7FF4BDAE684B1B7823F00403013B012B3FF689AE5F4B1B78002B3FF484AE624B4FF400721A637EE6013A082A0FD8DFE802F00A0C0E0E080E0E0EE3
S34500012480050005221A70DAE70122FBE70222F9E70622F7E70022F5E71378ABB1494B4FF00008562083F8008082F8008012F0FCFD45490246454804F02FFE4E4B18704E4B2B
S345000124C083F8008004F068FA012D7FF47BAE6F2323704A4B00221A7048E61378ABB1394B4FF00008572083F8008082F8008012F0DBFD35490246354804F00EFE3D4B1870DB
S345000125003D4B83F8008004F047FA012D7FF45AAE7923DDE71378ABB12A4B4FF00008592083F8008082F8008012F0BEFD26490246264804F0F1FD2F4B18702F4B83F8008087
S3450001254004F02AFA012D7FF43DAEA123C0E71378ABB11C4B4FF000086C2083F8008082F8008012F0A1FD18490246184804F0D4FD204B1870204B83F8008004F00DFA012D3F
S345000125807FF420AEAB23A3E71378ABB10D4B4FF00008582083F8008082F8008012F084FD09490246094804F0B7FD124B1870124B83F8008004F0F0F9012D7FF403AE97234C
S345000125C086E700BFE774002067740020A77400202A2603002F260300CB5D00203D2603002E26030033260300382603008A7300200090044066740020E57300209273002002
S34500012600B37813F0100800F04F816FF34513B370AE4EDFF8E8823378DFF8FCA2142101FB038CDAF80020DCF80400904200F0B980DFF8E8E2CAF800008B465EF8042F90423F
S3450001264008BF9CF809200BF1FF3104BF42F040028CF8092011F0FF0BEFD1DFF8C4929C4889F800B001335A465946CDF800B004F0B7FD5946024689F8000095481DF033FBA2
S34500012680337889F80000142101FB03830246587A5B6810F0020F59468D4878D004F02CFF024689F8000059468A4B894804F07EFD337889F80000142101FB0383CDF800B092
S345000126C0024659461B7A8248DFF83092DFF850B204F086FD32788BF80000142101FB0292527A530608D59BF80020112A52D9784B1344042203F8012C04F020F93378142241
S3450001270002FB039999F80900DFF8E0C1DFF804921422534308EB030100F07F024A729CF80F2002F01F02803A8CF80F206A4A4FF0000882F80080694A89F80080C00782F85D
S34500012740008061D5664A98180832406800BA0490D3581BBA05930B7A002B4DD0082B28BF0823604903930DF1100B1BF8013B99F800205D4804F01EFE08F10108039B594913
S3450001278089F800005FFA88F84345EED80FE004F041FE85E74E4800211DF097FA8BF80000A1E79CF909209CF80900002AACDB4F4B4F48D97BDFF86C8111F0100116BF4D4AA9
S345000127C04D4A002104F0A8FC444B102D1870337821D198F80020CBB1013B33703178474B142202FB01335A7A62F07F025A7298F80030994226D2B9E4414A3A493A4804F0BD
S345000128008BFC89F80000D2E73E4AF6E7002AE5D0013A3270E2E7022D17D198F800000133DBB28342337024BF002333703178334B142202FB013388425A7A62F07F025A72A2
S345000128403FF694AC0023337090E4012D1DD12B4A142101FB0322506898B1537A83F04003590653720AD5FFF791FB4FF0FF333278CAF8003098F800309A42BBE7FFF7A8FBCE
S34500012880F3E798F800209A42DAE798F80020934201D300233370202D7FF468AC01232370194A3B70137061E43F2012F0FDFB17490246174804F030FC074B1870154B83F835
S345000128C00080064B83F80080E5E700BFD35D0020A9750020762C0300E7740020E5730020800D002067740020A7740020E85D002026740020773C0300BD310300780D002006
S34500012900442603004E260300CD5D0020E87400202875002066740020BC090020B83F002068750020D25D0020552012F0BDFB00210246AF48DFF8F09204F0EEFB804689F8DB
S345000129400000562012F0B0FB424603460021A84804F02CFC0021024689F80000A4481DF0C2F9A44A89F8000000231370A24A1370B378DA0602D52378013300E07223237054
S3450001298020E40121284607B0BDE8F04FFEF7DABA02239A4A237001233B70137012E4202D05D10223954A237001233B701370F37843F02003F370FFF7D9BB552012F074FBD4
S345000129C0002102468A48DFF8609204F0A5FB804689F80000572012F067FB424603460021834804F0E3FB0021024689F8000080481DF079F97F4A89F80000002313707E4A9E
S34500012A007F4813707F4A804992F800C003709E461A465FFA83F8C4450AD8BEF1000F01D080F800C012B1B378DB06A4D47C23A6E791F809E01EF0400F1CBF0132D2B2013324
S34500012A4014314FF0010EE4E702219BE70323A0E70A2012F029FB002102466C4804F05CFB644B6B4A187000231370634A137003F093FF80E7202D9AD1032393E7552012F06A
S34500012A8013FB002102465A48DFF89C9104F044FB804689F80000582012F006FB424603460021534804F082FB0021024689F800004F481DF018F94F4A89F8000000231370A0
S34500012AC04D4A137057E7284607B0BDE8F04FFEF77BBB06235DE7552012F0E6FA002102464348DFF8449104F017FB804689F80000592012F0D9FA4246034600213C4804F0DA
S34500012B0055FB0021024689F8000039481DF0EBF8384A89F8000000231370374A13703D4BFF221A7027E73C49142300224FF0FF3C51F8040F08BBC1F800C0013B13F0FF03C4
S34500012B40F6D1FAB1DFF8CC90DFF8E0A099F8002002F1804108310AEB8101132A14D90BB189F800205A2012F09FFA2C4902462C4804F0D2FA264B187079E701301CBF013218
S34500012B80D2B2DAE7A523FAE651F804CF501CBCF1FF3FC0B21CD00BB189F800205B2012F083FA1E49DFF8688002461D4804F0B4FA99F8003088F800000AEB830302465B6ABB
S34500012BC0B3F5805F07D30021154804F095FC06E002460123C1E71248002104F01BFC024688F800000F4B0E48002104F0DFFAC1E7A9750020E7740020E5730020CD5D002061
S34500012C00D35D0020D25D0020780D00202875002066740020D15D0020B83F002067740020A7740020E23A030068750020983F0020012D3FD152490B78132B1FD90023514896
S34500012C400B7015224FF0FF35013A12F0FF0211D10BB114230B704C4B0022597A013221F04001FA2A597203F11403F6D1A2232370FFF77CBA40F8045F0123E5E703F10802BB
S34500012C80424B03EB82034FF0FF325D685A603E4B002240F2E2405968A94208BF597A02F1050204BF21F040015972824203F11403F1D1DBE7102D0CD1314A13780133DBB2CB
S34500012CC0142B4FF0A20188BF002313702170FFF74DBA022DF0D0202D7FF448AA042323700123DDE53F2012F0DFF929490246294804F012FA284B1870237801332370202DE2
S34500012D007FF455AE04234DE6552012F0CDF9002102462248DFF8889004F0FEF9804689F800006C2012F0C0F94246034600211B4804F03CFA0021024689F8000017481CF070
S34500012D40D2FF89F8000016E6284607B0BDE8F04FFEF722BC05231CE6102D07D12378012B02D9013BDBB2BAE70623B8E7022D7FF4FDA92378052B01D80133F3E70123AEE75C
S34500012D80D15D0020B83F0020780D0020983F002067740020A774002066740020A975002068750020F0B51349134B144F1E780B78B34224BF00230B700D784FF0140C2B46FA
S34500012DC00CFB03705A1C90F909E0447ABEF1000FD2B206DA04F07F044472184613460B70F0BD96428CBF134600239D42E8D1FF20F5E700BFCA5D0020D25D0020780D002052
S34500012E00274B284AD3F800C02DE9F041264E274C274D284F42F20F7E136B9B0601D4BDE8F081738901339BB2734588BF00237381A37B617B0133DBB2FA2B28BF00239942E0
S34500012E4002BFA97841F02001A970A978880624D41421594347F801C0D2F88010D2F8840089024FF0140101FB03714BBF20F06040C0F38A404FF083084FF08108486081F8A5
S34500012E800980D2F88000C0F303400872D2F88800C860D2F88C000861A37320231363BBE7D809002000400240065B00205B7300207A730020002100202DE9F04F9F4BA04DB2
S34500012EC0A04CC9221A702A780026562A87B0267039D169780D2911D19B4B1B88022B0DD19A4B1A70582233205A7031229A70D8705A71322007221871227099712E78532E81
S34500012F0056D1AB780D2B0FD18F4A1288032A0BD16D7821788D484A1C322DD2B238D18C4D05262E7043542270237823B901232370864B07221A70874A537943F010035371E3
S34500012F4007B0BDE8F08F432AD8D16B780D2BD5D17D4B1B88022BD1D17D4B1E7000F0C2FC7D4B1E707D4B1E707D4B9E707D4B324640F2E24105368E425A725A6003F11403A7
S34500012F80F8D123785A1C2270704A0721D154B5E7342D02D16E4D0126C3E7352D02D16C4D0226BEE7362D40F02182694D0626B8E7582E0DD1AB780D2BB6D1634B1B88032B04
S34500012FC0B2D123785A1C2270604A0721D154ABE75A2E0FD16B78302BA6D1AA780D2AA3D1594B1B88032B9FD12378591C21705749CA5499E76D2E20D16B78462B94D1AB7805
S34500013000462B91D1EB78462B8ED12B79462B8BD16B79462B88D1AB79462B85D1EB79462B82D12B7A462B7FF47FAF6A7A0D2A7FF47BAF454B1B880A2BD5E74F2E40F0778119
S3450001304068780D287FF470AF3F4B1B88022B7FF46BAF3F4B22781D7825F004010139531C0129DBB2394903D9237007238B545BE7394E885435703A4D23700026AE7053E7AC
S3450001308003235BE1285C09F1020A0D285FFA8AFA08D1AAB981F800A023785A1C227007212A4AB0E0CDE900231CF0AAFD0F28DDE9002307F10107ECD800EB0B1B01224BE117
S345000130C0294B81F800A0C3F800B088F80090E3E788F80030009798469B465FFA88FA524509D8BBF1000F00F06A81204B81F8009083F800A063E115F8090009F101030D28EC
S34500013100DBB207D10B70BBF1000FC5D0174B83F800A0C1E7CDE902231CF072FD0F28DDE902230190EED8E85C09F102090D285FFA89F91DD181F80090E5E700BF897300206D
S34500013140DF72002093720020FA5A00209B720020E05D00207A7300208A730020DF5D00205B730020780D0020C0090020DC5D002002921CF045FD0F28029A08F10108D9D8F1
S34500013180019B00EB0310009B03F8010B4FF0010B0093A2E7BEF1000F02DA092D00F093803CF81380B8F1000F40F0918001B105708F4908688F4941F823008F49CA548F4A60
S345000131C0397802F8331002EBC30279785170B9789170F978D1703979117179795171B9799171F979D17101222CF81320844A134400229A712378834A7A21D154991C0133E5
S345000132002170DBB20D21D1540D2E7FF48DAE7E4B1B88012B7FF488AE7C4F3B78002B59D17B4F07F10809FFF7BDFDFF283FF47CAE14224243BD1894F800C095F80880697A3E
S345000132404646082E28BF082611F0020114BF0A23052303EB46035CFA83F33C2B3FF764AE6B68DFF8D0E102EB09056D6895FA85FA684DAD5872444FF0000E82F809E0664A89
S3450001328050730CF101022DBAD2B2CDE904A522705C4D81B3542105F80C102846714604F02BF9431C237006F130032B54B8F1000F28D123785A1C22700D22EA54574A1388A8
S345000132C001331380AFE70133DDB2012165E70133012182E021784B4D4A1C46206854D2B200212846227004F065F8431C237000232E543B7018E6742005F80C00284604F093
S3450001330089F8CEE7DFF8FCB00DF1100A4FF000081AF8013B22780021584604F04BF808F101085FFA88F846452070F1D8C1E7742E3FF4A6AE542E7FF467AF0823384A3949C6
S3450001334013700122DFF8E8800A70294A0027176088F80070BB463A465FFA87F909F101009945C0B2FFF48EAE2AB1214A0870C2F800B088F80090082B01BF1D4A136843F0D2
S34500013380004313600B7803F10109EB5C303BDAB25FFA89F9082A81F800903FF67DAE224F00233B707B70BB70FB703B717B71BB71FB71002A7FF48CAE082388F800300B78F6
S345000133C0EB5C0D2B7FF468AE18491948DFF868C091F909E0002303701946242BDDB27FF4D9AE00293FF458AE037055E6072399E5C0090020740A002099600020555F002091
S34500013400035E00209B720020FA5A0020DF5D0020780D0020880D00205B730020265B0020DE5D0020DD5D0020D45D00207A730020DC5D002000210020A44A0020154B9B78F0
S34500013440632B82BF144B4FF400721A63134A937899060BD51248017841F00801017011496FF345139370CB8B0133CB8393785A0641BF0B4A137843F0100313700A4A136BAB
S345000134801B0606D506490B7863F07F030B708023136370475B730020009004407A730020DF5D0020065B0020004002401D4B1E481E49002270B51A701D4B1E4D1A80192637
S345000134C0134606FB02F40132642A40F8043B01F8013B2B55F5D11849FF220A7017490B6017490A7017490A70174A1370174A1370174A1370174A1360174A1380174A517AA7
S3450001350021F050015172917A63F300019172144A1370144A1370144A1370144A1370144A137070BDE96A00200C0B0020836A0020F04A0020BE600020826A0020CC09002018
S345000135402F5E00202E5E0020D26E0020D36E002088730020B8400020EE4A00207A730020345E0020335E0020325E0020315E0020305E0020214B1B68D82B06D1B0F5005F55
S345000135802CBF002001204000704740F26A22934203D041F2F072934202D1B0F5804FEFE741F2642293420ED1A0F57043B3F5805F20D3A0F5FF00A0F5E040B0F5805F2CBF0D
S345000135C00020032070474AF64722934203D046F64762934207D1A0F58040B0F5304F34BF00200120704740F63912934204D1B0F5410FC5E70320704797207047B840002057
S3450001360070B5784C2378013B092B00F2E280DFE813F00A00350050006E008C009B00BD00E000E000CD00704A24230021013B13F0FF0322F8021BF9D16C496D4E422241206A
S34500013640C1E900206B490A603288002A00F0C38069486A4A816B6A4D11606A4A29881180694A1178694A1170694A12681DF0B4FE33882B802378013323700AE00021012085
S3450001368014F06AFC012812D0022804D0002840F09E80002070BD23780133DBB223705D4B1B78002B40F0938014F056FBF1E70A23F4E7594B1868FFF75DFF63280346E9D8F5
S345000136C008B10223D8E704222270544A544C107054480278FF25511C5607C9B203D1002BD7D00270D5E7A55401230A46F3E74E4B052119704B4B1A784C4B1A70002A66D025
S34500013700454A21701268DA70100C5870100A002298701A71344B01201880454B9A71454B1A80454B19225A74B3E7424B1B882BB1424B1B78AA2B50D1062323703E4B5B7C7D
S34500013740002BA6D19B20A5E7344D364B2A781B789342B6D9344B3A48314E082159700023D118C9B20133DBB2715C00F8011F082BF6D11D4B08322A7001225A802C4A002353
S34500013780D3712C4A138007232370CAE7294B1B882BB12A4B1B78222B21D106232370264B5B7C002B7FF475AF9D2073E7154B12481A88134B1A80114B00251A682B461DF05B
S345000137C00BFE124B25701A780F4B1A7061E7992060E79F205EE798205CE79A205AE79C2058E700BF88730020A44A0020740A0020EE4A0020E40900207018FF1FA00C0020B7
S34500013800EC5A0020EC4A0020EB710020E86A0020A40C0020EC710020843F0020E15D0020ED710020E571002099600020555F0020035E00205C4A0020E85D0020355E002009
S345000138405C5F002084B0F0B404AC84E80F00204B204C93F909300A460020002BC1B201DA09292BD054F8205095422AD11A4C1B4E34F810304FF6FF75AB421CBF013324F817
S345000138801030174C079D9DF81830235406EBC0042F0AE570A7702F0C2D0E06F830500898E071050AA571050C000E2071677065710894F0BC522004B007F02CBA0130C1B2B6
S345000138C0CEE701302428C8D1F0BC04B0704700BF7A730020E40900205C4A0020355E00207560002000231548154A10B519464FF0FF340133DBB2242B40F8044B22F8021B55
S34500013900F7D1104B5A7A61F3C7125A720E4B9B78632B09D90D4BD3F80021B2F1406F04BF4FF01062C3F80021094C237823B109481DF045FD0023237010BD00BFE40900201B
S34500013940A44A00207A7300205B73002000400240E77100208011FF1F082806D10B4A1378FF2B1CBF013313707047042801D1084AF5E7102801D1074AF1E7022801D1064A89
S34500013980EDE70128F0D1054AE9E700BF325E0020315E0020345E0020335E0020305E00204B4B93F90930002B2DE9F341494D80F28C802B7E3BB3012B40F08780464B5A6AC1
S345000139C0464B1B78934274D1454B46495A62464B46481C78464B5C720023DEB2B44202D90133092B60D143494B8A01334B82424B0093424B5B7A1021722007F08BF92B7EAD
S34500013A0001332B762AE03E4B5A8A3AB3DFF8048198F8006016BB01222A765E82304A2E4B56625A6A354B3749374F5B7A324C3B80FE20087088F8002010210094742007F0FD
S34500013A4069F998F80030022B0BD0032B06D0012B23D123882D4A5BBA9BB2136002B0BDE8F0812346294933F8482952BA92B20A603A88013A92B2032A0DD8254A93F84A105A
S34500013A80117093F84B10517093F84C1093F84D309170D370E2E73E80E0E7164B88F80060FF222E765A82D9E711F8016B00F8016F93E7144B1B78FF2BD0D10E494B820E4B23
S34500013AC0009328210023742097E7002399E700BF7A7300205B730020740A0020DC720020E40900209B720020DB7200207C5E0020756000205C4A00209D5F002099600020B4
S34500013B00A44A002094720020FA5A0020943F002022730020597300202DE9F74F5F4C94F90920637A002A03DAD80701D5FFF738FF627AA37A02F0010103F004030B43217BEE
S34500013B4001F001010B43564912D10888FF280FD04888FF280CD08888FF2809D0C888FF2806D00889FF2803D04989FF2940F08C80637ADFF840E14B484B49DFF824C14B4DA4
S34500013B8043F002036372002694F90930002B0EF1010A00F1010901F108080CF1020707DA092E05D1D64648464146BC460A26EBE7BCF800B0BBF1000F51D09EF80030002B79
S34500013BC04DD1D5F8003113F0706F0DD0D5F8003103F07063B3F1006F06D0D5F8003103F07063B3F1106F3AD14A780B78120402EB0362CB7813448A7803EB0223C5F80831F2
S34500013C004A790B79120402EB0362CB7913448A7903EB0223C5F80C31254B53F82620B2F5006F26D29304C5F8043103781B0403F4702303F14063BBF1FD0FC5F8003198BFD3
S34500013C400BF1FF3B4FF032038EF8003098BFACF800B0037800915420F1B207F05BF80136242ED64648464146BC468DD103B0BDE8F08F22F00043C5F8043103781B0403F4FC
S34500013C80702303F14263D6E79107EFD563F34102627203B0BDE8F04FFFF724BE7A730020A44A002099600020555F002000400240740A0020095E0020A0F1650310B53A2B0A
S34500013CC076D8DFE803F01E272A2D303336393C3F4245484B4E51575A75547575757575757575757575757575757575757575757575757575757575755D606366696C6F75A4
S34500013D007200304C304B22783049314803F04EFA207010BD2B4C2F4BF5E72A4C2E4BF2E7284C2E4BEFE7274C2D4BECE7254C2D4BE9E7244C2C4BE6E7224C2C4BE3E7214C50
S34500013D402B4BE0E71F4C2B4BDDE71E4C2A4BDAE71C4C2A4BD7E71B4C294BD4E7194C294BD1E7184C284BCEE7164C284BCBE7154C274BC8E7134C274BC5E7124C264BC2E76E
S34500013D80104C264BBFE70F4C254BBCE70D4C254BB9E70C4C244BB6E70A4C244BB3E7094C234BB0E7074C234BADE7064C224BAAE7C728AED9034CFF2822780CBF1F4B204BCA
S34500013DC0A2E700BF687500205326030069750020A97500205F2603006D2603007E2603008A2603009A260300A9260300B6260300C0260300CD260300D7260300DF260300EC
S34500013E00ED260300FE2603000A2703001927030027270300382703004A27030060270300732703008A270300A2270300B5270300C7270300DA270300EC270300FB270300EA
S34500013E40072803002DE9F3473A4C637A5B06054601D507F055F82379374E384A384939486FF382032371384B00241D70347003F053F92B463070024631493248009403F085
S34500013E80AFF9324B307002462D492E4803F08EF92F4B3070009402461B882949294803F09FF930702846FFF707FF02F047FD294B294D1C70294B2A4E1C702C700094337878
S34500013EC028492948224603F08BF9284B287002462449254803F06AF9337828701BBB02F05BFD234B63221A7002B0BDE8F08750232A7803FB0A933946404603F057F9337826
S34500013F002870013B9A450246B4BF1A4B1A4B3946404603F04BF90134287033785FFA84FA5345E4D8DBE7DFF854900E4FDFF83880F3E700BF7A730020687500200E2803001E
S34500013F4069750020A9750020EC710020D42C0300EC5A0020E774002066740020E5730020246F002067740020A77400201428030092730020F125030016280300256F0020D0
S34500013F802DE9F347DFF8B0C2A64EA74D0023337086F8503086F8A03086F8F0308CF80030DAB2A95C202927D0092925D053290BD1AB185978452907D19978542904D1DB7835
S34500013FC0202B04BF0432D2B2AB5C492B16D1AB1893F801E0AEF14603D3F1000E4EEB030E924B00211F788DF807100C46BA4208D30B2C3DD1662064E00133D1E74FF0000EBB
S34500014000EEE7AB5CA3F16100192815D8203BDBB20C2C00F2D180DFE814F0920039001D01CF00CF00CF00CF00CF00CF00CF00FB00FB00940000210A24002BD9D0272BD7D014
S345000140400C2C00F2B980DFE804F00A2CA0B7B7B7B7B7B7B74E4E0A0000210224ECE7202B01D0092B6BD10132D2B2974200F2C9806F496C481DF0C8FDF0B14223F3714F2313
S345000140803372542373720023B37215E09CF800300133DBB2042B8CF800300AD800210224A4E79CF800100131C9B204298CF800100BD9604B1B781BB9002002B0BDE8F087A9
S345000140C06920FFF7BFFE6320F7E7222B40F0B6809742CDD9AB5CA3F161011929AAD8203BDBB200210A2488464FF0500A4FF0000970E03D2B40F0AE80BEF1000F4FD19DF8BA
S34500014100070000F0FF0418BB002940F083809CF800004FF05008013808FB00F0013206EB0008D2B29742335488F80110A0D9AB5CA3F1610119294FF001013FF67DAF974224
S3450001414096D9AB5CA3F1610019289FD9012473E79CF80040481C013C4FF0500808FB0464C0B2635404F800E04F28A2D80132D2B297427FF67DAFAB5CA3F1610119294FF079
S3450001418002043CD8203BDBB20146202B01D0092BAFD19DF8070000F0FF0400283AD09CF800404FF05008013C08FB0464481CC0B2635400232354D7E7652082E797427FF6EA
S345000141C017AFAB5CA3F1610019283FF635AF203BDBB288469CF8000001310138C9B20AFB00604F2900F8083000F801903FF661AF0132222BD2B2E1D10134E4B2F6E60146ED
S345000142001AE7AB5CA3F16100192898D9002413E70B2468E797427FF62BAFAB5CA3F1610019288AE7256F0020ED710020EB71002018280300236F0020246F002097427FF6B2
S3450001424017AFAB5CA3F1610119293FF605AF203BDBB200219CF800404FF05008013C481C08FB0464C0B263544F284FF0000121543FF61FAF222B01BF9DF80730C3F10103E0
S34500014280DBB28DF8073071E7F8B5534953481DF0BBFC68B3524B1B78022B3BD06B20FFF7D1FD6320F8BD142101FB036138461DF0ABFC01350028F1D12078EBB29842F2D8E4
S345000142C000EB8000474A002106EB800002F024FF454A23781188454A22F81310444A916B444A42F823100133DBB2312B2370D5D841493A48394C1DF087FC00283ED004F157
S345000143004F01002211F8013F4BB10132502AF9D16720C4E7394C3A4E324F0025CCE7D2B2182AF5D894F85020562A3ED12C4A1278022A23D1334E192707FB03F29019B55C00
S3450001434095B10022D1B254FA82F5415C95F85050A94204D00133642BEED173209FE701320029EFD172209AE71E4A294602F0D4FE254A54FA85F393F8503053B923787B2B0B
S345000143801BD16378DBB9214A537A1C0711D56E2085E72B3BDBB2122B05D822FA03F3DE0701D577207BE70135E3E77720FFF74AFDE4E743F00803537201E07D2B01D0002071
S345000143C070E761780029FAD1104A537A1807DED561F3C303EFE700BF20280300256F0020246F0020756F0020EC5A0020F24A00207018FF1FAC0C002000350300E96A002049
S34500014400EA6A0020BE600020050004007A73002047292DE9F3410446154606D96720FFF711FD002002B0BDE8F081522343544B1CDBB25822C2548B1CDBB205F13002C254FA
S34500014440CA1CD2B23A26304F865457F825200B1D561CDBB20CD02D4E16F805C0BCF1000F06D0DFF8B0C03CF815C0BCF1000F04D1481D3F22E254C0B2D4E7B2F5805F37D202
S34500014480472BCBD84A1D6821C15457F82530D2B2002102F0BFFF2F2323540021421C0091735DD2B2204602F09BFE735D002BB9D03D222254431C0230DBB2C0B268224D28DC
S345000144C0E254ABD8124F4FF0000807EBC50717F8083002460021204602F06CFF08F101035FFA83F8735D43459CD34D28EFD995E7422B93D86822C2540531CAB257F8253004
S34500014500002102F0F9FFC6E7E409002075600020355E00205C4A0020F8B5164D00231926002206FB0354D1B2475C615CB94219D00133642BF4D10278562A0ED14278522AF7
S345000145400BD18278532A08D1C278322A05D10279332A02D14279322A09D07120FFF772FC632003E001320029DDD1D8B2F8BD1846FCE700BFBE6000202DE9F843914E0023CC
S3450001458033600C78025D562A0746884616D11BF063FB622810D88C4A98F80040125C22B96D20FFF74FFC632006E0884A52F82030336088F800400020BDE8F883303A092A5F
S345000145C04BD93B5D242B09D1A21CD2B20021541EE4B23B5D002B43D10029EAD13B5D542B07EB04055DD16B78582B40F0A380AA78A2F13003DBB2092B06D9A2F14103192B0D
S3450001460000F29880373AD3B2EA78432A3ED12A794F2A40F08F806A79552A40F08B80AA794E2A40F08780EA79542A40F08380684A32F813303360083461E0326805FB0233B9
S34500014640303B01343360E4B201223B5DA3F130010929F2D9002AB4D0ABE71A460A25F4E7A3F13000092808D8316803EB0113303B01323360D2B20121A9E7A3F1410005286A
S34500014680AAD8316803EB0113373BF1E7492A51D12A79442A4ED14F4A52F82330336005342DE0522B46D16B78582B43D1AA78A2F13003DBB2092B05D9A2F14103192B39D8F7
S345000146C0373AD3B2EA78432A0DD12A794F2A31D16A79552A2ED1AA794E2A2BD1EA79542A28D13D4AA4E7442A0BD12A794C2A0FD16A79432A1ED1394AD35C33600634E4B277
S3450001470057E7492A16D12A79442A13D1344AC3E7412A0FD16A79542A0CD1AA79412A09D1EA79303AD2B2072A04D82E4901EBC3039B5C7FE72C49052228461BF075FA40B173
S345000147402A4B1B8A33602A4B9B78632BA7D80023A4E728490B2228461BF066FA20B1244B9B7833601444CAE72349052228461BF05BFA10B1214B1B68F3E721490A222846ED
S345000147801BF052FA58B11F4B1B7833601E4B9B785B0602D54FF6FF7333600A34AFE71B49072228461BF040FA10B1194B1B88D8E718490C2228461BF037FA68B340F2295367
S345000147C0CFE700BF740D0020836A00200C0B0020A44A0020740A00205C4A002075600020E4090020355E00206A340300065B00205B7300202628030032280300C809002082
S3450001480038280300D25D00207A73002043280300265B00204B2803001D49062228461BF003FA80B3A5185FFA85F957FA85F51949022228461BF0F8F910B1174B1B78F9E612
S345000148401649042228461BF0EFF910B1144B1B78A2E7144928461BF0E7F908B1124BF6E71249052228461BF0DFF920B1104B1B7833600B3443E70F4928461BF0D5F908B180
S345000148800D4BF4E74C46A4F13800C0B289E600BF5828030002290300325E00204A3C0300315E002016290300345E002021290300335E00202D290300305E0020F0B585B053
S345000148C00023334D334E8DF80F3004469DF80F30E05CF8B12B2803D101338DF80F30F5E7522819D1E218517858293DD1D17800293AD19278303AD2B2092A35D8244F254880
S34500014900397803338DF80F30FFF782FD38700028DCD1632005B0F0BD222825D1002007462A784F2A02D90028D7D1CFE7591CC9B2605C222806D102338DF80F30154B00217E
S345000149409954C3E760B1531CDBB2502BB0542B70F7544FF0010005D16720FFF773FAD8E76620FAE70B46DBE70DF10F012046FFF703FE01460028CDD12A784A2AECD8064B4B
S3450001498000901B88304602F02BFC28709EE700BFD26E0020D36E0020740D00202DE9F34700230DF1070107468DF80730FFF7E4FDB8B9DFF86891DFF86881D9F80040DFF8AE
S345000149C064A106469DF80730F85C10B9C9F8004007E0022EC8F8004006D1FF20FFF732FA632002B0BDE8F087FD5C5A1CD2B22B2D8DF807201BD02F2D0DD8242D12D9A5F1A0
S34500014A0025020A2A0ED8DFE802F012120D0D0D120D0D120D12003E2D23D006D83C2D28D03D2D35D0373BD8B2D8E77C2DFAD10DF107013846FFF7A0FD0028D2D1D9F80030AF
S34500014A40CAF800302F2D44D8242D27D8023DD8F800400136042D3ED8DFE805F042464B505500BA5C3D2A15D102338DF807300425DDE7BA5C3E2A04D102338DF807300225C8
S34500014A80D5E73D2A08D102338DF807300625CEE70125CCE70325CAE70525C8E7253D0A2D36D8DFE805F00F143535350A063508350C001C4486E7E41A84E75C4382E7B4FBF7
S34500014AC0F3F47FE7B4FBF3F203FB12447AE71C4078E71C4376E7E31A5C425C41F6B271E7E41A18BF0124F9E79C4294BF00240124F4E79C4234BF00240124EFE79C422CBF82
S34500014B0000240124EAE79C428CBF00240124E5E79DF807003838C0B260E700BF740D0020080B0020040B00202DE9F04105460F463C483D4990461E461DF066F810B9002010
S34500014B40BDE8F0813948FFF729FF394B01221A700028F5D1A7F13004E4B2092C05D9A7F14103192B5AD8373FFCB208F1FF32032A56D8DFE802F002354014542D07D1032E1C
S34500014B80DDD12C4B1A682C4B43F82420D7E7522D46D1032ED3D1274B1A68284BF4E7542D14D1032ECBD1234B1A68254B23F81420244B234400229A71234B1B6BB3F5007FE6
S34500014BC0BDD07820FFF73EF96320B9E7522D27D1032EB4D1174B1A681C4B23F81420AEE7032EACD1134B1B68082B19D8542D17D1174A1355A3E7174BDB79303BDBB2072B8E
S34500014C000ED8032E9BD10B4A1168FF2908D8542D06D1114A02EBC402D15490E77420D1E76F20CFE7756F0020883B0300C56F0020BD600020740D0020740A0020E4090020DA
S34500014C40A44A0020035E0020009004405C4A002099600020256F0020555F00202DE9F043032893B0064634D18C4C637A5F070BD41D0729D58A498B481CF0C6FFE0B1637A5A
S34500014C806FF3C303637217E086490A786FF382037B2A6372DBB20DD1497803F0080281B922B16E20FFF7CEF8632406E043F008036372DFE71807DDD40124204613B0BDE8BE
S34500014CC0F083002AF8D0D5E7774B1A88774BC3F89021744D2B787B2B03D16B781BB90024EBE77D2BF9D072496E481CF08DFF044638B3704B1B78022B01D06B20D2E76E4F73
S34500014D00DFF8F881DFF8F09100253B78ECB2A342F3D9142101FB048148461CF075FF01350028F2D0032EDAD1644B654853F8242000231CF051FB634B33F81420624B1A8023
S34500014D40CDE7624957481CF05FFF00282DD0594B1B78022BD1D1584FDFF8A081DFF898913B78E5B2AB42C8D9142101FB058148461CF04AFF01340028F2D0032EAFD1544A1A
S34500014D8013880BB170208DE74F4C4D4821881180504A816B1160494A52F825201CF01CFB484B33F81530238099E74B493D481CF02BFF0446002892D148493A481CF024FF5F
S34500014DC078B1032E8BD1424D2B88002BDAD03E4A3B4813803F4B1A6823461CF0FDFA2C807DE73F492F481CF00FFF00287FF477AFDFF8C09099F80030012B40F2B2813949E4
S34500014E0028481CF001FF3849C8B126481CF0FCFE074600283AD000274FF002083349214809221AF001FF00286AD06B7A2B2B03D1AB7A002B08BF01274FF0050864E01948D7
S34500014E401CF0E2FE07460028E5D12B784D2B20D1274914480A221AF0E7FE2649044611481AF0E2FE80466CB100280CBF4FF003084FF00408AB7A2B2BD0D1EF7AB7FA87F706
S34500014E807F09CBE738B14FF00408F3E74FF00108C4E78046C2E70746C0E700BF7A7300205F280300256F0020FC5A00200C0B002061280300246F0020E96A0020AC0C00200C
S34500014EC07018FF1FF24A0020EC5A002066280300F04A0020A80C0020202803006B28030000350300722803005A2603008D2803007728030082280300756F0020EA6A0020CC
S34500014F00B8F1000F00F02D81AF4AB04800231370AF4A1370FFF7D2FC8146002868D195F8A030F3B995F8F03033B1AA48FFF7C6FC044600287FF4C1AE032E7FF4D0AEA64B6A
S34500014F400422B8F1030F1A7018D1A44C87B1A04B2278A349A34802F029F9207001F0EEFCBDE6A148FFF7AAFC04460028DAD0A4E6974A9B499B4802F0CFF8EEE7B8F1040F13
S34500014F8016D19A4A9A4C002313709A4A13704FB18F4B22789849994802F008F9207001F0FBFC9CE68A4A9449944802F0B5F8F5E7B8F1050F14D08D4A8F4990480023137033
S34500014FC08C4A1370824A02F0A7F8894B187001F0E3FCB8F1020F7FF467AEFEF783FC63E6874B1B7833B97620FEF72CFF4FF063094C4662E6834C2178002940F0A880824A88
S34500015000824D02A802F0A6F80246034695F87400002870D07E49897AC9076CD4B5F800E002F1480342F20F766B44B6454FF02E0103F8401C73464FF47A7128BF3346B3FBA4
S34500015040F1F1C1EB811C01EB8C1C01EB4C0C03EBCC030DF1480802F1010C58FA8CFC30310CF8401C9BB26421B3FBF1FC5FFA8CF1C1EB412801EB8808C1EBC80103EB8103C5
S3450001508002F1020812A951FA88F80CF1300108F8401CD11C0DF1480858FA81F19BB24FF00A0CB3FBFCFC0CF1300801F8408C5FFA8CFC511D0DF14808043258FA82F2CCEB4B
S345000150C04C38CCEB880C03EB4C03303302F8403C0EF10102A0F1410392B2C9B2B24288BF0022192B9CBF01F148036B442A8098BF03F8440C0B4603F148026A442E2102F874
S34500015100401C5A1C12A951FA82F24C2102F8401C9A1C12A951FA82F24F2102F8401CDA1C12A951FA82F2472102F8401C043312AA52FA83F3002203F8402C3648322202A97A
S345000151401BF074FD08B175204EE70123237017B91F4A314901E01E4A30492E480FF00AF846E799F80030012B40F09E802C492D481CF04AFD074638B1032E7FF4B0AD2A4B35
S345000151804FF400721A63AAE5284926481CF03CFD044628B1032E7FF4A2AD234B1F639EE5234920481CF030FD002872D0032E7FF496AD174A937A43F001039372104B1B7884
S345000151C0C3BB76206EE500BFD26E0020756F0020D36E002015700020BD6000206875002069750020A9750020C56F0020E774002066740020E573002067740020A77400202B
S3450001520094730020E7710020A5710020983F00207A7300208011FF1F052E0300642B030097280300256F002000900440A0280300AA2803009F4B1B78002B7FF43EAD9E4A3F
S34500015240214602A801F086FF00F148036B442E2203F8402C12AA431C52FA83F34C2203F8402C12AA831C52FA83F34F2203F8402C12AAC31C52FA83F3472203F8402C0430F6
S3450001528012AB53FA80F000F8404C02A81CF0ABFA13E58A498A481CF0B7FC28B1894A537A43F0800353721AE599F80030022B40F09581854982481CF0A7FC8449D0B18048AE
S345000152C01CF0A2FC00282DD08148FFF767FB814B032204461A7000287FF4EFAC7E4B1A68002A2FD01860774A537A23F00C0343F00403D7E772481CF087FC0028E4D1774942
S345000153006F481CF081FC002836D0754970481CF07BFCD0B1032E7FF4E2AC6A4A537A43F01003BFE76A48FFF739FB6A4B03221A70044600287FF4C1AC674B1B68002B7FF47A
S34500015340CEACD0E701221A60C9E46148FFF726FB604B01221A70044600287FF4AEAC032E7FF4BDAC5C4B1A685E4B1A605E4AFF2313705E4A1370B2E42B78572B42D16B78D2
S34500015380412B3FD1AB78492B3CD1EB78542B26D12B79522B23D16B79582B20D1EB79F3B9AB79514D514A2B70FF272F2B177014D9303BDBB2232B2B700FD84548FFF7EEFA51
S345000153C0444B01221A70044600287FF476AC032E16D1414B1A68434BB5E7742062E4EB78542B0FD12B79542B0CD16B79582B09D1EB793BB9AB793D4D3B4A2B70FF27D4E72F
S345000154002F706CE43A492E481CF0FEFB48B395F85030562B7FF463AC2D48FFF77DF8622804463FF64AAC032E7FF459AC314C324D324920700026324631482E701AF045FCDE
S345000154402178304B2870009633F821302B4902462B4801F0C5FE23782B4A28700121D1543DE42A4916481CF0CFFB044600285BD01748FFF793FA174A0123044613700028D4
S345000154807FF41BAC032E7FF42AAC214A1370124B1A68204B1A60204B1870174B187060200FF002FE1D4902461D4801F035FE1D4B187074E5E7710020A5710020B528030015
S345000154C0256F00207A730020C3280300C6280300756F0020BD600020740D0020CC2803002D290300CC0900202F5E00202E5E0020D1280300826A0020E5730020E67300208C
S34500015500267400200C0B0020836A0020D628030088730020B8400020E774002067740020A774002066740020984999481CF06CFB78B1984998481CF067FBF0B1032E08D14F
S34500015540964B4FF0FF320134E4B2142C43F8042FF9D193498E481CF057FB00283ED091498D481CF051FBC0B1032E7FF4B8AB8E4B002283F87420FFF7E2BB8748FFF70EFA61
S34500015580044600287FF499AB032E7FF4A8AB874B1868FCF7FBFCFFF7A2BB95F85030A3F14102192A07D895F8512022B97E4A82F87430FFF794BB7848FFF7F0F9044600281A
S345000155C07FF47BAB032E7FF48AAB784A764B12681A80402283F87420FFF781BB99F80020032A40F099802878542801D0522817D16B78582B5BD1A978A1F13003092B03D9FA
S34500015600A1F14103192B52D8EB78492B04D12B79442B05D1012236E0442B24D0432B38D0562844D15A48FEF777FF6228074604463FF643AB5E4958481CF0E6FA002836D033
S345000156405C48FFF7ABF95C4A01231370044600287FF433AB554A1168584A42F82710584AD355FFF72ABB2B794C2B04D16B79432BD6D1022207E0412BD2D16B79542BCFD1FF
S34500015680AB79412BCCD1334613B0BDE8F043FFF74BBA2B794F2BC3D16B79552BC0D1AB794E2BBDD1EB79542BBAD10422EBE7454937481CF0A9FA90B33D4937481CF0A4FAC1
S345000156C068B33C48FFF76AF93B4A01231370044600287FF4F2AA032E7FF401AB334A1268322A15D07D2A05D0FA2A13D0B2F5FA7F12D10623344A1370344B00229A70344B9C
S3450001570023F8022B0134E4B2242CF9D1FFF7E7BA0523EFE70223EDE76C20FFF7C3BA2D491B481CF071FAA0B121491B481CF06CFA78B12048FFF732F91F4B01221A700446B5
S3450001574000287FF4BAAA194B1A68234B1A60FFF7B4BA22490E481CF057FA002842D014490D481CF051FA00283CD01248FFF716F9114B01221A70044600287FF49EAA0B4B71
S345000157801A68174B1A80FFF798BA00BFDF280300256F0020EB280300756F0020B83F0020F1280300A2280300983F0020740D0020883B0300C56F0020BD6000200C0B00205F
S345000157C0836A00206A3403008A7300205B730020A44A002032280300C809002043280300265B00202B784B2B96D16B78452B93D1AB78592B90D1EB78502B8DD12B79412BF3
S345000158008AD16B79442B87D1204921481CF0FCF9002881D01F48FFF7C1F81F4B01221A70044600287FF449AA1C491D481CF0ECF918B11C4B1A681C4B1A701C4918481CF0DB
S34500015840E3F918B1174B1A68194B1A70194914481CF0DAF918B1134B1A68174B1A7017490F481CF0D1F918B10E4B1A68144B1A7014490B481CF0C8F900283FF430AA094B58
S345000158801A68114B1A70FFF72ABA00BF883B0300756F0020C56F0020BD600020FC280300256F0020740D0020325E002005290300315E002010290300345E00201B29030044
S345000158C0335E002027290300305E00206E4B1A682DE9F0410646A2B16C4A1278232A05D86B4931F812200AB100221A60694A117823291FD8684830F81110D9B91960FF2359
S345000159001370664C637ADA0617D4654A1278632A13D9644F3A8822B9634923F00C030A706372624B1B7863B1FDF76AFE28B1FEF789FA17E01B68002BE3D000252846BDE8D3
S34500015940F0815B4A137012F015F95A4B1B78002BF3D0554D2B78012BEFD8FEF711FB18B16328E4D86325E9E7DFF8988198F80030002BE2D0504951481CF046F9002863D04B
S3450001598098F80030022B5DD14D494E481CF03CF928B12B78002B55D101232B70CDE74A4948481CF031F9002831D02B78002B49D10127032E2F70C0D1444B1B78A3B9444A19
S345000159C01370444A612013700FF06EFB42490246424801F0A1FB424B187000F0DDFF637A43F010036372A8E7637A43F0400363723C4C2378002BA0D13B493C480A221BF0AB
S34500015A0015F9002899D13A4B2770186095E739492C481CF0F9F8A8B12A78637A012A03F0080302D073B16E2081E702222A70324A39881180314A916B314A1160002B3FF482
S34500015A407CAFF0E7682072E72B78012B7FF475AF012E03D1BDE8F041FEF716BCB31E012B3FF66BAF3046FFF7F9F8012805463FF464AF637A5B0602D5002005F09BF9012DE7
S34500015A807FF65BAF5AE700BFCC0900202F5E00205C4A00202E5E0020A44A00207A730020826A0020EC5A0020236F002088730020BD600020EB7100203B310300256F002016
S34500015AC033290300756F00203929030094730020E7740020E573002067740020A774002066740020E871002048290300D013FF1FD809002052290300EE4A00207018FF1F22
S34500015B00A40C0020246F002000230B480B4910B51A464FF0FF340133DBB2642B40F8044B01F8012BF7D1064B997A62F3C3019972044B9A80DA8010BD0C0B0020836A00205A
S34500015B407A730020065B00201E4B1A796FF382022DE9F3411A711C4B1C4F18708046FEF7ABF800F0EBFE1A4B1A4E1B4C1B4A00251D701B4B2570394630461D7001F0CCFAC9
S34500015B8043462070024639460095304601F028FB394602462070134B304601F007FB124B2070009502461B883946304601F018FB207000F0F1FE0D4B63221A7002B0BDE82E
S34500015BC0F08100BF7A730020EC71002067740020E7740020A7740020667400200E280300E5730020D42C0300EC5A0020927300202DE9F84F2F4A304F304CDFF8C8B092F850
S34500015C00008000233B7087F8503087F8A03087F8F030237019469E4618461A4699464FF0500A904502D9264DAE5C26B903B121700020BDE8F88F272EF8D0012809D0022830
S34500015C400DD0202E01D0092E2CD10132D2B20020E7E70131C9B2042926D9217019E0A6F12C05EDB2142D04D84BFA05F515F00105EBD04D1E0EF1010C5FFA8CFC0AFB057585
S34500015C80BCF14F0F05F80E6005F80C9006D9002BE3D1AC20FFF758FF6320CAE70132D2B2E646BEE70120BCE703464FF0000E0220B7E700BFEB710020256F0020246F00207F
S34500015CC0ED710020F6FFEFFFF8B52B4900230022C1E900230378682B2FD10225002212E0A4F13006F3B2092B18D8D1E90032120142EA13721B019B1942EBE6720135C1E947
S34500015D000032EDB201226B1EDBB2C45C002CE7D17ABBAD20FFF718FF6320F8BDA4F14103052BF5D8D1E90032120142EA1372373C1B011B1942EBE472E0E7303B092BE8D815
S34500015D4000252B460A270BE0D1E90036A3FB07349B1807FB064444EBE272C1E900320123EAB20135825C303AD4B2092CECD9002BCFD00020D1E700BF000400202DE9F341B6
S34500015D80994E338804465BB9984A1360984A1360984A517A63F38611974B5172FF22DA75964A97499748984D01F0B6F9002328700093024633889249924801F011FA934B7F
S34500015DC0287002468E498F4801F0F0F9022C287054D1DFF81CC2DCF80030002B4ED0834A1268934273D8DFF888E2834FBEF8000098B1FC7D002C6AD16E200FF055F9844946
S34500015E000246844801F088F9834B2C701870834B1C7000F0C1FD63205AE0814B4FF400721A63804BCCF800001A687F4B1A607F4B1A787F4B1A707F4BD3E900217E4B4FEA72
S34500015E40116883F800804FEA114883F80180D9704FEA1128110E1971110C5971110A9971DA7183F802800123744AAEF80030744B9871938801339380FF23FB7511F07AFE74
S34500015E80704B1B781BB3FFF7B3FE08BB3388012B52D16D4B1B78022B57D16C496C480C2219F0C2FE002850D06A48FFF70DFF78B9504B9B78DB0601D4022C0CD15F4B198A62
S34500015EC0654BD3E90023002B08BF914225D1002002B0BDE8F081012C1FD15F4AD2E90032A3F13201114303D15C4B05221A70EEE7A3F17D01114302D1584B0122F6E7A3F12A
S34500015F00FA01114302D1554B0222EFE7A3F5FA73134302D1514B0622E8E76D200FF0C4F83B4902463B4801F0F7F83B4B3B4A187000232B7013706CE7022B08D1484944481C
S34500015F40082219F071FE0028C1D1AE2048E03E4B1B78042BF9D13F48FFF7B6FE0028B7D13D4E304D33683F482B60FFF7ADFE0028AED1D6E90032092B72F1000280F09A80C1
S34500015F80DFF8A880384888F80030FFF79DFE00289ED1D6E90023274F98F80010C7E90023072911D908B1C7E90023012C62D12F4A29680023144652F8040B884287D0013080
S34500015FC00AD144F8231082E71B02013143EA1263C9B212020120E3E70133642BEBD1AF20FFF7B2FD17E700BFEC5A0020D8090020E00900207A730020E85D0020252603009C
S34500016000E874002028750020E77400205629030067740020A774002066740020E573002000900440DC090020740A00202D5E00209960002008040020555F0020065B0020BF
S34500016040035E0020EB710020246F002059290300256F0020756F0020000400208A73002066290300C56F0020157000200C0B0020A44A0020022C7FF468AF0F48FFF724FEF4
S3450001608000287FF425AF33680C4A29680C4C012B38BF012313600B4B53F8045B8D4203D1255C002D7FF413AF01306428F4D1002313600CE7AD200BE7256F0020E0090020C9
S345000160C0836A00200C0B00202DE9F0411A4D1422294600234FF0FF3451F8040F00BB0C60013A12F0FF02F7D1C3B1144B9B78DA061BD5134F134EDFF85480142455F8042F08
S34500016100531C07D0B2F5805F34BF4146394630460EF030F8013C14F0FF04EFD1BDE8F08101301CBF0133DBB2DAE7BDE8F041064904480EF01FB800BFB83F00207A73002026
S34500016140772903007018FF1F7F2903006F2903002DE9F04F364B9B78DB0685B060D5354F14223946002351F8040F013018BF013302F1FF3218BFDBB212F0FF02F3D1002BE7
S345000161804ED0DFF8D090142409F1080B57F804AFBAF1FF3F40D00021884632E014235A43254B13445868824529D193F90900597A002838DA01F07F0159721E7A1F492048E0
S345000161C002EB09035B681BBA02935BF802301BBA03930DF0CFFF8EB1082E1A4928BF082602AB0025013513F8012B15480193EDB20DF0C0FFAE421349019BF3D8012108F171
S345000162000108114B1B785FFA88F29342C6D819B90E490B480DF0AEFF013C14F0FF04B5D105B0BDE8F08F0A4905480DF0A3FFE5E77A730020B83F0020780D0020BE25030096
S345000162407018FF1FC1250300D25D00208C29030089290300800D00200A4B987810F010000ED0094A1423002052F8041F013118BF013003F1FF3318BFC0B213F0FF03F3D143
S34500016280704700BF7A730020B83F0020F0B50F4B0F4D104F1C7838260023D8B2844210D800200DE0002106FB035CCAB21CF802E03A4492F87520724505D10131002AF4D1EB
S345000162C0F0BD3F2BEED90133E7E700BF957300208C340020983F0020F0B50F4B0F4D104F1C7838260023D8B2844210D800200DE0002106FB035CCAB21CF802E03A4492F8EA
S34500016300B520724505D10131002AF4D1F0BD3F2BEED90133E7E700BF957300208C340020983F002030B5034600254C5DE8B234B91C70074B1A7964F382021A7103E0824234
S3450001634002D800221A7030BD03F8014B0135ECE77A7300202DE9F04F954B964F964900248FB0054695483C701C701BF040F9002840F07381924EDFF84482914940461BF012
S3450001638083F988B18D481BF076F997F800C0BCF1000F00F05E81DFF82C920CF1FF3A4FF0380800239E464DE1B37E002BEAD02E2BE3D0347B14F01004DFD1DFF8209219F846
S345000163C0013CDBB9002CD8D097F800907D4C7E49C9EBC900322204EBC000FFF7A3FF382303FB09443289738903EB0243636309F10103DBB2312B3B70BFD9C3E72E2B29D1AD
S34500016400012D4AD199F80030522B09D199F80130452B1FD199F80230432B08BF012419E0722B07D199F80130652B13D199F80230632BF2E7482B07D199F80130452B09D190
S3450001644099F80230582BE8E7682B06D0532B14D0732B0AD009F10109B1E799F80130652BF8D199F80230782BD7E799F80130312B0DD199F80230392BCFE799F80130312BEB
S34500016480F7D0522BE6D199F80230452BC5E7722BE0D199F80230652BBFE7022D4FD199F80030502B07D199F80130472BD2D199F80230542BB1E7702B07D199F80130672BD9
S345000164C0C8D199F80230742BA7E7542B26D199F80130582BBED199F80230542BBAD13B4939481BF091FB728B45F251539A4203D1F269374B9A421BD0B0FA80F46409354924
S3450001650031481BF081FB344900282F4818BF00241BF07AFB002818BF00249BE7742B99D199F80130782B95D199F80230742BD5E7328C44F24F739A42DED10024DFE7032DCB
S3450001654005D0052D1CD0062D28D0042D65E799F80030432B08D199F80130412B7FF47AAF99F802304E2B58E7632B7FF473AF99F80130612B7FF46EAF99F802306E2B4CE79C
S3450001658099F80030432B7FF465AF99F80130532B7FF460AF99F80230562B3EE799F80030432B7FF457AF99F80130522BF0E700BF9673002095730020F225030030050020B6
S345000165C0100400208C3400202A0400208F29030049434B4C9C290300AC2903002B04002008FB049B04FB08844C44DBF83410626B914225D25F460FCF6E460FC60FCF0FC63B
S345000166000FCF0FC697E80300254686E803000FCDABE80F000FCDABE80F000FCDABE80F0095E8030087E803006F460FCF0FC40FCF0FC40FCF0FC496E8030085E803000123F9
S345000166400EF1010E5FFA8EF45445C9DB002B7FF4A8AE60460FB0BDE8F08FA446F9E700BF38B50C4648B90846FFF774FE20B3012C134D1AD1FFF70AFE2870114D114B2A78B4
S345000166801B789A4224BF00222A702C78A34215D90D4B0E48C4EBC401322203EBC1010134FFF740FE2C70002038BD032C01D0052CE3D1FFF711FEDFE70120F5E70220F3E765
S345000166C096730020957300208C340020A57100202DE9F84F1F4BDFF894801F4F1F492048002588F800501D707D631AF080FF044670BB1C4EDFF868904FF0380A1949484632
S345000167001AF0C2FFF0B9B37EE3B12E2BF6D0337BDB06F3D498F80000338975890AFB007B05EB0345DBF83430AB42E7D2C0EBC0000D49322207EBC000FFF7F4FD0124CBF82F
S345000167403450DBE706481AF096FF2046BDE8F88F2C46FAE7967300208C340020F225030030050020100400202A04002095730020024903484022FFF7D5BD00BFA571002063
S345000167800D400020024903484022FFF7CBBD00BFA57100204D400020064B93F8FA302A2B06D1054B1868054B002808BF1846704702487047983F002088340020C0432158A7
S345000167C02DE9F047514B52481B78524CE4B0694632AE00220D46D7B2BB4237D84E494F4A09784F481944C9B28B4239D14D4B4E4A1B784E480B44DBB28B423ED14C4B4D4F76
S345000168001878DFF834C10022884288BF1A706A541A78002402F0FE0223464FF02008A85C1E46002865D010F0800F54D094BB13F0010469D03F484FF0200E013300F806E0F4
S34500016840DBB2112BEBD964B0BDE8F08710F8017B01F8017B14F8017B06F8017B0132BAE712F8014BEC5403F5C8746C4410F8016B04F8C86C0133DBB2B6E712F8014B6C54F3
S3450001688001F5C8746C4410F8016B04F8C86C0131C9B2B1E7DFF89C90DFF89CE009F8030002F5C87068445E1C10F8C80C0EF80300501CC0B2F6B215F800A009F806A000F5A3
S345000168C0C8706844023310F8C80C0EF806000232DBB2D2B2B5E7F85402F5C8706844013210F8C80C0CF803000133DBB2D2B20024A7E707F803800CF80300132903F10103BE
S34500016900DBB228BF00229CE7012488E7E774002028750020E874002066740020A774002067740020E573002026740020E6730020E2730020BB730020977300200F4B0020AD
S3450001694030B518730E4B0F4D18700F4B02221A700E4BFF221A702B78122B09D90C492024CC549A1C0133D2B2DBB22A70CC548854084B1A796FF300021A7130BDE85D002024
S34500016980E473002068750020E3730020E0730020A97500207A730020164B1748002230B55A73164B164D1A70164B007802211970154BFF21197015492B7809781944014494
S345000169C012290DDD591C1248C9B22024C4544454D91C0233C9B2DBB22970C454425401220C4B997962F304111A7999716FF341021A7130BDE85D0020E5730020E2730020B2
S34500016A0066740020E1730020DF730020E7740020A77400207A730020364B997A4A1E072A65D8DFE802F00415263444445361382292FAA2F23049120E0A70304A0021117031
S34500016A402F4A0121117002229A722E4B1A8070470C2292FAA2F22849120E0A70274A00211170274A0121117003229A72254B0222ECE7062292FAA2F21F49120E0A701F4A2E
S34500016A80002111701E4A012111700422EDE7012191FAA1F21848120E0270184A00201070174A117005229A72164B1022CEE73C2292FAA2F21048120E0270104A0020107035
S34500016AC001200F4A014410709972CFE7382292FAA2F20949120E0A70084A00211170084A012111700822C0E764229A7270470022FBE700BF5B730020EB750020E975002077
S34500016B00EA7500205A4A0020AB4A118889B22DE9F84F002956D1A94CA37AC92B00F084801AD8642BA648A74DA74E4DD005D80BB3013B122B27D9002323E0652B50D0C82B49
S34500016B40F9D1E172902393FAA3F31B0E037001232B703170C92341E0991DC9B20429EAD8FB3B032B00F28480DFE813F0540280006902800003702B7033704FF4FA73138019
S34500016B800123A37201E0FFF747FF8D4A8E4B11781B788E4C8B4801EB032189B2C4F8801019F088F803786BB172B6037801EB03239BB2C4F8803019F07DF80023C4F88010ED
S34500016BC0037062B6BDE8F88FE172802393FAA3F31B0E037001232B7031706523A37219E0E37A112B19D87A49C95C01707949C95C29B179490978CF0744BF20210170017841
S34500016C0091FAA1F1090E017004213170012129700B44E37202231380B7E7704A137943F001031371C823ACE7E37A112B19D86C496348C95C01706B49C95C29B16A49097847
S34500016C40C90744BF20210170017891FAA1F1090E01705D49042008705A49012008700344D7E75E4A137943F002031371FA2388E75A4BDB7A1F0700F1BA81DFF880B19BF884
S34500016C800C30002B40F0C980584B544D1878AB7857491E070A7866D5AB7913F0040362D1824288BF0B700A78494EDFF828C1DFF85091002302F0FE021F464FF0200A4D4D7F
S34500016CC015F802E09846BEF1000F3FD01EF0800F30D09FB913F0010743D0013306F808A0DBB2112BEBD9444A1378002B40F08A800A78122888BF531C0B7085E006F803E0C8
S34500016D0002F1010819F802E00CF803E05FFA88F803F1010E374D5FFA8EFE15F8085019F8088006F80E50023302320CF80E80DBB2D2B2D6E719F802700CF8037006F803E033
S34500016D4001320133DBB2D2B20027CAE706F803A00CF803E0132803F10103DBB228BF0022BFE70127ABE7824284BF00230B700B78184F174EDFF87CC0DFF8848012224FF0B6
S34500016D80200E1CF80390B9F1000F0ED086F8009018F803900133DBB2013A12F0FF0207F8019B06F10106ECD19DE7132886F800E028BF0023F0E700BF5A4A00205B730020EB
S34500016DC0EB750020EA750020E975002000F00F40CD730020A9730020E07300207A730020BB73002097730020DF73002068750020E4730020A9750020E3730020E85D00203D
S34500016E0069750020013B1370954A137801331370237B8BF80C306423A3729BF80D30002B40F0C6808F4A93781D071ED5937958071BD4FFF7C5FC8C4A1378002B00F0A28059
S34500016E40013B1370894A137801331370237B8BF80D306423A3729BF81030002B40F0AC80A372FF238BF81030A6E0814B814A1E78814B82491B7892F800E00F788048DFF87C
S34500016E800482F218122A2CDD774506D900270F7074498A7967F304128A717949DFF80892DFF808C2774F8E4600225FFA82FAB24553D3C3F11203744F744EDAB250FA83F071
S34500016EC058FA83F3112A52D9714B1B78002BB2D012232322013B13F0FF0301F8012BF9D1A9E7C2F112027745D2B208D95D4DAF794FF0000C6CF3041781F800C0AF71002A25
S34500016F00CBD0097806EB080A06EB000C0027614D15F80190FDB2754513D2B9F1000F10D05D4D8CF8009015F801900131C9B201370AF8019B5FFA87F94A450CF1010CE6D8C5
S34500016F40ABE772454FF0200538BF00218CF800502CBF4FF000098946E9E719F801AB0EF801AB1CF801AB07F801AB01329DE717F801CB00F801CB013216F801CB03F801CB9B
S34500016F80D2B29FE73D493B480A78007801320A70374A12780244384800780244122A3FF751AF0B702F498A7963F304128A7149E7A37A642B3FF44FAF2A4A9378190702D52F
S34500016FC093795B0713D5A37AFA2B10D12A4B2C491B782C4E2C4D2D48C3F11203DAB251FA83F156FA83F3112A09D9C823A3722B4A002313702A4A13702A4A1370C5E515F875
S34500017000016B01F8016B013210F8016B03F8016BD2B2E8E7E17E91FAA1F320481B0E0370204B002018701E4B0120814218704FF00203138004BF10231380FC23A1E5237F06
S3450001704093FAA3F315491B0E0B70164B04211970134B0121197002231380FE2391E500BFE07300207A730020E1730020DF730020E774002066740020E5730020E2730020F6
S34500017080BB7300209773002026740020E673002087730020A774002067740020EB750020EA750020E975002028750020E8740020104A11480023F0B59372104A104F13804C
S345000170C0104E114D114C124A1946013317F801CB06F801CBDBB214F801CB05F8011B122B00F801CB02F8011BEFD10A4B4FF45E721A81F0BD5B730020BB7300205A4A0020D7
S34500017100E8290300CD730020A9730020D629030097730020FC5A002030B50D4D0446002012F8013B33B90A4A2370117963F38201117130BD04F8013B21B12B79C3F380037B
S3450001714001F8013B3F289CBF431CD8B2E8E700BF7A73002070B5134600251E4613F8014B7CB9114E013A034612F8014F6CB90E4A00241C701179181A64F382011171C0B206
S3450001718070BD2E2C08BF3546E7E72E2C01D19542EDD003F8014B0029E6D03479C4F3800401F8014BE0E700BF7A73002030B50B4D0446104613F8012B22542AB9074B19793A
S345000171C062F38201197130BD19B12A79C2F380020A543F289CBF421CD0B2EBE77A7300202DE9F04F3F4C89B084460E462068616801AD03C5218929800DF1100E04F10A0545
S345000172001A3428686968774603C70835A542BE46F7D19DF84850DFF8D09005F00705072D0CBF03F00F0E4FF0000E10460EF1200211BF71461B09012100250DEB020E0DF1F1
S345000172400E080024052295420DD14FF02E070CF8007026B199F80470C7F3800737543F289CBF0130C0B2013A38F802ADD2B20027534507F1010B20D25FFA87FA54FA87F703
S34500017280FCB2954204BF0134E4B26CB102291BD00AF1300A0CF800A026B199F80470C7F3800737540130C0B2002ACCD101290DD102211EF8103C0D46C1E7A3EB0A039BB226
S345000172C05F46D5E70021BEE7002AFBD100210CF80010054B1A7961F382021A7109B0BDE8F08F00BF602103007A73002038B50D4A0D490E480E4DFFF70FFF0E4B28701B78EF
S345000173009B0704464CBF09200A200DF0CDFE2246034605490548FFF749FF2870BDE83840FFF73ABBB8380300E673002026740020E57300207A73002070B51D4624238354B9
S34500017340044621B11A4B1B79C3F380038B543F2A98BF01324FEA151098BFD2B218F0D1FCA0542846A61818F0CCFC61B93F2A07D80132D2B2A054402A1CBF0132D2B200E0FF
S345000173803070104670BD0A4B1D793F2AC5F380058D5405D930701B79C3F380038B54F0E70132D2B2A0541B79C3F380038B54E2E77A73002070B50446861818091D4618F06A
S345000173C0A0FCA054284618F09CFC61B93F2A07D80132D2B2A054402A1CBF0132D2B200E03070104670BD0A4B1D793F2AC5F380058D5405D930701B79C3F380038B54F0E769
S345000174000132D2B2A0541B79C3F380038B54E2E77A730020F8B50E4F0646C3F30B050324C5F3072018F06DFCB05419B13B79C3F380038B543F2A98BF013204F1FF3498BF79
S34500017440D2B214F0FF044FEA0515E9D11046F8BD7A730020F8B51C4624238354054621B10F4B1B79C3F380038B5401320C4FD2B20426200B18F045FCA85419B13B79C3F325
S3450001748080038B543F2A98BF013206F1FF3698BFD2B2240116F0FF06A4B2EAD11046F8BD7A730020F8B51E4624238354054621B1104B1B79C3F380038B5401320D4FD2B2AA
S345000174C00624C6F3075018F01CFCA85419B13B79C3F380038B543F2A98BF013204F1FF3498BFD2B214F0FF044FEA0616E9D11046F8BD00BF7A730020F8B50D4F06461D46FE
S345000175000824280F18F0FDFBB05419B13B79C3F380038B543F2A98BF013204F1FF3498BFD2B214F0FF044FEA0515EAD11046F8BD7A730020632BF8B5064628BF63230A2006
S34500017540B3FBF0F0C0EB4014C0EB840403EB4403DFB22023B354B51818F0D3FB49BB3F2A1FD8541CE4B23055402C50D1384618F0C8FB06F1400586F84000002958D02D4B09
S345000175801B79C3F3800301F1400081F84030224625232B70274B1B79C3F3800303701046F8BD2870384618F0ACFB287025232B70F5E7204B1C793F2AC4F380048C541ED93D
S345000175C028701B79C3F380038B54384618F099FB2870184C23793F2AC3F380038B5401EB0200D5D80132D2B22523B3542379C3F380038B54402A1CBF0132D2B2CFE7541C96
S34500017600E4B230551B79C3F380030B55ACE73846651C18F076FBEAB256FA85F5B0540029D7D1402AC2D00234E2B22523B354E1E72246BBE77A730020134B144A73B5187055
S34500017640134B1449144D00261E70144B044614481E70FFF761FD0F4928700246009610482346FFF7BDFD032C0246287005D10D4B08490B48FFF79AFD2870FFF78DF90A4B36
S3450001768000221A7002B070BD99720020B9290300E77400206774002066740020E5730020A7740020C42903005973002070B50E4D014600244FF6FF704AF20106A3B2994217
S345000176C000D870BD15F8013B0822584000F00103400813B180EA060398B2013A92B2002AF4D10134EAE700BFDF72002038B5074D2C782046FFF7DAFF054BA21C1855013448
S34500017700E4B2000A18552A7038BD00BFDD720020DF7200201148C37913F00103F0B51BD10F4F104E012540F6D86CC3F3CC0203F00701BC5C05FA01F124EA0104BC54B45CC3
S34500017740013324EA01016345B154EED143796FF341034371044B1D70F0BD00BF7A73002083E8FF1FA8E6FF1F177100200023044A19460133DBB23C2B02F8011BF9D170477B
S34500017780667000202DE9F843234B1B78012B04460D4606D0214BDA796FF30002DA71FFF7B9FFA4F51C53103B3B2B05D81B4B5879C0F34000BDE8F883204618F0ABFA40F696
S345000177C0D7639842044624D8144BDFF854C05979DFF85080012001F0010100228646D3B2AB42E7D2A318DE1003F0070339B11CF806700EFA03F947EA09070CF8067018F84F
S34500017800066046FA03F313F0010F08BF00200132E5E70320CEE700BF177100207A730020A8E6FF1F83E8FF1F38B504460D46FFF7A9FF58B9A4F51C520D4B103A3B2A197853
S3450001784005D819B903221A700A4B187038BD094A39B901211970084B10701C60074B1D80F4E71278052A84BF18700420EEE700BF5973002094720020943F0020FA5A002013
S34500017880F8B50E4B1D78012D05D118F043FA40F6D76398420FD9F8BD8318DF1003F00703F45D05FA03F324EA0303F3550132D3B29942F1D8EFE7024E0022F8E717710020A2
S345000178C083E8FF1F08B518F025FA054AC0F3CF0300F00700D35C43FA00F000F0010008BDA8E6FF1FF0B54FF6FF7642F20F7701B9F0BD0E4C00231A46A44634F8025BB542C4
S345000179000DD0854208BF013203F1010308BFD2B21E2BF2D101390130C9B280B2E7E7002AF8D1B84298BF2CF81300F3E75C4B0020054A00234FF6FF710133DBB21E2B22F806
S34500017940021BF9D1704700BF5C4B002008B50D4B00221A700C4B1A700C4B197962F3C3011971597962F304115971D97962F30001D971FFF7CFFEFFF7DBFFBDE80840FFF740
S34500017980F5BE00BF59730020947200207A730020392816D006D813281DD0262816D0104B187070473E2806D06028F8D10D4B01221A70382203E00B4B00221A7030225A7027
S345000179C0EDE7084B00221A703422F8E7054B00221A704E22F3E7034B00221A709C22EEE72173002000B006402DE9F74FA74C237B5E0706D4A64B1B88322BA64B50D964223E
S34500017A009A76E37A5D0740F1A480A34FFB78002B40F05484DFF8A882A04E98F800503370022D40F2EE862846FFF740FE002840F0E886032D3DD19A4B1A78032A40F0E18659
S34500017A40452199705A21D9704D21197141215971582199710521D971292119722179C9095972E1798C0622D411F0400F08BF00229A728C4A917ED27B1A730E2232700022CF
S34500017A805A730C22D9725A70FFF730FE864A002388F80030D37843F08003D37000F0C1BE9B7E002BADD16020FFF772FFA9E70222DEE7062D40F0A286794B1A78012A40F0D7
S34500017AC0A086B3F801104EF60302914235D1DA78042A32D15A70754A357092F8F610997092F8F710D97092F8F81092F8F92019715A71C9E76A4B1A78022A40F08286B3F8C7
S34500017B0001104EF60302914217D1DA78042A14D1664A197982F8F610597982F8F710997982F8F810D97982F8F91003221A7001213270002259709A70A6E7594B1A7862F0C9
S34500017B407F021A7001225A7002229A70032333709AE72379564D13F0080200F07A82207B4D494E4A032340070B711278CB7817D5DAB91BBB4F4B1B78FF2B40F05986484B89
S34500017B801B78013B022B00F253864B4A13780133DBB2042B137040F24B866020FFF7F8FE3E4B1B78002B00F03F86CB78002B00F0448603E0013B1370FA23CB702B783549B6
S34500017BC0FF2B05D18B7D632B9EBF3A4B00221A70E3790A7A03F00103134340F06F83374B1B78002B00F06A832E4B324A987F042800F2EF85DFE810F0CB05C605DC05E00528
S34500017C00E2050133DBB2142B2B7000F21F8696F800A02B4BBAF1FF0F187870D1294A204910700023284A3370DEB2864261D3637943F01003637160B1244AD38901339BB284
S34500017C4042F20F718B4288BF0023D3811A4B00221A7063795A06B1D41D4B1A781D4B1A70ACE7012B04D100232B70392000F0F9BD022B04D100232B70262000F0F2BD032BDC
S34500017C802AD100232B70132000F0EBBD7A730020FC5A0020E85D0020035E0020DD720020DF7200205B73002000B00640983F002094720020597300201F730020947300202A
S34500017CC0DE720020937200209B720020065B00209A720020957200206020FFF759FE0B780133DBB2052B40F2C08500230B702B708DE711F8016B02F8016B013394E7BA4EF0
S34500017D0096F80090002800F0998194F80580B74B18F0400F187005D1B54B1A78B54B1A70B54B187003280AD849F0080986F80090032002F0ABFFAD4A0023137089E7FFF759
S34500017D40B5FC28B149F0100986F800900420F0E7DFF89CB2E3799BF9002043F01003002AE3719BF800300BDAA44B9BF801201A7049F02009FF2386F800902B700220D8E73B
S34500017D809A4540F02B81B9F1000F40F027819C499C4A0193FF2088759B49137009689B4A1FFA81FA504682F8009017F0B3FF019B082B064636D09BF801200192934A484678
S34500017DC0CC460BF1020B019F5FFA80FE774542D8BCF1000F01D082F80090012B22D192F800E06423B1FBF3F398B200EB800202EB8202F244AAEB820A854A052812781FFABD
S34500017E008AFA68D140F2252399426CD8814B5879504538BF83F805A0012A03D140F6D7639E422CD9774B1B78022B6FD0032B40F0A3807649784A0E78704900239372D8B294
S34500017E40864200F29380637943F0020363716C4B19221A7270E0B9F13F0F0AD8674F1BF800E007F809E009F1010C5FFA8CF94FF0010C0130A7E740F6D7639E4235D8674811
S34500017E80DFF87891DFF8A0A1DFF8A4B108F00103304400220193D3B29E4526D919F801CB00F801CB93194FEAE30C012703F007031AF80C8007FA03F3DBB2019F43EA080871
S34500017EC00AF80C802FB11BF80C8043EA08030BF80C300132DFE74F489BB210F803C0D44538BF00F803A0012AC5D0B1F57A7F99D1BEF1040F96D14149494A0B885BBA538218
S34500017F004B885BBA93820EF0BDFC8BE7404B1A78012A11D140F6D7639E420DD8414BDFF8FC80DFF810914049B3F800C00023D8B2604503F1010E08D33C4B00221A7063792B
S34500017F4062F3861363710120F3E6331819F8000008F80300D81003F0070311F800A002FA03F343EA0A030B547346E0E711F8010B02F8010B013362E7082BDDD1244B93F8D3
S34500017F800090B9F1010FD7D1DFF8AC80184EDFF898A01E214FF6FF7B38F8020B5845CBD017F0B8FE40F6D76398421C4A0FD896F801C002F800C0C0F3CF0C00F007001AF8E9
S34500017FC00CE009FA00F040EA0E000AF80C00013911F0FF0106F10106DED1ADE749F0400986F800900520A4E69A720020DD720020DF72002097720020967200209B72002010
S34500018000E85D0020DC720020943F0020DB7200201771002066700020DB700020DA4B0020065B0020FA5A002083E8FF1F59730020A8E6FF1F227300205C4B0020AE4B69F0D4
S345000180407F090122FF2086F800905A7002F01EFEFFE5AA4E96F800A0BAF1000F00F037832878FF2800F033836179A54FDFF8B482032311F040013B7108BFA24B88F800202B
S3450001808008BF1960BAF1380F5ED8BAF1320F0AD8BAF1080F40D9AAF10902D2B2172A0ED90023337008E1AAF13403042B00F2FC81DFE813F06A0201022B026A028E020123B1
S345000180C093404DF2B502134240F05C8142F20822134240F0888213F4400FE1D0DFF834E285489EF8003000F803A0874A03F1010C12685FFA8CFC4FEA122900F80C9003F116
S34500018100030C8EF800C00233DBB2C254002940F040817C4B1A603CE10AF1FF33072BBFD801A050F823F000BFE18301002784010075830100E7850100A1800100A180010027
S34500018140A180010001860100BAF1630F00F04882BAF1FF0FA4D16D486D4A8389DFF8C891C82151760133644942F20F729BB2934288BF002391F800C08381237BBCF1030F25
S3450001818003F0010220D191F801C0BCF1FF0F03D0BAB1FAF791FE8BE089784129F8D1B9F800100329F4D162B1A27A6FF300036FF3C7122373A272DB074FF000028281C281DB
S345000181C0E7D499F80030CDE0BCF1560F16D191F801E0BEF10D0F38D1B9F800100229D7D1002AD6D1A17A828143F0010362F3C71142812373A17203F00102C9E7002A60D1C4
S34500018200BCF1630FB9F80030DBD191F801B0BBF1000FD6D1042BD4D13E4F3F4B02223A703E4A83F800C012785A70FFF75FFA3C4B3A781A70637986F800B043F010036371E9
S34500018240A9F800B085F800A038E0BEF1520F9FD191F802A0BAF1530F9AD1C8780D2897D1B9F80010042993D12B4981F800C04FF0330C312781F804C04FF0320CCF7081F82A
S3450001828005C08F7181F801E081F802A0C8716179234F4FF0080C41F0100187F800C0617132B16FF300032373A37A6FF3C713A37200233370A9F80030FF232B7003B0BDE85A
S345000182C0F08FBCF1580F7FF464AF4878B9F8002030282BD188780D2839D1032A37D10E4A0F4982F800C050706279022742F010020F706271D5E700BFDF72002059730020E9
S34500018300035E0020903F0020943F0020065B0020E85D0020DD7200209B7200202173002093720020E25D0020FA5A002031280ED18B780D2B0BD1032A09D1B64A01211170AC
S34500018340B54A1370637943F010036371B0E7531E9BB2A9F800300022D0B2984202F1010C03D3DBB2AD4A137015E00A1852780A546246F1E7A94A1378591C1170A84A0321B4
S34500018380D15406E0A54A1378591C1170A44A02F803A0FFF7ABF902F03FFCA24B00221A70A14AD37843F08003D370237943F0080323716423FB709A4B1B78082B40F07781EE
S345000183C0FA23FB70637913F040037FF4F7AB974A31781170964A1370964A1370FFF7EEBBDFF838928E4A99F800300120D0549248D0F800C0581CC0B24FEA1C2E02F800E023
S3450001840003F1020E5FFA8EFED81C02F80EC0C0B211B98A49C1F800C0894904330988115489F80030B5E7864BB3F800C0BCF1000F37D0DFF8E8917A4899F800304FF0020E9B
S3450001844000F803E0DFF8F0E1DEF800A003F1010E5FFA8EFE4FEA1A2B00F80EB003F1020B5FFA8BFB03F1030E00F80BA05FFA8EFE11B97249C1F800A0043300F80EC0DFF8C1
S34500018480C4A1DBB2964601321946D2B21AF80EE000F801E001339445DBB2F3D889F8003077E70023337009E75C4A1378591C11705B4A332164E7DFF86491594899F8003035
S345000184C03522C2545C4A03F1010C12685FFA8CFC4FEA122E00F80CE003F1020E5FFA8EFE03F1030C00F80E205FFA8CFC09B953490A605349098800F80C10591D0433DBB273
S34500018500120CC25489F8001043E74D4BB3F800E0BEF1000FC5D0DFF80491DFF804C199F8003036200CF803004348D0F800A0581CC0B24FEA1A2B0CF800B003F1020B5FFA44
S345000185408BFBD81C0CF80BA0C0B211B93B49C1F800A00CF800E0581D0433DBB24FEA1A410CF80310DFF8DCA0C0B2114601320346D2B21AF801100CF8031001309645C0B216
S34500018580F3D889F8000004E7DFF890C0DFF890E09CF800300EF803A0581C294BDFF8A4A0B3F80090C0B28CF80000002183184A45DBB205D300293FF4ECAE8CF80030E8E646
S345000185C0511C1AF802200EF80320CAB20121EDE7DFF848E012489EF800303822C25484E500287FF4D6AE0D4A0D48137803F1020C00F803A082F800C0124A0133127883E591
S34500018600114B1A884FF6FF739A421FD100233370BFE600BF937200209B720020DD720020DF720020DE72002000B00640987200209772002096720020943F0020903F002093
S34500018640FA5A0020227300205C4B00208848DFF860C20278531CDBB24FF0080E0CF802E0037029B98349D1F800E08349C1F800E03D32DFF84092D2B200214FF6FF7A39F8AE
S3450001868002EBD64504D100293FF483AE037080E64FEA1E2B0CF803B0591C0233C9B2DBB293420CF801E04FF00101E8D1EEE7332B01D0362B03D1082388F8003080E6342BF8
S345000186C003D0373B012B3FF67DAE2823F4E713F020033FD1694A1278032A7FF46FAA684A684916780978452E19D150785A2816D190784D2813D1D078412810D11079582854
S345000187000DD105293FF65AAA227942F0200222715D4A13805D4A002918BF33465DE62379594843F020032371584B00271F70078000293FF443AA06291E707FF63FAA937957
S34500018740038009297FF63AAA527A03EB02230380FFF734BA4E4A6379127903F0200313437FF42CAA4B4B1B78002B3FF427AA4A4B1A884FF6FF739A423FF420AA12F06EFF5C
S34500018780FFF71CBA2079800601D502209877237B13F040001FD06FF38613237301231370344B4FF47A721A603C4B04221A8085E50D2010700320E9E70420E7E701201070AC
S345000187C02C484FF47A7606603448042606800520DCE70020DAE7637960F341032C486371007913780343887903437FF467AD03231370FE232B7032238B715FE50A2D3FF439
S3450001880079A9274BDA7802F07F02DA70DA7802F0BF02DA70DA7842F02002DA70002388F800306423FB7049E5CB78002B7FF4C6A91C4A1378002B7FF4BDA923791A4E6FF3B1
S34500018840C30323712B78FF2B7FF4DBA933780B2B7FF4DDA915490B78002B7FF402AA2B703E20FFF795F80B7801330B70FFF7CFB9DD720020943F0020903F0020DC720020E3
S345000188809B720020DB720020F45A00208F720020035E002094730020CE5A0020FA5A002000B00640E25D00205973002020730020DF7200205C4B002008B5104B104A002165
S345000188C01970104B1970104B1970536B43F4006353636020FFF75CF80C4B2C22597199709971DA7008229A71094B202283F8212302225A60BDE80840FFF728B8DE720020E1
S3450001890000800440DD7200202073002000B0064000E100E0F0B5424BDA78140627D541490A78A2B93E4BDA7802F07F02DA70DA7842F04002DA703C4A002313703B4A1370B6
S34500018940374B1A7912F02F0F00D0DB79F0BD18790006F5D53448013AD2B20A7001784C1C04703348415CD971002AE9D1DAE7DA7812F0400208D0DA7802F0BF02DA70DA7849
S3450001898042F02002DA70E1E71979C90708D5DB79254B1A70254A137843F002031370D5E71A799206D2D5204DDB792A783F2A09D8D9B213431FBF531C2B701D4B99541D4B47
S345000189C000221A701C4C1D480323E370C37A13F00407BBD116492A7891F900500E78002D03DA042AB2D1E770B0E74D7805F1040C624502D1082EF6D1A8E7032AA6D10279AD
S34500018A0012F02002A2D1032EA0D1FF2D9ED18978412901BF43F00203C372094B9A7695E700B00640DD720020DE7200209A720020DF720020E25D0020035E00207A73002084
S34500018A405B73002013B55B4C6378062B00F2AF80DFE803F00414375F839DA800564BDA781AB9012262700622DA70544A1389117A534A1B0A1170537002B010BD0021514804
S34500018A8000916A46ADF8041019F05FF900214D4819F06AF90106F9D54A4B4B4A1B6913804A4A127B52075EBF1B015622B3FBF2F3424A54BF9BB200231380637801336370DA
S34500018AC0D3E700214FF480733E4800916A46ADF8043019F03AF93B48002119F045F90006F9D5384B1A69384B1B8811B29942D8BF9B1A364A127BD4BF1BB2002351075CBFAA
S34500018B003E2293FBF2F32D4A54BF9BB232235380D3E71A2300212B4800936A46ADF8041019F013F92748002119F01EF90206F9D5244B1B69B3F57F7F99B20CD2C3F57E73CF
S34500018B400333B3F5007F34BF5B08FF23DBB21B4AA371D180B1E70023F9E71B230021194800936A46ADF8041019F0EFF81548002119F0FAF80306F9D5124B1B69642253432E
S34500018B8040F2D942B3FBF2F30C4A938095E732232373A379312B05D8C3F13203DBB29B0032332373094A937843F002039370002385E700BF5B730020E85D0020FC5A0020ED
S34500018BC000C00C4000B00340285B00207A730020174B012230B59A70164A174CD36A174D43F48053D362164B85B0C02283F8212001A819F03FF8204601A914F0C3FB236A2C
S34500018C0023F04003236220460E4C19F04BF8A378002262F341036A70A370A3789B0703D532232B7305B030BDFFF70CFFF5E700BF00D007400080044000B003405B73002001
S34500018C4000C00C407A7300202C4B2D489A6B42F4007210B59A639A6B42F480629A639A6B42F400629A639A6B42F480529A639A6B42F400529A63234A4FF4407100249161BA
S34500018C80D161016041601C6100F532204FF40073136053609360D360F023C0F8D4304FF48073136153619361D361A2F5005240F203114465116051609160D1601164516418
S34500018CC09164D16440F2FF52C0F894200E4A136053609360D360136153619361D361136293624FF481735162D362084B44614FF4A0725A609A605A6110BD00BF00800440CB
S34500018D0000D0044000C0044000B0044000900440024B00221A6026225A61704700F00F40014B00225A61704700F00F4008B50F4B0F4A5A640F4814F06BFD0F4B0F4A1A602D
S34500018D4000221146022014F009FD0D4A1378002103F0C703137008460A4A14F0B3FD0A4814F0DCFB094B0A4A1A6008BD0080044000000713642003003C4A00200024F40077
S34500018D8000400640022A03006C200300B801002000389C1C2DE9F7439B4C2378063B5C2B9EBF9A4B64221A710CF040F823782A2B05462ED82A2B2FD8DFE813F035006C0076
S34500018DC08100A800B600D300E5002E002E002E0005011B017B0184012E00B101C401D001E501F50111022E00330239024B02550270022E002E002E002E002E002E00760283
S34500018E008C02CB02E2022E002E002E00E60206031803632B00F0F882202D67D0012D6DD12378632B61E046200CF03EF97849794E02467948FEF770F9754930700246764818
S34500018E4016F051FF3070FDF779FD744B1B888BB9734B1B78002BDFD11B200CF025F9714902467148FEF758F9704B1870FDF794FD632306E06E4B93F90430002B03DA237813
S34500018E8001332370C8E76B4A002313706A4A15201370E2E7614B1A8840F2EE439A420BD1664B1B78422B07D8624A594900231370614A1370624AD4E7FEF718FADFE75C4BAF
S34500018EC0DA78082842F01002DA7001D0042809D11A78C2F34001C94361F341021A70012323700BE001280CD0202807D1554B02221A704F4B1A786FF300021A7003B0BDE848
S34500018F00F0831B789A07F9D50323E9E74E494F480A2217F08BFE08B117209EE74C4B01221A7023781344ACE7424B404F002611201E700CF0B9F83B4902463B48FEF7ECF8C1
S34500018F40384938700246384816F0BFFE3A4B38701E70FDF721FD2378013323703D4B1E705AE7334E337A5B0701D5062389E70EF037FE00283FF450AF0228F6D1337A43F053
S34500018F8004033372F1E7254B33491A882F480BF0F1F80028C0DB294B30491A782B480BF0E9F82F4A002313702E4A1370204AD17963F30001D171FEF7ADFB2B4B4FF4FA6293
S34500018FC01A600A235DE71C4F274B2849284800263E7000961B883246FEF702F9214A387001231370234A1380234B1E701C4B1E7045E7214B1B78012B42D1204B1B78012B0D
S345000190003ED10C233DE700BF92730020035E00206975002068750020A9750020F45A0020A470002067740020A7740020667400207A730020E7740020E57300208F72002036
S34500019040052A030094730020152A03007018FF1FEA71002090720020222A03002E2A03009472002059730020943F0020E673002026740020FA5A0020DC720020DB720020DA
S34500019080994B1B78FF2B09D1984B1B78022B0CD1974A1368643313600D23F2E6052B04D8944B1B78002B7FF4B7AE0F20FEF7C4FADEE68E4B8E4A1B7812888F498F480BF091
S345000190C059F8DCE68A4B1A68511C19600A212170A2F63301B1F5617F0BD24FF47A721A601A68A2F61C42B2F5C87F09D240F6AC5213E0A2F24B41B1F5617F08D200221A6001
S345000191001B68B3F5616FFFF487AE0F23B9E6633AB2F5617FE4D240F6B8321A607CE6784B5A786FF345125A70764B774A1A60774B02F533721A60764A00231360754A1360EA
S3450001914010239EE66B4B09221A70734A00231380724A1370644A1370112392E66F4B1B78092B05D16E4B1B780A2B01D9142388E65D4B1B78052B04D85E4B1B78002B7FF4BF
S345000191804BAE12237DE65B4A01231370624A1380574B4FF42F621A60604A00231370524A137013236DE65D4B1B78012B05D15C4B1B78012B01D1162363E64B4B1B78FF2B5A
S345000191C00BD14A4B1B78023B012B3FF66EAF484A136864331360282353E6032B5FE7484A4849537843F020035370404BD3F8012012BA0A60D3F80520444912BA0A601A78A1
S34500019200022AD8D9B3F80D10DA7BD3F8113049BA02EB01223E4912020A603E4A1BBA1360C9E7384B1A68324B1A6017232370304A3649136809688B423CD328232370354BA1
S345000192401B68002B3FF4E8AD314B1B681360212317E6324B1B78352B70D1314B1B78202B6CD119230DE6224B2E491A6823481F4FDFF8C490DFF884800AF07CFF202617F838
S34500019280012B49464046013E0AF074FF16F0FF06F5D1254919480AF06DFFF0E5144A1368203313601723ECE5114B1A4A1B681268934290D21D4F1E491E48002632463E70BC
S345000192C0FEF7F0F80B4B387035221A70124B20221A8089E6114B1B78352B2FD1104B1B78202B2BD12323CCE5947200209B720020943F0020597300203C2A03007018FF1F47
S345000193007A730020C840002000FC1300C4400020C0400020BC400020FA5A0020DC720020DB720020452A0300CD2D0300E5730020E6730020267400204D2A0300354B1B788C
S34500019340032B04D8344B1B78002B7FF465AD1320ACE6324B32491A683248334FDFF8F890DFF8C0800AF006FF202617F8012B49464046013E0AF0FEFE16F0FF06F5D188E75F
S34500019380264A1368203361E7284926480AF0F2FE244818F014F888B11A200BF085FE244902462448FDF7B8FE234B1870FDF7F4FA63232370214B00221A702DE518F057FCA5
S345000193C023780133DBB2F4E720200BF06DFE1C4902461C48FDF7A0FE1B4B174A1870002313701A4A1370FDF7D7FA48E5184B1B78602B3FF43DAD0EF063FC00283FF40CAD09
S345000194006020FEF7C5FA07E5124AD37843F02003D37001E59472002059730020943F0020522A03007018FF1F9B7200205A2A030067740020A774002066740020EA71002056
S34500019440E874002028750020E7740020E5730020217300207A7300204D2A0300204A1378012B17D0022B21D00BB1002070471D49487863F3451048701B491C4808601C49A7
S3450001948000F5337008601B490B601B490B6001231370EAE7194B09211970194900230B8018490B7018490B700223F1E7154B1B78092B0AD1154B1B780A2B06D9094A53788C
S345000194C043F020035370012070470F4B1B78052BF9D80A4B1878B0FA80F04009704700BF8F7300207A730020C840002000FC1300C4400020C0400020BC4000205973002016
S34500019500FA5A0020DC72002094720020DB7200202DE9F041494C2378A3F11F02082A3DD8DFE802F00512253E4B5F7B797900444B09221A70434A00231380434A1370434ACE
S3450001954013702023237029E03F4B1B78092B05D13F4B1B780A2B01D92123F3E73B4B1B78052B02D8364B1B78C3B92823EAE7394A3949537843F020035370384AD2F80130DC
S34500019580D2F805201BBA0B60354912BA0A60354993420B604FF022012170E6D2BDE8F081274B35221A70274B20221A80264A00231370264A13702323C4E7234B1B78352B46
S345000195C005D1234B1B78202B01D12423BAE71F4B1B78032B03D81A4B1B78002BDED13223B0E7204B20491A6820481C4EDFF888801E4F0AF0BFFD202516F8012B4146384616
S34500019600013D0AF0B7FD15F0FF05F5D1184917480AF0B0FD2378013394E7124A136820331360222222700E4A12689342B6D311490E480AF09FFD262384E700BF9273002036
S3450001964059730020FA5A0020DC72002094720020DB7200207A730020C84000209B720020C4400020943F0020452A03007018FF1FCD2D03005A2A03004D2A030030B5174CAB
S34500019680174D2378E95CA1F13002D2B2581C092AC0B205D9A1F14102052A15D83739CAB2295CA1F13000C0B2120102330928D2B2DBB205D9A1F14100052806D83739C8B25A
S345000196C01044C0B2237008E003462370054B12221A70054B64221A70002030BD18710020ED710020EC71002092730020F0B50D4DDFF834C02E8800231F464FF0060E10FA9D
S3450001970083F416FA83F28B42A4B292B203D10FB133442B80F0BD0EFB02F201332CF802400127ECE7B45A0020D005FF1F2DE9F7438B4C0BF07BFB2378322B054636D8322B63
S3450001974037D8DFE813F03D0073008A00B1003B01360036003600360036009E0185008A00AE01DC01E801FD01240230024F0263027302BD02CC02DE02ED0236003600360032
S345000197803600F80219035603A003A70336003600360036003600B503E703390449045A04360036003600360036006504642B00F03C84202D68D0012D6ED12378632B62E005
S345000197C047200BF071FC6749674E02466748FDF7A3FC644930700246644816F084FA3070FDF7ACF8624B1B888BB9624B1B78002BDFD11B200BF058FC5F4902465F48FDF7E3
S345000198008BFC5F4B1870FDF7C7F8632337E15D4B93F90430002B02DA237801332FE15A4A00231370594A15201370E3E7504B1A8840F2EE439A420BD1554B1B78422B07D883
S34500019840514A484900231370504A1370514AD5E7FDF74CFDFDF7A0F8DEE74A4AD178082841F01001D17001D0042809D11178C1F34000C04360F341011170013B23700BE056
S3450001988001280CD0202807D1434B02221A703D4B1A786FF300021A7003B0BDE8F08312789007F9D50133E9E73C493D48012217F0BDF93C4B00261E8060B148200BF0F4FBE2
S345000198C02D4902462D48FDF727FC2D4B18702F4B1E7098E7344B01221A700EF04BF9334B1B78062B04D8324B0B221A706423C6E0304E3378502BF6D17378472BF3D1B378EC
S34500019900542BF0D1F3783D2BEDD133794D2BEAD1294F05233B700BF019FF3B78F35C13B1234B0C22E1E7124BB0F5837F1B8804D140F2EE4293423FF46FAF98423FF46CAFBC
S345000199402F200BF0B1FB0C4902460C48FDF7E4FB0B4B0D4A1870002313700C4A137052E7927300206975002068750020A9750020F45A0020A470002067740020A774002003
S34500019980667400207A730020E7740020E57300208F720020052A030094730020152A03007018FF1FEC5A0020EA710020EB710020EC710020ED710020187100200EF0DAF873
S345000199C0A24B1B78062B8ED9A14E3378502B8AD17378472B87D1B378542B84D1F3783D2B81D13379562B7FF47EAFDFF8CC82052388F800300BF0AAFE98F8003016F8038041
S34500019A000746B8F1000F8BD1DFF8B09299F80030834233D249200BF047FB8E498E4E02468E48FDF779FB8E4B8A4983F800808D4B3070024683F8008088488B4BFDF7B6FB8E
S34500019A404FF001083070CDF80080024699F8003080498248FDF7C4FB844B7E49307002467E48FDF7A3FB7B4930700246CDF800807A483B46FDF7B4FB3070C4E60A232370AC
S34500019A8097E67B4B1A781E206FF341021A700BF00BFB704902467148FDF73EFB6E4B1870D8E64A200BF000FB6A496D4E02467148FDF732FB6749307002466E4816F005F934
S34500019AC0654B307000261E70664B1E70FCF764FF694B1E70694B1E70694B1E80644B5A7866F345125A70674B674A1A60674B02F533721A60664B1E80664B1E808CE65F4B96
S34500019B0009221A70644A00231380644A13705A4A13700F23B3E7614B1B78092B05D1604B1B780A2B01D91023A9E7534B1B78052B04D8524B1B78002B7FF43BAE14239EE7D8
S34500019B404B4A5349537843F020035370554BB3F8092052BA0A80B3F80110DA7849BA02EB0122484912020A60D3F80520474912BA0A601A78012A04D9B3F80B30454A5BBAB5
S34500019B801380494B4FF416621A60112377E73B4A01231370404A1380404A00231370364A137012236BE73D4B1B78012B05D13C4B1B78012B01D1132361E72F4B1B78FF2BC3
S34500019BC005D1384B1B78022B08D11E2357E7052B04D82A4B1B78002B7FF4EBAD0F20FDF72BFD12E62F4B304F93F900303E68002B05DBA6F5C870012180B2FFF777FD013632
S34500019C0040F6C3139E423E60DFD8BEE7274A4FF6FF731380264A1380264B01221A80164A00231370154A1370152328E7214B188811F080FC022803D800283FF4BAADEBE5FC
S34500019C40FF287FF4B6AD0C20C9E700BFEB710020ED7100206774002066740020A7740020E7740020E5730020602A0300632A03007A7300202875002094720020597300202F
S34500019C80B45A0020C840002000FC1300C4400020C05A0020BE5A0020FA5A0020DC720020DB7200209B720020943F0020C45A0020C25A0020E85A0020187100208F7200208D
S34500019CC09F4B588848B111F0A9FD9E4B18604FF6FF739842B0D10D2081E71923CFE6984E994BF2881A80974B186811F09FFE974B1B78013B022BF0D87089002111F060F803
S34500019D008AE5012011F09AF801283FF485AD632804D000283FF44DAD13206BE5207048E5894B8B4A1B881380012B3FF44EAF002B7FF47AAFF0E7874B874F00261E70874B70
S34500019D401E70874BDA7966F30002DA71FDF7E2FC11200BF0A9F9834902468348FDF7DCF9804938700246804815F0AFFF7F4B38701E707F4B1E706DE57E4F0DF0FBFE012376
S34500019D803B707D4B1B780BB9322378E67B4E3278412A1AD1032B1ED90BF0D8FC784B18603B78F25C3D2A0DD101333B700BF0CEFC744B18703B78F35C002B3FF42DAD724BFF
S34500019DC0102292E5704B0F228FE5242A03D1482B01D1282353E66D49684817F015FF0028D2D13378212B01D11F2348E6664B13227BE5634B1A68A2F57A73632B28D8644BAC
S34500019E001B889A4222D0591C8A421FD00233991A4B424B415F4909888A4207D0481C824204D002318A4201D0002BDDD04B4A1378002B7FF4BEAC02211170574A01211180D9
S34500019E40564A1370434A1370212318E60123E1E7A2F5FA63632BE9D8514BDFF858C11E88002319464FF0060ED8B2B04202D30029BAD0DBE70EFB00F001333CF80000824245
S34500019E8008BF0121F0E7454B1B78022B40F0AA802223F4E5364E3A4B424943480022327000921B88FDF79CF93070FCF775FD9BE7334E00233360FFF7E1FB00023060FFF75A
S34500019EC0DDFB3368184400023060FFF7D7FB3368184423783060632B3FF66BAC2549274E0A78B65C3D2E17BF274B01330F221A700CBFDBB2642323702C4B1B6804BF0132BB
S34500019F000A709842FFF470AF294B1B689842BFF46BAF4EE41B4F2026FFF7B0FB013E16F0FF0607F8010BF7D12378632B3FF641AC104A124912788A5C002A7FF440AF6CE42A
S34500019F40D05A0020CC4000202A5B002085710020E85A002094720020E7740020597300207A730020E87400202875002066740020E573002018710020EB710020ED7100205F
S34500019F80943F002022730020EC710020662A0300C05A0020BE5A0020FA5A0020DC720020B45A0020E673002026740020C8400020C4400020D005FF1F1E4A1378002B7FF45D
S34500019FC0F8AB362111701C4A202111801B4A13701B4A13702B2352E5184B1B78362B01D12C234CE5164B1B78052B04D8114B1B78002B7FF4DEAB0E20F1E5124B124E1B684F
S3450001A0001249134800223270FDF74CFA3070EBE620200BF049F80F4902460F48FDF77CF80E4B0F4A1870002396E403F039FFFFF7ECBB00BF59730020FA5A0020DC720020ED
S3450001A04094720020943F0020E5730020E673002026740020E874002028750020E7740020667400202DE9F341704C23780646642B00F29480DFE813F065005F015F0199005D
S3450001A080FE00560175015F015F015F017E0190019301B301ED01F9010E0231023D029F02B302C302D202E102F302010392009200920092000A032B03F2035D04630492004F
S3450001A0C0920092009200920072049F04B304D204E30492009200920092009200EE049200920092009200920092009200920092009200920092009200920092009200920006
S3450001A10092009200920092009200920092009200920092009200920092009200920092009200920092009200920092009200920092009200920092009200920092009200D8
S3450001A14028053B4B3B4F00251D803B4B72201D700AF0AAFF394902463948FCF7DDFF374938700246364815F0BEFD3870FCF7E6FB344B1B8853B91B200AF096FF3249024692
S3450001A1803248FCF7C9FF324B18704BE0237801332370304B1A7865F341021A70202E00F09A84012E40F00D8115E12B4B01221A700DF0E0FC294B1B78062B0FD9284D2B782C
S3450001A1C0502B0BD16B78472B08D1AB78542B05D1EB783D2B02D12B794D2B06D00B23214A6420137002B0BDE8F0811F4F05233B700BF0ACFA3B78ED5C0DB10C23EFE7114B66
S3450001A2001B88834200F096802F200AF04DFF0E4902460E48FCF780FF0D4B1870134B1D70134B1D70FCF7B8FB6320DBE719710020EC5A002068750020EC7500206975002080
S3450001A240A9750020F45A002067740020A7740020667400207A730020EA710020EB710020ED710020EC71002018710020E7740020E57300200DF07EFCA34B1B78062BADD9B1
S3450001A280A24D2B78502BA9D16B78472BA6D1AB78542BA3D1EB783D2BA0D12B79562B9DD1DFF8E082052388F800300BF04FFA98F80030ED5C0746002D9FD1DFF8CC8298F862
S3450001A2C00030834236D249200AF0EEFE9049914C02469148FCF720FF904B8D491D70904B207002461D708C488E4BFCF75FFF012520700095024698F8003085498648FCF7C4
S3450001A3006FFF894B8249207002468348FCF74EFF7F492070024600957F483B46FCF760FF20707FE70DF026FC8049784817F06CFC054618B12378013323702FE77C4A74493B
S3450001A3407548744EFCF7E8FE0446307049200AF0ABFE6F49034622466F48FCF727FF30705CE70DF007FC7349684817F04DFC0028E0D033E7704B1A781E206FF341021A7004
S3450001A3800AF092FE624902466348FCF7C5FE614B1870FCF701FBCDE7FCF7A8FFF9E7664BDA78082842F01002DA7001D004280AD11A78C2F34001C94361F341021A700B23EB
S3450001A3C0237000200EE7012840F082831B78980701D50D232370594B1B78632B79E34A200AF062FE4A494D4D02465548FCF794FE474928700246524815F067FC454B28706F
S3450001A40000251D70464B1D70FCF7C6FA4D4B1D704D4B1D704D4B1D80474B5A7865F345125A704B4B4B4A1A604B4B02F533721A604A4B1D804A4B1D80237801332370494B8B
S3450001A4401B78002B3FF4AAAE4749484809F092FEA4E63D4B09221A70454A00231380454A1370384A13700F2366E7424B1B78092B05D1414B1B780A2B01D910235CE7314BF7
S3450001A4801B78052B04D8304B1B78002B7FF486AE142351E7284A3149537843F020035370364BB3F8092052BA0A80D3F80120284912BA0A60D3F80520274912BA0A601A7831
S3450001A4C0012A04D9B3F80B30254A5BBA13802C4B4FF416621A6011232EE71B4A01231370234A1380234A00231370164A1370122322E7204B1B78012B48D11F4B1B78012BAF
S3450001A50044D1132318E700BFEB710020ED7100206774002066740020A7740020E7740020E5730020602A0300632A03006A2A0300762A03007C2A03007A73002092730020BC
S3450001A540287500209472002059730020B45A0020C840002000FC1300C4400020C05A0020BE5A0020E8710020892A0300D013FF1FFA5A0020DC720020DB7200209B7200205E
S3450001A580943F0020187100208F720020954B1B78FF2B05D1944B1B78022B08D11E23CBE6052B04D8914B1B78002B7FF4F7AD0F20FDF742F838E68C4B8D4F93F900303D68AE
S3450001A5C0002B05DBA5F5C870012180B2FFF78EF8013540F6C3139D423D60DFD87BE7854A4FF6FF731380844A1380844B01221A807C4A002313707D4A137015239CE67F4B90
S3450001A600188810F097FF022803D800283FF4C6AD90E6FF287FF4C2AD0C20C9E7784B588848B111F0FBF8774B18604FF6FF739842EBD10D20BCE719237EE6714D724BEA883B
S3450001A6401A80704B186811F0F1F9704B1B78013B022BF0D86889002110F0B2FB6AE6012010F0ECFB01283FF465AE63283FF4DCAD00283FF493AD13207EE5634B5F4A1B889C
S3450001A6801380012B8AD0002BB7D1F4E7554B604F00251D70554B1D705E4BDA7965F30002DA71FDF737F811200AF0FEFC5A4902465A48FCF731FD584938700246574815F0F2
S3450001A6C004FB574B38701D70564B1D7061E6DFF888810DF04FFA98F800300BB932232BE6514D2B78002B5CD15049514817F08CFA00283FF453AD01232B704E4B1B78002B2F
S3450001A70049D14D494A4817F07FFA00284DD14B4F00233B702B78002B3FF440AD98F80020434DBAB12B785B2B3FF438AD062A3FD94D2B4BD16B784F2B0CD1AB78442B09D146
S3450001A740EB78452B06D12B794C2B03D16B793D2B3FF424AD3A49364817F056FA0028BDD13849334817F050FA0028B7D10AF0EEFF1F4B18603B78EA5C3D2A31D101333B70D4
S3450001A7800AF0E4FF304B18703B78EB5C002B3FF4D1AD102323E52D4B2D491A882D4809F0E9FC2B78012BB2D1ABE702232B70AEE7D0D1432BCED16B78552BCBD1AB78532B37
S3450001A7C0C8D1EB78542BC5D12B79C0E7432BF2D0242BBFD1482ABDD101233B702823ABE50F23FCE4947200209B72002059730020943F0020C45A0020C25A0020E85A00201D
S3450001A800D05A0020CC4000202A5B002085710020E77400207A730020E87400202875002066740020E5730020EC7500209B2A0300ED710020E8710020AA2A030018710020ED
S3450001A840662A0300D82A030022730020EC5A0020BD2A0300D013FF1FEB710020A24DA34F2B784BB1A24BA34A1B7800933B681288A149A24809F07EFC3B68A3F57A72632AFF
S3450001A8801FD89F4A1288934219D0511C8B4216D00232D11A4A424A419A4909888B4231D0481C83422ED002318B422BD052BB1F2323702B78002B3FF471AC9349C5E50122F6
S3450001A8C0EAE7A3F5FA62632A1CD8904ADFF8A0E21788002211464FF00608D0B2B84208D381B91F2323702B78002B3FF457AC8849ABE508FB00F001323EF80000834208BFC0
S3450001A9000121EAE7834A1378002B7FF447AC02211170814A01211180804A1370804A137023780B4423702B78002B3FF437AC7D498BE57A4B1B78022B76D12223FCE47A4D29
S3450001A9406A4B7A497A4800222A7000921B88FCF747FC2870FCF720F81F23EDE4634D00232B60FEF78BFE00022860FEF787FE2B68184400022860FEF781FE2B6818446D4B45
S3450001A98028601B78632B3FF609AC6B4A6B491378C95C3D297FF424AF01331370237801332370674B1B689842D6D3664B1B689842FFF4F4ABD0E74E4F2025FEF75FFE013D9E
S3450001A9C015F0FF0507F8010BF7D15A4B1B78632B3FF6E4AB584B594A1B78D35CD6E64D4A1378002B7FF4DAAB362111704A4A202111804A4A13704A4A13702B2323703A4B0F
S3450001AA001B78002B3FF4CAAB384B3A4A1B6812884D493A4809F0AEFBFFF7C0BB3F4B1B78362B01D12C2387E43D4B1B78052B04D8384B1B78002B7FF4B1AB0E20B8E52B4BD8
S3450001AA40394D1B6839493A4800222A70FCF72AFD287081E73D4B3E4C002520201D700AF023FB3C4902463C48FCF756FB2E4B20701D703A4B1B78012B024616D8354936482F
S3450001AA8015F023F90546207013200AF00DFB314903462A463048FCF789FB314B207002462C492D48FCF782FB2070FBF775FF0E4B1B78002B3FF4B8AB0E4B2A491A880F4826
S3450001AAC009F058FBFFF7B0BB03F0EAF9FFF7ACBB20287FF476AC244B02221A70234B1A786FF300021A706CE4E8710020943F002022730020EC5A0020E62A0300D013FF1F9C
S3450001AB00C05A0020BE5A0020FD2A0300B45A0020072B030059730020FA5A0020DC72002094720020132B0300E5730020E6730020267400209273002018710020ED710020E3
S3450001AB40C8400020C44000201B2B0300E77400206674002067740020A7740020EC750020E23A0300302B0300947300207A730020D005FF1F014916F0D6BF00BFD013FF1FC4
S3450001AB801B4B37B51B4A1968914284BF00221A601A68684606230A24013BB2FBF4F113F0FF0304FB112200F8012B0A46F4D10DF10605052415F8010D013C3030C0B2E4B2ED
S3450001ABC0FFF7D8FFFF2C05D12C2003B0BDE83040FFF7D0BF022CEDD12E20FFF7CBFF15F8010D3030C0B2FFF7C5FF0124E2E700BFD80900203F420F0038B5064D0309044672
S3450001AC0004F00F04E85CFFF7B5FF285DBDE83840FFF7B0BFC22B0300184B5B7A03F0C003402B70B528D0164B1B782BB3FFF7A8FF2020FFF79FFF5420FFF79CFF114D124EA5
S3450001AC403A20FFF797FF00232A789A4207D80D20FFF790FFBDE870400A20FFF78BBFF05C5C1CFFF7C9FF2B78E4B2A34202D92D20FFF780FF2346E7E770BD00BF7A73002089
S3450001AC80E8710020DD720020DF7200201C4B5B7A03F0C003402B70B5044630D0194B1B786BB3FFF76DFF5220FFF764FFFF2C0AD13F20FFF75FFF0D20FFF75CFFBDE870409A
S3450001ACC00A20FFF757BF104B104D114E04F00F04185DFFF74FFF3A20FFF74CFF00232A789A42E8D9F05C5C1CFFF786FF2B78E4B2A34202D92D20FFF73DFF2346EFE770BD20
S3450001AD007A730020E8710020C22B0300DD720020DF7200202DE9F0411C46214B069D1B7880460E461746002B38D01E4B5B7A5B0634D5FFF725FF1C491C4809F01BFA4046A2
S3450001AD40FFF718FF06F13000C0B2FFF713FF5820FFF710FF3A20FFF70DFFC7F30720FFF74BFFF8B2FFF748FF2F20FFF703FF104B185DFFF7FFFE3D20FFF7FCFE2C44A5428F
S3450001AD8007D10D20FFF7F6FEBDE8F0410A20FFF7F1BE15F8010BFFF72FFFF0E7BDE8F081E87100207A730020442B0300D013FF1FC22B030010B52E4B1B780446002B55D07A
S3450001ADC02C4B5B7A5B0651D5FFF7DAFE2A4B1A88002C49D029492A4C2A4809F0CBF92A492848224609F0C6F994F85030BBB12749244804F1500209F0BDF994F8A03073B16B
S3450001AE002249204804F1A00209F0B4F994F8F0302BB11E491B4804F1F00209F0ABF91C4C2378012B05D11B4B1B491A68154809F0A1F92378032B07D1184B194A1B68126880
S3450001AE401849104809F096F92378042B04D1164A16490C4809F08EF90D20FFF78BFEBDE810400A20FFF786BE1149B4E710BD00BFE87100207A730020EC5A00204B2B03006D
S3450001AE80256F0020D013FF1F642B0300632B0300BD600020740D0020672B0300040B0020080B00206D2B0300D36E0020762B0300572B030008B50B4B1B7893B10A4B5B7AA5
S3450001AEC05B060ED5FFF75CFE084B09491A88094809F050F9BDE80840074A0849054809F049B908BDE87100207A730020EC5A00207C2B0300D013FF1FED710020052E0300F6
S3450001AF0010B50F4B1B780446CBB10E4B5B7A5B0615D5FFF735FE0C4A0C4912880C48234609F028F90B4B0C491A68094809F022F9BDE81040094A0A49054809F01BB910BDC0
S3450001AF40E87100207A730020EC5A0020892B0300D013FF1F740D0020A02B0300D36E0020B12B030070B5ECB00146044610A816F03EFB034600283AD169460D46E25C5E1CF8
S3450001AF800ABB2F21E954AA5524A910A816F07CFB10BB9DF8AA30FBB10DF1A901AA1911F8013F02F8013B002BF9D19DF89C30DB060DD4284616F017FC0028E5D10D4A5388B8
S3450001AFC001335380E0E701F8012B3346D6E72846FFF7C8FF0028ECD0204616F004FC18B9044A53880133538010A816F044FB00206CB070BD065B002070B52F4D2F4EEEB002
S3450001B0002F23ADF8043095F904300024A342748050DA012201A9204608F068F92B79214664F3C71320462B710BF08AFC95F90430A3423FDA224912A816F0D9FA002839D1BA
S3450001B04026A912A816F020FB044680BB9DF8B2306BB39DF8A43003F01403102BF0D1738863B102A826AA631C1444DBB2A27EC254DAB92F230370FFF775FFE1E7114B124A31
S3450001B080187012491248FCF747F8124B1870124B1C70FBF781FC2B7964F341032B712B799B07DED4FBF730FDF9E71C46DAE712A816F0E1FA6EB070BD7A730020065B002074
S3450001B0C0F2250300E7740020D32B0300E8740020A774002066740020E573002010B5002009F0E2FF002102460F48FCF715F80F4B1870FBF723FC432009F0D6FF0C4902464A
S3450001B1000C48FCF709F80C4B18700C4B00241C70FBF714FCFBF740FC094B1C70094B1C80094BFF229A7510BDA975002068750020E8740020A774002066740020E573002025
S3450001B140EF750020F85A0020E85D0020014B02221A707047EF7500202DE9F74F9A4D9B4C2B78032B1EBF9A4A0021117022780B2A0FD80B2A10D8DFE812F0120017003900DC
S3450001B1808800F5005301890105020F000F0018023202642A00F0298203B0BDE8F08F0123237000232B70F7E78A4A11780B2919D100231370884B1B78042B10D1874B1A786C
S3450001B1C0542A0CD15A78452A09D19A78532A06D1DB78542B02BF824B43F239021A8002232370D9E7002BD7D10B23DBE7794A11780D2935D100231370774A1278112ACBD177
S3450001B2007649784A08781070774A784D16461F464FF0010C11F8010F02F8010B10F0800F1CBF803802F8010C12F8010C05F8017B03F1010318BF05F801CCDBB2002808BF06
S3450001B2402020102B02F8010CE4D1202333747374674B12221A70FBF771FB23780133BFE77BB95F4A108843F23901884207D1614991F904100029AABF6423138023700D233F
S3450001B28090E75D4B32229A7186E7524A11780E2964D1514B1B780020112B10707FF47CAF4E4A564913780B70802B37D109F0FCFE5349544D524E544F02465348FBF72CFFFF
S3450001B2C0524B4F49287002464F48FBF76FFF0223024628704A4900934B4840F22953FBF77FFF02460F2A2A7012D9474B20221A745A74444B12221A70454A00231370454A18
S3450001B3001370FBF749FB444B1A7B3B4BDA71A4E73146384614F0D9FC0246E3E73A4B384D0646012712F8011F03F8011B11F0800F1CBF803903F8011C13F8011C05F8016B61
S3450001B34000F1010018BF05F8017CC0B2002908BF2021102803F8011CE4D1C6E7002B90D10E231FE7002B7FF417AF1A4B1B780C2B3FF435AF284BDB7B5F0601D505232FE77F
S3450001B38009F054FD86060BD00C232B70234B187012287FF401AF184BFF22DA740A231FE7104B1B782BB1144BDB7913B902232370EEE7124B1B78002BEAD00F4BDB79002B2F
S3450001B3C0E6D10323F3E700BF59730020EF75002094720020DC720020DB7200209B720020F85A0020EE750020A975002069750020687500207A730020E85D0020ED75002010
S3450001B400E8740020E774002028750020602A030066740020E57300205B730020227300203E2009F041FE7A497A4E02467A48FBF773FE774930700246774814F054FC3070C6
S3450001B440FBF77CFA112009F02FFE7449744E02467448FBF761FE744A307000231370734A1370FBF799FA724BDB7B13F00C0F01D1180608D5272009F017FE6849024669486C
S3450001B480FBF74AFE3070237801332370684FFB7B13F00C0F7FF480AE19063FF57DAE2E78002E4DD1634B1A78042A66D1DFF8A4A11E709AF80030012B42D95F4BDFF860B103
S3450001B4C093F80090B9F1000F42D0DFF858815B4A52494046FBF720FE8BF800004FEA191014F00FFC88F80100484614F00AFC88F803004D48524A50499AF800C00023037097
S3450001B5004FF0010E90464FF0800A5FFA8EF9CC4521D833B1BCF1000F0CF1FF3308BF002303700278002308F80230404A13700EB1FBF732FA434B3A7BDA7123780133237058
S3450001B540FB7B13F040037FF427AE0222227029E68BF80060CDE74B780BB981F801A011F8013F92F8009002F8013B99451CBF0136F6B20EF1010E0123C7E704232B70324B73
S3450001B5801E70DDE72A4BDB7B5A067FF528AE13F00C0F7FF4F3AE1B063FF5F0AE294BDB79002B7FF4F9AD06231AE6284A18491A48184EFBF7B1FD05463070272009F074FD8C
S3450001B5C02A46034612491448FBF7F0FD164A307000231370124A1370144A13703DE6194BDB7C002B3FF4FBADD6E50949184A0A48FBF792FD074B0C4A187000231370084A41
S3450001B60013700A4A1370FBF799F9FBF7C5F924E66975002068750020A9750020E8740020E77400202875002066740020E57300205B730020DC7200209B720020DE2B030077
S3450001B640A7740020E85D002022730020E42B0300EB2B0300DB720020144A01231380144A1380144A00231370134A1370134A1370134A1370134A32211170134A517821F0C4
S3450001B6800A01517011490B7011490B7011490B70117A21F0030111720F4A19460133DBB21E2B22F8021BF9D1704700BFE85A0020E45A0020F975002087730020F2750020ED
S3450001B6C0F1750020FA7500207A730020F8750020A8700020F7750020984B0020034B03221A70034B01221A70704700BFFA750020F575002010B5074B074A1B781278D342AC
S3450001B70006D0064C06492278064814F0DEFA207010BD00BFE774002066740020E5730020E673002026740020F8B5584C584F2378584E0C2B14D8DFE803F0072956812992B3
S3450001B7409F13131356A39F0001232370524B00211970C8237B72514BDA7961F30412DA717B7A63B94D4BDB79DB0608D5FF2323704B4B4FF6FF721A804A4BFE221A70337898
S3450001B780FF2B02BF444B00221A70F8BD464A11780B2920D100201070444A1278042A15D1434A1178542911D1517845290ED1917853290BD1D278542A08D1384A517960F371
S3450001B7C0C71151713B4A43F23901118001332370C8237B72C4E7304A1378002BC0D10B2111703370BCE730490A780E2A20D1013323702E4B1B780022112B0A70B0D12C4D5C
S3450001B8006B7B202BACD1EB7B202BA9D12B7C202BA6D129496A73681C16F0F6F900289FD0AB7B264A303B137023780133237097E7194A1378002B93D10E21D1E7164A1378AD
S3450001B840002B8DD1184909780C2901D10223EDE70C2133701A4B117002221A7080E7124B1B780D2B01D10623E0E70B4B1A78002A7FF476AF0D22F0E7642323700023B0E71D
S3450001B8800E4B63221A706523D0E700BFF9750020E85D002094720020597300207A730020E85A0020FA750020DC720020DB7200209B720020F85A0020FC2B0300B97000202B
S3450001B8C02273002030B52B4B89B001AA03F1180518685968144603C40833AB422246F7D11868254920600A78012A1FD1234B1878432817D158784F2814D19878442811D19C
S3450001B900D87845280ED1187920280BD15879302808D19879302805D1D879302802D11B7A302B1AD000230B7009B030BD531EDBB21C2BF7D820336B4413F81C0C0028F3D0A0
S3450001B9400F4B1C780C2C0AD101320A700D4A002018701378023B1370E6E70023EAE70A4A1378002BE0D10C211170084A1070084AF1E700BF2A2C03008773002028750020B3
S3450001B980DC720020FA75002059730020227300209472002010B5204B1A78FE2A22D1FF2238201A7009F080FB1C4902461C48FBF7B3FB1C4B1870FAF7C1FF1B4B0024392034
S3450001B9C01C7009F071FB194902461948FBF7A4FB184B1870184B1C70FAF7DEFF174918480AF0E6FE09F022FA202813D1FFF776FBFFF732FEFBF7AAFF0A4A002313700A4AB6
S3450001BA0013700C4A13700C4A13700E4A517963F3C711517110BD00BFFA75002069750020A975002068750020E774002067740020A774002066740020E5730020F225030027
S3450001BA40092C03007A730020102822D004D8012822D0022803D0704720282BD070471E4BDB88002B36D01D4A118899421CBF13801B4B1C491CBF00221A701B4B0870002213
S3450001BA8001281A70194B18D0597862F3410159707047114B9B88E4E714490F4A497853898907DED51389124A0A211170114AC8215172D6E7084B1B89D3E702200870597834
S3450001BAC062F34101CAB25970C90742BF22F0030202435A70704700BFD05A0020E85A00201B710020F1750020FA7500207A730020F9750020E85D0020102838B504460AD13F
S3450001BB001D4A13780BB1013B13701C4B1C701C4B00221A7013E0022807D1174A19491378897B9942F1D90133EEE708280AD007D8022802D8012802D1E7E7042802D038BDEC
S3450001BB402028F8E70F4DA8894FF6FF739842DCD0A97B0029D9D0FBF793FEAB89A3F5FA639BB2632BD1D8FBF7D5FD074BDA796FF30002DA71C9E700BF1B710020F2750020ED
S3450001BB80FA750020D05A00207A7300200E4A30B5014604460B1BD8B2155C15F0DF0302D10B7020B930BD01F8015BF3E7545450FA83F4E4B2D9B2145D0133002CF6D1034B0F
